
SDI_MainApp.elf:     file format elf32-avr

Sections:
Idx Name          Size      VMA       LMA       File off  Algn
  0 .text         0000278c  00000000  00000000  00000094  2**1
                  CONTENTS, ALLOC, LOAD, READONLY, CODE
  1 .data         000000b6  00802000  0000278c  00002820  2**1
                  CONTENTS, ALLOC, LOAD, DATA
  2 .bss          0000028a  008020b6  008020b6  000028d6  2**2
                  ALLOC
  3 .comment      00000030  00000000  00000000  000028d6  2**0
                  CONTENTS, READONLY
  4 .note.gnu.avr.deviceinfo 00000040  00000000  00000000  00002908  2**2
                  CONTENTS, READONLY
  5 .debug_aranges 00000528  00000000  00000000  00002948  2**0
                  CONTENTS, READONLY, DEBUGGING
  6 .debug_info   00008aa0  00000000  00000000  00002e70  2**0
                  CONTENTS, READONLY, DEBUGGING
  7 .debug_abbrev 00001ddf  00000000  00000000  0000b910  2**0
                  CONTENTS, READONLY, DEBUGGING
  8 .debug_line   0000806d  00000000  00000000  0000d6ef  2**0
                  CONTENTS, READONLY, DEBUGGING
  9 .debug_frame  00000e38  00000000  00000000  0001575c  2**2
                  CONTENTS, READONLY, DEBUGGING
 10 .debug_str    00031993  00000000  00000000  00016594  2**0
                  CONTENTS, READONLY, DEBUGGING
 11 .debug_loc    0000378c  00000000  00000000  00047f27  2**0
                  CONTENTS, READONLY, DEBUGGING
 12 .debug_ranges 000004c0  00000000  00000000  0004b6b3  2**0
                  CONTENTS, READONLY, DEBUGGING
 13 .debug_macro  0000b3ed  00000000  00000000  0004bb73  2**0
                  CONTENTS, READONLY, DEBUGGING

Disassembly of section .text:

00000000 <__vectors>:
       0:	0c 94 2d 01 	jmp	0x25a	; 0x25a <__ctors_end>
       4:	0c 94 53 01 	jmp	0x2a6	; 0x2a6 <__bad_interrupt>
       8:	0c 94 53 01 	jmp	0x2a6	; 0x2a6 <__bad_interrupt>
       c:	0c 94 53 01 	jmp	0x2a6	; 0x2a6 <__bad_interrupt>
      10:	0c 94 53 01 	jmp	0x2a6	; 0x2a6 <__bad_interrupt>
      14:	0c 94 53 01 	jmp	0x2a6	; 0x2a6 <__bad_interrupt>
      18:	0c 94 53 01 	jmp	0x2a6	; 0x2a6 <__bad_interrupt>
      1c:	0c 94 53 01 	jmp	0x2a6	; 0x2a6 <__bad_interrupt>
      20:	0c 94 53 01 	jmp	0x2a6	; 0x2a6 <__bad_interrupt>
      24:	0c 94 53 01 	jmp	0x2a6	; 0x2a6 <__bad_interrupt>
      28:	0c 94 53 01 	jmp	0x2a6	; 0x2a6 <__bad_interrupt>
      2c:	0c 94 53 01 	jmp	0x2a6	; 0x2a6 <__bad_interrupt>
      30:	0c 94 53 01 	jmp	0x2a6	; 0x2a6 <__bad_interrupt>
      34:	0c 94 d0 09 	jmp	0x13a0	; 0x13a0 <__vector_13>
      38:	0c 94 53 01 	jmp	0x2a6	; 0x2a6 <__bad_interrupt>
      3c:	0c 94 53 01 	jmp	0x2a6	; 0x2a6 <__bad_interrupt>
      40:	0c 94 53 01 	jmp	0x2a6	; 0x2a6 <__bad_interrupt>
      44:	0c 94 53 01 	jmp	0x2a6	; 0x2a6 <__bad_interrupt>
      48:	0c 94 53 01 	jmp	0x2a6	; 0x2a6 <__bad_interrupt>
      4c:	0c 94 53 01 	jmp	0x2a6	; 0x2a6 <__bad_interrupt>
      50:	0c 94 53 01 	jmp	0x2a6	; 0x2a6 <__bad_interrupt>
      54:	0c 94 53 01 	jmp	0x2a6	; 0x2a6 <__bad_interrupt>
      58:	0c 94 53 01 	jmp	0x2a6	; 0x2a6 <__bad_interrupt>
      5c:	0c 94 53 01 	jmp	0x2a6	; 0x2a6 <__bad_interrupt>
      60:	0c 94 53 01 	jmp	0x2a6	; 0x2a6 <__bad_interrupt>
      64:	0c 94 35 12 	jmp	0x246a	; 0x246a <__vector_25>
      68:	0c 94 83 12 	jmp	0x2506	; 0x2506 <__vector_26>
      6c:	0c 94 53 01 	jmp	0x2a6	; 0x2a6 <__bad_interrupt>
      70:	0c 94 53 01 	jmp	0x2a6	; 0x2a6 <__bad_interrupt>
      74:	0c 94 53 01 	jmp	0x2a6	; 0x2a6 <__bad_interrupt>
      78:	0c 94 53 01 	jmp	0x2a6	; 0x2a6 <__bad_interrupt>
      7c:	0c 94 53 01 	jmp	0x2a6	; 0x2a6 <__bad_interrupt>
      80:	0c 94 53 01 	jmp	0x2a6	; 0x2a6 <__bad_interrupt>
      84:	0c 94 53 01 	jmp	0x2a6	; 0x2a6 <__bad_interrupt>
      88:	0c 94 53 01 	jmp	0x2a6	; 0x2a6 <__bad_interrupt>
      8c:	0c 94 53 01 	jmp	0x2a6	; 0x2a6 <__bad_interrupt>
      90:	0c 94 53 01 	jmp	0x2a6	; 0x2a6 <__bad_interrupt>
      94:	0c 94 53 01 	jmp	0x2a6	; 0x2a6 <__bad_interrupt>
      98:	0c 94 53 01 	jmp	0x2a6	; 0x2a6 <__bad_interrupt>
      9c:	0c 94 53 01 	jmp	0x2a6	; 0x2a6 <__bad_interrupt>
      a0:	0c 94 53 01 	jmp	0x2a6	; 0x2a6 <__bad_interrupt>
      a4:	0c 94 53 01 	jmp	0x2a6	; 0x2a6 <__bad_interrupt>
      a8:	0c 94 53 01 	jmp	0x2a6	; 0x2a6 <__bad_interrupt>
      ac:	0c 94 53 01 	jmp	0x2a6	; 0x2a6 <__bad_interrupt>
      b0:	0c 94 53 01 	jmp	0x2a6	; 0x2a6 <__bad_interrupt>
      b4:	0c 94 53 01 	jmp	0x2a6	; 0x2a6 <__bad_interrupt>
      b8:	0c 94 03 0a 	jmp	0x1406	; 0x1406 <__vector_46>
      bc:	0c 94 53 01 	jmp	0x2a6	; 0x2a6 <__bad_interrupt>
      c0:	0c 94 53 01 	jmp	0x2a6	; 0x2a6 <__bad_interrupt>
      c4:	0c 94 53 01 	jmp	0x2a6	; 0x2a6 <__bad_interrupt>
      c8:	0c 94 53 01 	jmp	0x2a6	; 0x2a6 <__bad_interrupt>
      cc:	0c 94 53 01 	jmp	0x2a6	; 0x2a6 <__bad_interrupt>
      d0:	0c 94 53 01 	jmp	0x2a6	; 0x2a6 <__bad_interrupt>
      d4:	0c 94 53 01 	jmp	0x2a6	; 0x2a6 <__bad_interrupt>
      d8:	0c 94 53 01 	jmp	0x2a6	; 0x2a6 <__bad_interrupt>
      dc:	0c 94 53 01 	jmp	0x2a6	; 0x2a6 <__bad_interrupt>
      e0:	0c 94 53 01 	jmp	0x2a6	; 0x2a6 <__bad_interrupt>
      e4:	0c 94 53 01 	jmp	0x2a6	; 0x2a6 <__bad_interrupt>
      e8:	0c 94 53 01 	jmp	0x2a6	; 0x2a6 <__bad_interrupt>
      ec:	0c 94 53 01 	jmp	0x2a6	; 0x2a6 <__bad_interrupt>
      f0:	0c 94 53 01 	jmp	0x2a6	; 0x2a6 <__bad_interrupt>
      f4:	0c 94 53 01 	jmp	0x2a6	; 0x2a6 <__bad_interrupt>
      f8:	0c 94 53 01 	jmp	0x2a6	; 0x2a6 <__bad_interrupt>
      fc:	0c 94 53 01 	jmp	0x2a6	; 0x2a6 <__bad_interrupt>
     100:	0c 94 53 01 	jmp	0x2a6	; 0x2a6 <__bad_interrupt>
     104:	0c 94 53 01 	jmp	0x2a6	; 0x2a6 <__bad_interrupt>
     108:	0c 94 53 01 	jmp	0x2a6	; 0x2a6 <__bad_interrupt>
     10c:	0c 94 53 01 	jmp	0x2a6	; 0x2a6 <__bad_interrupt>
     110:	0c 94 53 01 	jmp	0x2a6	; 0x2a6 <__bad_interrupt>
     114:	0c 94 53 01 	jmp	0x2a6	; 0x2a6 <__bad_interrupt>
     118:	0c 94 53 01 	jmp	0x2a6	; 0x2a6 <__bad_interrupt>
     11c:	0c 94 53 01 	jmp	0x2a6	; 0x2a6 <__bad_interrupt>
     120:	0c 94 53 01 	jmp	0x2a6	; 0x2a6 <__bad_interrupt>
     124:	0c 94 53 01 	jmp	0x2a6	; 0x2a6 <__bad_interrupt>
     128:	0c 94 53 01 	jmp	0x2a6	; 0x2a6 <__bad_interrupt>
     12c:	0c 94 53 01 	jmp	0x2a6	; 0x2a6 <__bad_interrupt>
     130:	0c 94 53 01 	jmp	0x2a6	; 0x2a6 <__bad_interrupt>
     134:	0c 94 53 01 	jmp	0x2a6	; 0x2a6 <__bad_interrupt>
     138:	0c 94 53 01 	jmp	0x2a6	; 0x2a6 <__bad_interrupt>
     13c:	0c 94 53 01 	jmp	0x2a6	; 0x2a6 <__bad_interrupt>
     140:	0c 94 53 01 	jmp	0x2a6	; 0x2a6 <__bad_interrupt>
     144:	0c 94 53 01 	jmp	0x2a6	; 0x2a6 <__bad_interrupt>
     148:	0c 94 53 01 	jmp	0x2a6	; 0x2a6 <__bad_interrupt>
     14c:	0c 94 53 01 	jmp	0x2a6	; 0x2a6 <__bad_interrupt>
     150:	0c 94 53 01 	jmp	0x2a6	; 0x2a6 <__bad_interrupt>
     154:	0c 94 53 01 	jmp	0x2a6	; 0x2a6 <__bad_interrupt>
     158:	0c 94 53 01 	jmp	0x2a6	; 0x2a6 <__bad_interrupt>
     15c:	0c 94 53 01 	jmp	0x2a6	; 0x2a6 <__bad_interrupt>
     160:	0c 94 53 01 	jmp	0x2a6	; 0x2a6 <__bad_interrupt>
     164:	0c 94 53 01 	jmp	0x2a6	; 0x2a6 <__bad_interrupt>
     168:	0c 94 53 01 	jmp	0x2a6	; 0x2a6 <__bad_interrupt>
     16c:	0c 94 53 01 	jmp	0x2a6	; 0x2a6 <__bad_interrupt>
     170:	0c 94 53 01 	jmp	0x2a6	; 0x2a6 <__bad_interrupt>
     174:	0c 94 53 01 	jmp	0x2a6	; 0x2a6 <__bad_interrupt>
     178:	0c 94 53 01 	jmp	0x2a6	; 0x2a6 <__bad_interrupt>
     17c:	0c 94 53 01 	jmp	0x2a6	; 0x2a6 <__bad_interrupt>
     180:	0c 94 53 01 	jmp	0x2a6	; 0x2a6 <__bad_interrupt>
     184:	0c 94 53 01 	jmp	0x2a6	; 0x2a6 <__bad_interrupt>
     188:	0c 94 53 01 	jmp	0x2a6	; 0x2a6 <__bad_interrupt>
     18c:	0c 94 53 01 	jmp	0x2a6	; 0x2a6 <__bad_interrupt>
     190:	0c 94 53 01 	jmp	0x2a6	; 0x2a6 <__bad_interrupt>
     194:	0c 94 53 01 	jmp	0x2a6	; 0x2a6 <__bad_interrupt>
     198:	0c 94 53 01 	jmp	0x2a6	; 0x2a6 <__bad_interrupt>
     19c:	0c 94 53 01 	jmp	0x2a6	; 0x2a6 <__bad_interrupt>
     1a0:	0c 94 53 01 	jmp	0x2a6	; 0x2a6 <__bad_interrupt>
     1a4:	0c 94 53 01 	jmp	0x2a6	; 0x2a6 <__bad_interrupt>
     1a8:	0c 94 53 01 	jmp	0x2a6	; 0x2a6 <__bad_interrupt>
     1ac:	0c 94 53 01 	jmp	0x2a6	; 0x2a6 <__bad_interrupt>
     1b0:	0c 94 53 01 	jmp	0x2a6	; 0x2a6 <__bad_interrupt>
     1b4:	0c 94 53 01 	jmp	0x2a6	; 0x2a6 <__bad_interrupt>
     1b8:	0c 94 53 01 	jmp	0x2a6	; 0x2a6 <__bad_interrupt>
     1bc:	0c 94 53 01 	jmp	0x2a6	; 0x2a6 <__bad_interrupt>
     1c0:	0c 94 53 01 	jmp	0x2a6	; 0x2a6 <__bad_interrupt>
     1c4:	0c 94 53 01 	jmp	0x2a6	; 0x2a6 <__bad_interrupt>
     1c8:	0c 94 53 01 	jmp	0x2a6	; 0x2a6 <__bad_interrupt>
     1cc:	0c 94 53 01 	jmp	0x2a6	; 0x2a6 <__bad_interrupt>
     1d0:	0c 94 53 01 	jmp	0x2a6	; 0x2a6 <__bad_interrupt>
     1d4:	0c 94 53 01 	jmp	0x2a6	; 0x2a6 <__bad_interrupt>
     1d8:	0c 94 53 01 	jmp	0x2a6	; 0x2a6 <__bad_interrupt>
     1dc:	0c 94 53 01 	jmp	0x2a6	; 0x2a6 <__bad_interrupt>
     1e0:	0c 94 53 01 	jmp	0x2a6	; 0x2a6 <__bad_interrupt>
     1e4:	0c 94 53 01 	jmp	0x2a6	; 0x2a6 <__bad_interrupt>
     1e8:	0c 94 53 01 	jmp	0x2a6	; 0x2a6 <__bad_interrupt>
     1ec:	0c 94 53 01 	jmp	0x2a6	; 0x2a6 <__bad_interrupt>
     1f0:	0c 94 53 01 	jmp	0x2a6	; 0x2a6 <__bad_interrupt>
     1f4:	0c 94 a7 0f 	jmp	0x1f4e	; 0x1f4e <__vector_125>
     1f8:	0c 94 74 10 	jmp	0x20e8	; 0x20e8 <__vector_126>
     1fc:	38 0b       	sbc	r19, r24
     1fe:	3b 0b       	sbc	r19, r27
     200:	3e 0b       	sbc	r19, r30
     202:	41 0b       	sbc	r20, r17
     204:	44 0b       	sbc	r20, r20
     206:	47 0b       	sbc	r20, r23
     208:	4a 0b       	sbc	r20, r26

0000020a <__trampolines_start>:
     20a:	0c 94 3e 0b 	jmp	0x167c	; 0x167c <udd_ep_get_size+0x2e>
     20e:	0c 94 a8 02 	jmp	0x550	; 0x550 <udi_cdc_data_sent>
     212:	0c 94 2f 03 	jmp	0x65e	; 0x65e <udi_cdc_data_disable>
     216:	0c 94 47 0b 	jmp	0x168e	; 0x168e <udd_ep_get_size+0x40>
     21a:	0c 94 46 04 	jmp	0x88c	; 0x88c <udi_cdc_data_received>
     21e:	0c 94 97 05 	jmp	0xb2e	; 0xb2e <udc_valid_address>
     222:	0c 94 be 01 	jmp	0x37c	; 0x37c <udi_cdc_line_coding_received>
     226:	0c 94 b4 01 	jmp	0x368	; 0x368 <udi_cdc_comm_disable>
     22a:	0c 94 3b 0b 	jmp	0x1676	; 0x1676 <udd_ep_get_size+0x28>
     22e:	0c 94 41 0b 	jmp	0x1682	; 0x1682 <udd_ep_get_size+0x34>
     232:	0c 94 c4 01 	jmp	0x388	; 0x388 <udi_cdc_comm_enable>
     236:	0c 94 38 0b 	jmp	0x1670	; 0x1670 <udd_ep_get_size+0x22>
     23a:	0c 94 4a 0b 	jmp	0x1694	; 0x1694 <udd_ep_get_size+0x46>
     23e:	0c 94 44 0b 	jmp	0x1688	; 0x1688 <udd_ep_get_size+0x3a>
     242:	0c 94 12 04 	jmp	0x824	; 0x824 <udi_cdc_data_enable>
     246:	0c 94 bc 01 	jmp	0x378	; 0x378 <udi_cdc_getsetting>
     24a:	0c 94 3b 03 	jmp	0x676	; 0x676 <udi_cdc_comm_setup>
     24e:	0c 94 c1 02 	jmp	0x582	; 0x582 <udi_cdc_data_sof_notify>
     252:	0c 94 18 03 	jmp	0x630	; 0x630 <udi_cdc_serial_state_msg_sent>
     256:	0c 94 ba 01 	jmp	0x374	; 0x374 <udi_cdc_data_setup>

0000025a <__ctors_end>:
     25a:	11 24       	eor	r1, r1
     25c:	1f be       	out	0x3f, r1	; 63
     25e:	cf ef       	ldi	r28, 0xFF	; 255
     260:	cd bf       	out	0x3d, r28	; 61
     262:	df e3       	ldi	r29, 0x3F	; 63
     264:	de bf       	out	0x3e, r29	; 62
     266:	00 e0       	ldi	r16, 0x00	; 0
     268:	0c bf       	out	0x3c, r16	; 60
     26a:	18 be       	out	0x38, r1	; 56
     26c:	19 be       	out	0x39, r1	; 57
     26e:	1a be       	out	0x3a, r1	; 58
     270:	1b be       	out	0x3b, r1	; 59

00000272 <__do_copy_data>:
     272:	10 e2       	ldi	r17, 0x20	; 32
     274:	a0 e0       	ldi	r26, 0x00	; 0
     276:	b0 e2       	ldi	r27, 0x20	; 32
     278:	ec e8       	ldi	r30, 0x8C	; 140
     27a:	f7 e2       	ldi	r31, 0x27	; 39
     27c:	00 e0       	ldi	r16, 0x00	; 0
     27e:	0b bf       	out	0x3b, r16	; 59
     280:	02 c0       	rjmp	.+4      	; 0x286 <__do_copy_data+0x14>
     282:	07 90       	elpm	r0, Z+
     284:	0d 92       	st	X+, r0
     286:	a6 3b       	cpi	r26, 0xB6	; 182
     288:	b1 07       	cpc	r27, r17
     28a:	d9 f7       	brne	.-10     	; 0x282 <__do_copy_data+0x10>
     28c:	1b be       	out	0x3b, r1	; 59

0000028e <__do_clear_bss>:
     28e:	23 e2       	ldi	r18, 0x23	; 35
     290:	a6 eb       	ldi	r26, 0xB6	; 182
     292:	b0 e2       	ldi	r27, 0x20	; 32
     294:	01 c0       	rjmp	.+2      	; 0x298 <.do_clear_bss_start>

00000296 <.do_clear_bss_loop>:
     296:	1d 92       	st	X+, r1

00000298 <.do_clear_bss_start>:
     298:	a0 34       	cpi	r26, 0x40	; 64
     29a:	b2 07       	cpc	r27, r18
     29c:	e1 f7       	brne	.-8      	; 0x296 <.do_clear_bss_loop>
     29e:	0e 94 55 01 	call	0x2aa	; 0x2aa <main>
     2a2:	0c 94 c4 13 	jmp	0x2788	; 0x2788 <_exit>

000002a6 <__bad_interrupt>:
     2a6:	0c 94 00 00 	jmp	0	; 0x0 <__vectors>

000002aa <main>:
static volatile bool main_b_cdc_enable = false;

int main(void)
{
	int error = 0;
	irq_initialize_vectors();
     2aa:	87 e0       	ldi	r24, 0x07	; 7
     2ac:	80 93 a2 00 	sts	0x00A2, r24	; 0x8000a2 <__TEXT_REGION_LENGTH__+0x7000a2>
	cpu_irq_enable();
     2b0:	78 94       	sei
{
#ifdef CONFIG_SLEEPMGR_ENABLE
	uint8_t i;

	for (i = 0; i < SLEEPMGR_NR_OF_MODES - 1; i++) {
		sleepmgr_locks[i] = 0;
     2b2:	ea e2       	ldi	r30, 0x2A	; 42
     2b4:	f3 e2       	ldi	r31, 0x23	; 35
     2b6:	10 82       	st	Z, r1
     2b8:	11 82       	std	Z+1, r1	; 0x01
     2ba:	12 82       	std	Z+2, r1	; 0x02
     2bc:	13 82       	std	Z+3, r1	; 0x03
     2be:	14 82       	std	Z+4, r1	; 0x04
	}
	sleepmgr_locks[SLEEPMGR_NR_OF_MODES - 1] = 1;
     2c0:	81 e0       	ldi	r24, 0x01	; 1
     2c2:	85 83       	std	Z+5, r24	; 0x05

	// Initialize the sleep manager
	sleepmgr_init();

	#if !SAM0
		sysclk_init();
     2c4:	0e 94 c4 12 	call	0x2588	; 0x2588 <sysclk_init>
		board_init();
     2c8:	0e 94 27 13 	call	0x264e	; 0x264e <board_init>
			write(str_cmd, CMD_LENGTH);
		}
	};
#endif // _cplusplus
	return error;
}
     2cc:	80 e0       	ldi	r24, 0x00	; 0
     2ce:	90 e0       	ldi	r25, 0x00	; 0
     2d0:	08 95       	ret

000002d2 <ui_powerdown>:
		bool level)
{
	PORT_t *base = arch_ioport_pin_to_base(pin);

	if (level) {
		base->OUTSET = arch_ioport_pin_to_mask(pin);
     2d2:	e0 e0       	ldi	r30, 0x00	; 0
     2d4:	f6 e0       	ldi	r31, 0x06	; 6
     2d6:	81 e0       	ldi	r24, 0x01	; 1
     2d8:	85 83       	std	Z+5, r24	; 0x05
     2da:	82 e0       	ldi	r24, 0x02	; 2
     2dc:	85 83       	std	Z+5, r24	; 0x05
     2de:	84 e0       	ldi	r24, 0x04	; 4
     2e0:	85 83       	std	Z+5, r24	; 0x05
     2e2:	80 e1       	ldi	r24, 0x10	; 16
     2e4:	85 83       	std	Z+5, r24	; 0x05
     2e6:	80 e2       	ldi	r24, 0x20	; 32
     2e8:	85 83       	std	Z+5, r24	; 0x05
     2ea:	80 e4       	ldi	r24, 0x40	; 64
     2ec:	85 83       	std	Z+5, r24	; 0x05
     2ee:	80 e8       	ldi	r24, 0x80	; 128
     2f0:	85 83       	std	Z+5, r24	; 0x05
     2f2:	08 95       	ret

000002f4 <ui_wakeup>:
	} else {
		base->OUTCLR = arch_ioport_pin_to_mask(pin);
     2f4:	81 e0       	ldi	r24, 0x01	; 1
     2f6:	80 93 06 06 	sts	0x0606, r24	; 0x800606 <__TEXT_REGION_LENGTH__+0x700606>
     2fa:	08 95       	ret

000002fc <ui_com_open>:
     2fc:	84 e0       	ldi	r24, 0x04	; 4
     2fe:	80 93 06 06 	sts	0x0606, r24	; 0x800606 <__TEXT_REGION_LENGTH__+0x700606>
     302:	08 95       	ret

00000304 <ui_com_close>:
		bool level)
{
	PORT_t *base = arch_ioport_pin_to_base(pin);

	if (level) {
		base->OUTSET = arch_ioport_pin_to_mask(pin);
     304:	e0 e0       	ldi	r30, 0x00	; 0
     306:	f6 e0       	ldi	r31, 0x06	; 6
     308:	84 e0       	ldi	r24, 0x04	; 4
     30a:	85 83       	std	Z+5, r24	; 0x05
     30c:	80 e1       	ldi	r24, 0x10	; 16
     30e:	85 83       	std	Z+5, r24	; 0x05
     310:	80 e2       	ldi	r24, 0x20	; 32
     312:	85 83       	std	Z+5, r24	; 0x05
     314:	80 e4       	ldi	r24, 0x40	; 64
     316:	85 83       	std	Z+5, r24	; 0x05
     318:	80 e8       	ldi	r24, 0x80	; 128
     31a:	85 83       	std	Z+5, r24	; 0x05
     31c:	08 95       	ret

0000031e <ui_com_rx_start>:
	} else {
		base->OUTCLR = arch_ioport_pin_to_mask(pin);
     31e:	80 e1       	ldi	r24, 0x10	; 16
     320:	80 93 06 06 	sts	0x0606, r24	; 0x800606 <__TEXT_REGION_LENGTH__+0x700606>
     324:	08 95       	ret

00000326 <ui_com_rx_stop>:
		bool level)
{
	PORT_t *base = arch_ioport_pin_to_base(pin);

	if (level) {
		base->OUTSET = arch_ioport_pin_to_mask(pin);
     326:	80 e1       	ldi	r24, 0x10	; 16
     328:	80 93 05 06 	sts	0x0605, r24	; 0x800605 <__TEXT_REGION_LENGTH__+0x700605>
     32c:	08 95       	ret

0000032e <ui_com_tx_start>:
	} else {
		base->OUTCLR = arch_ioport_pin_to_mask(pin);
     32e:	80 e2       	ldi	r24, 0x20	; 32
     330:	80 93 06 06 	sts	0x0606, r24	; 0x800606 <__TEXT_REGION_LENGTH__+0x700606>
     334:	08 95       	ret

00000336 <ui_com_tx_stop>:
		bool level)
{
	PORT_t *base = arch_ioport_pin_to_base(pin);

	if (level) {
		base->OUTSET = arch_ioport_pin_to_mask(pin);
     336:	80 e2       	ldi	r24, 0x20	; 32
     338:	80 93 05 06 	sts	0x0605, r24	; 0x800605 <__TEXT_REGION_LENGTH__+0x700605>
     33c:	08 95       	ret

0000033e <ui_com_error>:
	} else {
		base->OUTCLR = arch_ioport_pin_to_mask(pin);
     33e:	80 e4       	ldi	r24, 0x40	; 64
     340:	80 93 06 06 	sts	0x0606, r24	; 0x800606 <__TEXT_REGION_LENGTH__+0x700606>
     344:	08 95       	ret

00000346 <ui_com_overflow>:
     346:	80 e8       	ldi	r24, 0x80	; 128
     348:	80 93 06 06 	sts	0x0606, r24	; 0x800606 <__TEXT_REGION_LENGTH__+0x700606>
     34c:	08 95       	ret

0000034e <ui_process>:
	LED_On(LED7_GPIO);
}

void ui_process(uint16_t framenumber)
{
	if (0 == framenumber) {
     34e:	00 97       	sbiw	r24, 0x00	; 0
     350:	21 f4       	brne	.+8      	; 0x35a <ui_process+0xc>
     352:	82 e0       	ldi	r24, 0x02	; 2
     354:	80 93 06 06 	sts	0x0606, r24	; 0x800606 <__TEXT_REGION_LENGTH__+0x700606>
     358:	08 95       	ret
		LED_On(LED1_GPIO);
	}
	if (1000 == framenumber) {
     35a:	88 3e       	cpi	r24, 0xE8	; 232
     35c:	93 40       	sbci	r25, 0x03	; 3
     35e:	19 f4       	brne	.+6      	; 0x366 <ui_process+0x18>
		bool level)
{
	PORT_t *base = arch_ioport_pin_to_base(pin);

	if (level) {
		base->OUTSET = arch_ioport_pin_to_mask(pin);
     360:	82 e0       	ldi	r24, 0x02	; 2
     362:	80 93 05 06 	sts	0x0605, r24	; 0x800605 <__TEXT_REGION_LENGTH__+0x700605>
     366:	08 95       	ret

00000368 <udi_cdc_comm_disable>:
}

iram_size_t udi_cdc_get_free_tx_buffer(void)
{
	return udi_cdc_multi_get_free_tx_buffer(0);
}
     368:	80 91 cc 21 	lds	r24, 0x21CC	; 0x8021cc <udi_cdc_nb_comm_enabled>
     36c:	81 50       	subi	r24, 0x01	; 1
     36e:	80 93 cc 21 	sts	0x21CC, r24	; 0x8021cc <udi_cdc_nb_comm_enabled>
     372:	08 95       	ret

00000374 <udi_cdc_data_setup>:
     374:	80 e0       	ldi	r24, 0x00	; 0
     376:	08 95       	ret

00000378 <udi_cdc_getsetting>:
     378:	80 e0       	ldi	r24, 0x00	; 0
     37a:	08 95       	ret

0000037c <udi_cdc_line_coding_received>:
     37c:	6c ed       	ldi	r22, 0xDC	; 220
     37e:	71 e2       	ldi	r23, 0x21	; 33
     380:	80 e0       	ldi	r24, 0x00	; 0
     382:	0e 94 a7 11 	call	0x234e	; 0x234e <uart_config>
     386:	08 95       	ret

00000388 <udi_cdc_comm_enable>:
     388:	10 92 cc 21 	sts	0x21CC, r1	; 0x8021cc <udi_cdc_nb_comm_enabled>
     38c:	10 92 d8 21 	sts	0x21D8, r1	; 0x8021d8 <udi_cdc_state>
     390:	10 92 d9 21 	sts	0x21D9, r1	; 0x8021d9 <udi_cdc_state+0x1>
     394:	ee ec       	ldi	r30, 0xCE	; 206
     396:	f1 e2       	ldi	r31, 0x21	; 33
     398:	81 ea       	ldi	r24, 0xA1	; 161
     39a:	80 83       	st	Z, r24
     39c:	80 e2       	ldi	r24, 0x20	; 32
     39e:	81 83       	std	Z+1, r24	; 0x01
     3a0:	12 82       	std	Z+2, r1	; 0x02
     3a2:	13 82       	std	Z+3, r1	; 0x03
     3a4:	14 82       	std	Z+4, r1	; 0x04
     3a6:	15 82       	std	Z+5, r1	; 0x05
     3a8:	82 e0       	ldi	r24, 0x02	; 2
     3aa:	90 e0       	ldi	r25, 0x00	; 0
     3ac:	86 83       	std	Z+6, r24	; 0x06
     3ae:	97 83       	std	Z+7, r25	; 0x07
     3b0:	10 86       	std	Z+8, r1	; 0x08
     3b2:	11 86       	std	Z+9, r1	; 0x09
     3b4:	ec ed       	ldi	r30, 0xDC	; 220
     3b6:	f1 e2       	ldi	r31, 0x21	; 33
     3b8:	80 e0       	ldi	r24, 0x00	; 0
     3ba:	92 ec       	ldi	r25, 0xC2	; 194
     3bc:	a1 e0       	ldi	r26, 0x01	; 1
     3be:	b0 e0       	ldi	r27, 0x00	; 0
     3c0:	80 83       	st	Z, r24
     3c2:	91 83       	std	Z+1, r25	; 0x01
     3c4:	a2 83       	std	Z+2, r26	; 0x02
     3c6:	b3 83       	std	Z+3, r27	; 0x03
     3c8:	14 82       	std	Z+4, r1	; 0x04
     3ca:	15 82       	std	Z+5, r1	; 0x05
     3cc:	88 e0       	ldi	r24, 0x08	; 8
     3ce:	86 83       	std	Z+6, r24	; 0x06
     3d0:	bf 01       	movw	r22, r30
     3d2:	80 e0       	ldi	r24, 0x00	; 0
     3d4:	0e 94 a7 11 	call	0x234e	; 0x234e <uart_config>
     3d8:	80 e0       	ldi	r24, 0x00	; 0
     3da:	0e 94 93 11 	call	0x2326	; 0x2326 <main_cdc_enable>
     3de:	88 23       	and	r24, r24
     3e0:	29 f0       	breq	.+10     	; 0x3ec <udi_cdc_comm_enable+0x64>
     3e2:	90 91 cc 21 	lds	r25, 0x21CC	; 0x8021cc <udi_cdc_nb_comm_enabled>
     3e6:	9f 5f       	subi	r25, 0xFF	; 255
     3e8:	90 93 cc 21 	sts	0x21CC, r25	; 0x8021cc <udi_cdc_nb_comm_enabled>
     3ec:	08 95       	ret

000003ee <udi_cdc_tx_send>:
     3ee:	ff 92       	push	r15
     3f0:	0f 93       	push	r16
     3f2:	1f 93       	push	r17
     3f4:	cf 93       	push	r28
     3f6:	df 93       	push	r29
     3f8:	1f 92       	push	r1
     3fa:	cd b7       	in	r28, 0x3d	; 61
     3fc:	de b7       	in	r29, 0x3e	; 62
     3fe:	80 91 b9 20 	lds	r24, 0x20B9	; 0x8020b9 <udi_cdc_tx_trans_ongoing>
     402:	81 11       	cpse	r24, r1
     404:	9e c0       	rjmp	.+316    	; 0x542 <__FUSE_REGION_LENGTH__+0x142>
     406:	0e 94 65 0d 	call	0x1aca	; 0x1aca <udd_is_high_speed>
     40a:	88 23       	and	r24, r24
     40c:	51 f0       	breq	.+20     	; 0x422 <__FUSE_REGION_LENGTH__+0x22>
     40e:	00 91 ba 20 	lds	r16, 0x20BA	; 0x8020ba <udi_cdc_tx_sof_num>
     412:	10 91 bb 20 	lds	r17, 0x20BB	; 0x8020bb <udi_cdc_tx_sof_num+0x1>
     416:	0e 94 72 0d 	call	0x1ae4	; 0x1ae4 <udd_get_micro_frame_number>
     41a:	08 17       	cp	r16, r24
     41c:	19 07       	cpc	r17, r25
     41e:	59 f4       	brne	.+22     	; 0x436 <__FUSE_REGION_LENGTH__+0x36>
     420:	90 c0       	rjmp	.+288    	; 0x542 <__FUSE_REGION_LENGTH__+0x142>
     422:	00 91 ba 20 	lds	r16, 0x20BA	; 0x8020ba <udi_cdc_tx_sof_num>
     426:	10 91 bb 20 	lds	r17, 0x20BB	; 0x8020bb <udi_cdc_tx_sof_num+0x1>
     42a:	0e 94 6d 0d 	call	0x1ada	; 0x1ada <udd_get_frame_number>
     42e:	08 17       	cp	r16, r24
     430:	19 07       	cpc	r17, r25
     432:	09 f4       	brne	.+2      	; 0x436 <__FUSE_REGION_LENGTH__+0x36>
     434:	86 c0       	rjmp	.+268    	; 0x542 <__FUSE_REGION_LENGTH__+0x142>
     436:	8f b7       	in	r24, 0x3f	; 63
     438:	89 83       	std	Y+1, r24	; 0x01
     43a:	f8 94       	cli
     43c:	19 81       	ldd	r17, Y+1	; 0x01
     43e:	00 91 bc 20 	lds	r16, 0x20BC	; 0x8020bc <udi_cdc_tx_buf_sel>
     442:	e0 2f       	mov	r30, r16
     444:	f0 e0       	ldi	r31, 0x00	; 0
     446:	ee 0f       	add	r30, r30
     448:	ff 1f       	adc	r31, r31
     44a:	e3 54       	subi	r30, 0x43	; 67
     44c:	ff 4d       	sbci	r31, 0xDF	; 223
     44e:	80 81       	ld	r24, Z
     450:	91 81       	ldd	r25, Z+1	; 0x01
     452:	89 2b       	or	r24, r25
     454:	09 f5       	brne	.+66     	; 0x498 <__FUSE_REGION_LENGTH__+0x98>
     456:	80 91 b6 20 	lds	r24, 0x20B6	; 0x8020b6 <__data_end>
     45a:	90 91 b7 20 	lds	r25, 0x20B7	; 0x8020b7 <__data_end+0x1>
     45e:	01 96       	adiw	r24, 0x01	; 1
     460:	80 93 b6 20 	sts	0x20B6, r24	; 0x8020b6 <__data_end>
     464:	90 93 b7 20 	sts	0x20B7, r25	; 0x8020b7 <__data_end+0x1>
     468:	0e 94 65 0d 	call	0x1aca	; 0x1aca <udd_is_high_speed>
     46c:	81 11       	cpse	r24, r1
     46e:	07 c0       	rjmp	.+14     	; 0x47e <__FUSE_REGION_LENGTH__+0x7e>
     470:	80 91 b6 20 	lds	r24, 0x20B6	; 0x8020b6 <__data_end>
     474:	90 91 b7 20 	lds	r25, 0x20B7	; 0x8020b7 <__data_end+0x1>
     478:	84 36       	cpi	r24, 0x64	; 100
     47a:	91 05       	cpc	r25, r1
     47c:	58 f0       	brcs	.+22     	; 0x494 <__FUSE_REGION_LENGTH__+0x94>
     47e:	0e 94 65 0d 	call	0x1aca	; 0x1aca <udd_is_high_speed>
     482:	88 23       	and	r24, r24
     484:	49 f0       	breq	.+18     	; 0x498 <__FUSE_REGION_LENGTH__+0x98>
     486:	80 91 b6 20 	lds	r24, 0x20B6	; 0x8020b6 <__data_end>
     48a:	90 91 b7 20 	lds	r25, 0x20B7	; 0x8020b7 <__data_end+0x1>
     48e:	80 32       	cpi	r24, 0x20	; 32
     490:	93 40       	sbci	r25, 0x03	; 3
     492:	10 f4       	brcc	.+4      	; 0x498 <__FUSE_REGION_LENGTH__+0x98>
     494:	1f bf       	out	0x3f, r17	; 63
     496:	55 c0       	rjmp	.+170    	; 0x542 <__FUSE_REGION_LENGTH__+0x142>
     498:	10 92 b6 20 	sts	0x20B6, r1	; 0x8020b6 <__data_end>
     49c:	10 92 b7 20 	sts	0x20B7, r1	; 0x8020b7 <__data_end+0x1>
     4a0:	80 91 b8 20 	lds	r24, 0x20B8	; 0x8020b8 <udi_cdc_tx_both_buf_to_send>
     4a4:	81 11       	cpse	r24, r1
     4a6:	06 c0       	rjmp	.+12     	; 0x4b4 <__FUSE_REGION_LENGTH__+0xb4>
     4a8:	81 e0       	ldi	r24, 0x01	; 1
     4aa:	01 11       	cpse	r16, r1
     4ac:	80 e0       	ldi	r24, 0x00	; 0
     4ae:	80 93 bc 20 	sts	0x20BC, r24	; 0x8020bc <udi_cdc_tx_buf_sel>
     4b2:	04 c0       	rjmp	.+8      	; 0x4bc <__FUSE_REGION_LENGTH__+0xbc>
     4b4:	81 e0       	ldi	r24, 0x01	; 1
     4b6:	01 11       	cpse	r16, r1
     4b8:	80 e0       	ldi	r24, 0x00	; 0
     4ba:	08 2f       	mov	r16, r24
     4bc:	81 e0       	ldi	r24, 0x01	; 1
     4be:	80 93 b9 20 	sts	0x20B9, r24	; 0x8020b9 <udi_cdc_tx_trans_ongoing>
     4c2:	1f bf       	out	0x3f, r17	; 63
     4c4:	10 e0       	ldi	r17, 0x00	; 0
     4c6:	f8 01       	movw	r30, r16
     4c8:	ee 0f       	add	r30, r30
     4ca:	ff 1f       	adc	r31, r31
     4cc:	e3 54       	subi	r30, 0x43	; 67
     4ce:	ff 4d       	sbci	r31, 0xDF	; 223
     4d0:	ff 24       	eor	r15, r15
     4d2:	f3 94       	inc	r15
     4d4:	80 81       	ld	r24, Z
     4d6:	91 81       	ldd	r25, Z+1	; 0x01
     4d8:	80 34       	cpi	r24, 0x40	; 64
     4da:	91 05       	cpc	r25, r1
     4dc:	09 f4       	brne	.+2      	; 0x4e0 <__FUSE_REGION_LENGTH__+0xe0>
     4de:	f1 2c       	mov	r15, r1
     4e0:	ff 20       	and	r15, r15
     4e2:	91 f0       	breq	.+36     	; 0x508 <__FUSE_REGION_LENGTH__+0x108>
     4e4:	0e 94 65 0d 	call	0x1aca	; 0x1aca <udd_is_high_speed>
     4e8:	88 23       	and	r24, r24
     4ea:	39 f0       	breq	.+14     	; 0x4fa <__FUSE_REGION_LENGTH__+0xfa>
     4ec:	0e 94 72 0d 	call	0x1ae4	; 0x1ae4 <udd_get_micro_frame_number>
     4f0:	80 93 ba 20 	sts	0x20BA, r24	; 0x8020ba <udi_cdc_tx_sof_num>
     4f4:	90 93 bb 20 	sts	0x20BB, r25	; 0x8020bb <udi_cdc_tx_sof_num+0x1>
     4f8:	0b c0       	rjmp	.+22     	; 0x510 <__FUSE_REGION_LENGTH__+0x110>
     4fa:	0e 94 6d 0d 	call	0x1ada	; 0x1ada <udd_get_frame_number>
     4fe:	80 93 ba 20 	sts	0x20BA, r24	; 0x8020ba <udi_cdc_tx_sof_num>
     502:	90 93 bb 20 	sts	0x20BB, r25	; 0x8020bb <udi_cdc_tx_sof_num+0x1>
     506:	04 c0       	rjmp	.+8      	; 0x510 <__FUSE_REGION_LENGTH__+0x110>
     508:	10 92 ba 20 	sts	0x20BA, r1	; 0x8020ba <udi_cdc_tx_sof_num>
     50c:	10 92 bb 20 	sts	0x20BB, r1	; 0x8020bb <udi_cdc_tx_sof_num+0x1>
     510:	f8 01       	movw	r30, r16
     512:	ee 0f       	add	r30, r30
     514:	ff 1f       	adc	r31, r31
     516:	e3 54       	subi	r30, 0x43	; 67
     518:	ff 4d       	sbci	r31, 0xDF	; 223
     51a:	20 81       	ld	r18, Z
     51c:	31 81       	ldd	r19, Z+1	; 0x01
     51e:	a8 01       	movw	r20, r16
     520:	00 24       	eor	r0, r0
     522:	56 95       	lsr	r21
     524:	47 95       	ror	r20
     526:	07 94       	ror	r0
     528:	56 95       	lsr	r21
     52a:	47 95       	ror	r20
     52c:	07 94       	ror	r0
     52e:	54 2f       	mov	r21, r20
     530:	40 2d       	mov	r20, r0
     532:	4e 53       	subi	r20, 0x3E	; 62
     534:	5f 4d       	sbci	r21, 0xDF	; 223
     536:	08 ea       	ldi	r16, 0xA8	; 168
     538:	12 e0       	ldi	r17, 0x02	; 2
     53a:	6f 2d       	mov	r22, r15
     53c:	81 e8       	ldi	r24, 0x81	; 129
     53e:	0e 94 57 0e 	call	0x1cae	; 0x1cae <udd_ep_run>
     542:	0f 90       	pop	r0
     544:	df 91       	pop	r29
     546:	cf 91       	pop	r28
     548:	1f 91       	pop	r17
     54a:	0f 91       	pop	r16
     54c:	ff 90       	pop	r15
     54e:	08 95       	ret

00000550 <udi_cdc_data_sent>:
     550:	81 11       	cpse	r24, r1
     552:	16 c0       	rjmp	.+44     	; 0x580 <udi_cdc_data_sent+0x30>
     554:	20 91 bc 20 	lds	r18, 0x20BC	; 0x8020bc <udi_cdc_tx_buf_sel>
     558:	81 e0       	ldi	r24, 0x01	; 1
     55a:	90 e0       	ldi	r25, 0x00	; 0
     55c:	22 23       	and	r18, r18
     55e:	11 f0       	breq	.+4      	; 0x564 <udi_cdc_data_sent+0x14>
     560:	80 e0       	ldi	r24, 0x00	; 0
     562:	90 e0       	ldi	r25, 0x00	; 0
     564:	88 0f       	add	r24, r24
     566:	99 1f       	adc	r25, r25
     568:	fc 01       	movw	r30, r24
     56a:	e3 54       	subi	r30, 0x43	; 67
     56c:	ff 4d       	sbci	r31, 0xDF	; 223
     56e:	10 82       	st	Z, r1
     570:	11 82       	std	Z+1, r1	; 0x01
     572:	10 92 b8 20 	sts	0x20B8, r1	; 0x8020b8 <udi_cdc_tx_both_buf_to_send>
     576:	10 92 b9 20 	sts	0x20B9, r1	; 0x8020b9 <udi_cdc_tx_trans_ongoing>
     57a:	80 e0       	ldi	r24, 0x00	; 0
     57c:	0e 94 f7 01 	call	0x3ee	; 0x3ee <udi_cdc_tx_send>
     580:	08 95       	ret

00000582 <udi_cdc_data_sof_notify>:
     582:	80 e0       	ldi	r24, 0x00	; 0
     584:	0e 94 f7 01 	call	0x3ee	; 0x3ee <udi_cdc_tx_send>
     588:	08 95       	ret

0000058a <udi_cdc_ctrl_state_notify>:
     58a:	0f 93       	push	r16
     58c:	1f 93       	push	r17
     58e:	80 91 da 21 	lds	r24, 0x21DA	; 0x8021da <udi_cdc_serial_state_msg_ongoing>
     592:	81 11       	cpse	r24, r1
     594:	1f c0       	rjmp	.+62     	; 0x5d4 <udi_cdc_ctrl_state_notify+0x4a>
     596:	20 91 d8 21 	lds	r18, 0x21D8	; 0x8021d8 <udi_cdc_state>
     59a:	30 91 d9 21 	lds	r19, 0x21D9	; 0x8021d9 <udi_cdc_state+0x1>
     59e:	80 91 d6 21 	lds	r24, 0x21D6	; 0x8021d6 <uid_cdc_state_msg+0x8>
     5a2:	90 91 d7 21 	lds	r25, 0x21D7	; 0x8021d7 <uid_cdc_state_msg+0x9>
     5a6:	28 17       	cp	r18, r24
     5a8:	39 07       	cpc	r19, r25
     5aa:	a1 f0       	breq	.+40     	; 0x5d4 <udi_cdc_ctrl_state_notify+0x4a>
     5ac:	86 2f       	mov	r24, r22
     5ae:	20 91 d8 21 	lds	r18, 0x21D8	; 0x8021d8 <udi_cdc_state>
     5b2:	30 91 d9 21 	lds	r19, 0x21D9	; 0x8021d9 <udi_cdc_state+0x1>
     5b6:	20 93 d6 21 	sts	0x21D6, r18	; 0x8021d6 <uid_cdc_state_msg+0x8>
     5ba:	30 93 d7 21 	sts	0x21D7, r19	; 0x8021d7 <uid_cdc_state_msg+0x9>
     5be:	08 e1       	ldi	r16, 0x18	; 24
     5c0:	13 e0       	ldi	r17, 0x03	; 3
     5c2:	2a e0       	ldi	r18, 0x0A	; 10
     5c4:	30 e0       	ldi	r19, 0x00	; 0
     5c6:	4e ec       	ldi	r20, 0xCE	; 206
     5c8:	51 e2       	ldi	r21, 0x21	; 33
     5ca:	60 e0       	ldi	r22, 0x00	; 0
     5cc:	0e 94 57 0e 	call	0x1cae	; 0x1cae <udd_ep_run>
     5d0:	80 93 da 21 	sts	0x21DA, r24	; 0x8021da <udi_cdc_serial_state_msg_ongoing>
     5d4:	1f 91       	pop	r17
     5d6:	0f 91       	pop	r16
     5d8:	08 95       	ret

000005da <udi_cdc_ctrl_state_change>:
     5da:	cf 93       	push	r28
     5dc:	df 93       	push	r29
     5de:	1f 92       	push	r1
     5e0:	cd b7       	in	r28, 0x3d	; 61
     5e2:	de b7       	in	r29, 0x3e	; 62
     5e4:	8f b7       	in	r24, 0x3f	; 63
     5e6:	89 83       	std	Y+1, r24	; 0x01
     5e8:	f8 94       	cli
     5ea:	29 81       	ldd	r18, Y+1	; 0x01
     5ec:	66 23       	and	r22, r22
     5ee:	59 f0       	breq	.+22     	; 0x606 <udi_cdc_ctrl_state_change+0x2c>
     5f0:	80 91 d8 21 	lds	r24, 0x21D8	; 0x8021d8 <udi_cdc_state>
     5f4:	90 91 d9 21 	lds	r25, 0x21D9	; 0x8021d9 <udi_cdc_state+0x1>
     5f8:	48 2b       	or	r20, r24
     5fa:	59 2b       	or	r21, r25
     5fc:	40 93 d8 21 	sts	0x21D8, r20	; 0x8021d8 <udi_cdc_state>
     600:	50 93 d9 21 	sts	0x21D9, r21	; 0x8021d9 <udi_cdc_state+0x1>
     604:	0c c0       	rjmp	.+24     	; 0x61e <udi_cdc_ctrl_state_change+0x44>
     606:	80 91 d8 21 	lds	r24, 0x21D8	; 0x8021d8 <udi_cdc_state>
     60a:	90 91 d9 21 	lds	r25, 0x21D9	; 0x8021d9 <udi_cdc_state+0x1>
     60e:	40 95       	com	r20
     610:	50 95       	com	r21
     612:	48 23       	and	r20, r24
     614:	59 23       	and	r21, r25
     616:	40 93 d8 21 	sts	0x21D8, r20	; 0x8021d8 <udi_cdc_state>
     61a:	50 93 d9 21 	sts	0x21D9, r21	; 0x8021d9 <udi_cdc_state+0x1>
     61e:	2f bf       	out	0x3f, r18	; 63
     620:	62 e8       	ldi	r22, 0x82	; 130
     622:	80 e0       	ldi	r24, 0x00	; 0
     624:	0e 94 c5 02 	call	0x58a	; 0x58a <udi_cdc_ctrl_state_notify>
     628:	0f 90       	pop	r0
     62a:	df 91       	pop	r29
     62c:	cf 91       	pop	r28
     62e:	08 95       	ret

00000630 <udi_cdc_serial_state_msg_sent>:
     630:	10 92 da 21 	sts	0x21DA, r1	; 0x8021da <udi_cdc_serial_state_msg_ongoing>
     634:	80 91 d8 21 	lds	r24, 0x21D8	; 0x8021d8 <udi_cdc_state>
     638:	90 91 d9 21 	lds	r25, 0x21D9	; 0x8021d9 <udi_cdc_state+0x1>
     63c:	83 78       	andi	r24, 0x83	; 131
     63e:	80 93 d8 21 	sts	0x21D8, r24	; 0x8021d8 <udi_cdc_state>
     642:	90 93 d9 21 	sts	0x21D9, r25	; 0x8021d9 <udi_cdc_state+0x1>
     646:	ee ec       	ldi	r30, 0xCE	; 206
     648:	f1 e2       	ldi	r31, 0x21	; 33
     64a:	80 85       	ldd	r24, Z+8	; 0x08
     64c:	91 85       	ldd	r25, Z+9	; 0x09
     64e:	83 78       	andi	r24, 0x83	; 131
     650:	80 87       	std	Z+8, r24	; 0x08
     652:	91 87       	std	Z+9, r25	; 0x09
     654:	64 2f       	mov	r22, r20
     656:	80 e0       	ldi	r24, 0x00	; 0
     658:	0e 94 c5 02 	call	0x58a	; 0x58a <udi_cdc_ctrl_state_notify>
     65c:	08 95       	ret

0000065e <udi_cdc_data_disable>:
     65e:	80 91 cb 21 	lds	r24, 0x21CB	; 0x8021cb <udi_cdc_nb_data_enabled>
     662:	81 50       	subi	r24, 0x01	; 1
     664:	80 93 cb 21 	sts	0x21CB, r24	; 0x8021cb <udi_cdc_nb_data_enabled>
     668:	80 91 cb 21 	lds	r24, 0x21CB	; 0x8021cb <udi_cdc_nb_data_enabled>
     66c:	0e 94 9a 11 	call	0x2334	; 0x2334 <main_cdc_disable>
     670:	10 92 ca 21 	sts	0x21CA, r1	; 0x8021ca <udi_cdc_data_running>
     674:	08 95       	ret

00000676 <udi_cdc_comm_setup>:
     676:	80 91 30 23 	lds	r24, 0x2330	; 0x802330 <udd_g_ctrlreq>
     67a:	88 23       	and	r24, r24
     67c:	cc f4       	brge	.+50     	; 0x6b0 <udi_cdc_comm_setup+0x3a>
     67e:	80 76       	andi	r24, 0x60	; 96
     680:	80 32       	cpi	r24, 0x20	; 32
     682:	f1 f5       	brne	.+124    	; 0x700 <udi_cdc_comm_setup+0x8a>
     684:	80 91 31 23 	lds	r24, 0x2331	; 0x802331 <udd_g_ctrlreq+0x1>
     688:	81 32       	cpi	r24, 0x21	; 33
     68a:	e1 f5       	brne	.+120    	; 0x704 <udi_cdc_comm_setup+0x8e>
     68c:	80 91 36 23 	lds	r24, 0x2336	; 0x802336 <udd_g_ctrlreq+0x6>
     690:	90 91 37 23 	lds	r25, 0x2337	; 0x802337 <udd_g_ctrlreq+0x7>
     694:	07 97       	sbiw	r24, 0x07	; 7
     696:	c1 f5       	brne	.+112    	; 0x708 <udi_cdc_comm_setup+0x92>
     698:	e0 e3       	ldi	r30, 0x30	; 48
     69a:	f3 e2       	ldi	r31, 0x23	; 35
     69c:	8c ed       	ldi	r24, 0xDC	; 220
     69e:	91 e2       	ldi	r25, 0x21	; 33
     6a0:	80 87       	std	Z+8, r24	; 0x08
     6a2:	91 87       	std	Z+9, r25	; 0x09
     6a4:	87 e0       	ldi	r24, 0x07	; 7
     6a6:	90 e0       	ldi	r25, 0x00	; 0
     6a8:	82 87       	std	Z+10, r24	; 0x0a
     6aa:	93 87       	std	Z+11, r25	; 0x0b
     6ac:	81 e0       	ldi	r24, 0x01	; 1
     6ae:	08 95       	ret
     6b0:	80 76       	andi	r24, 0x60	; 96
     6b2:	80 32       	cpi	r24, 0x20	; 32
     6b4:	59 f5       	brne	.+86     	; 0x70c <udi_cdc_comm_setup+0x96>
     6b6:	80 91 31 23 	lds	r24, 0x2331	; 0x802331 <udd_g_ctrlreq+0x1>
     6ba:	80 32       	cpi	r24, 0x20	; 32
     6bc:	19 f0       	breq	.+6      	; 0x6c4 <udi_cdc_comm_setup+0x4e>
     6be:	82 32       	cpi	r24, 0x22	; 34
     6c0:	b9 f0       	breq	.+46     	; 0x6f0 <udi_cdc_comm_setup+0x7a>
     6c2:	26 c0       	rjmp	.+76     	; 0x710 <udi_cdc_comm_setup+0x9a>
     6c4:	80 91 36 23 	lds	r24, 0x2336	; 0x802336 <udd_g_ctrlreq+0x6>
     6c8:	90 91 37 23 	lds	r25, 0x2337	; 0x802337 <udd_g_ctrlreq+0x7>
     6cc:	07 97       	sbiw	r24, 0x07	; 7
     6ce:	11 f5       	brne	.+68     	; 0x714 <udi_cdc_comm_setup+0x9e>
     6d0:	e0 e3       	ldi	r30, 0x30	; 48
     6d2:	f3 e2       	ldi	r31, 0x23	; 35
     6d4:	8e eb       	ldi	r24, 0xBE	; 190
     6d6:	91 e0       	ldi	r25, 0x01	; 1
     6d8:	84 87       	std	Z+12, r24	; 0x0c
     6da:	95 87       	std	Z+13, r25	; 0x0d
     6dc:	8c ed       	ldi	r24, 0xDC	; 220
     6de:	91 e2       	ldi	r25, 0x21	; 33
     6e0:	80 87       	std	Z+8, r24	; 0x08
     6e2:	91 87       	std	Z+9, r25	; 0x09
     6e4:	87 e0       	ldi	r24, 0x07	; 7
     6e6:	90 e0       	ldi	r25, 0x00	; 0
     6e8:	82 87       	std	Z+10, r24	; 0x0a
     6ea:	93 87       	std	Z+11, r25	; 0x0b
     6ec:	81 e0       	ldi	r24, 0x01	; 1
     6ee:	08 95       	ret
     6f0:	60 91 32 23 	lds	r22, 0x2332	; 0x802332 <udd_g_ctrlreq+0x2>
     6f4:	61 70       	andi	r22, 0x01	; 1
     6f6:	80 e0       	ldi	r24, 0x00	; 0
     6f8:	0e 94 9f 11 	call	0x233e	; 0x233e <main_cdc_set_dtr>
     6fc:	81 e0       	ldi	r24, 0x01	; 1
     6fe:	08 95       	ret
     700:	80 e0       	ldi	r24, 0x00	; 0
     702:	08 95       	ret
     704:	80 e0       	ldi	r24, 0x00	; 0
     706:	08 95       	ret
     708:	80 e0       	ldi	r24, 0x00	; 0
     70a:	08 95       	ret
     70c:	80 e0       	ldi	r24, 0x00	; 0
     70e:	08 95       	ret
     710:	80 e0       	ldi	r24, 0x00	; 0
     712:	08 95       	ret
     714:	80 e0       	ldi	r24, 0x00	; 0
     716:	08 95       	ret

00000718 <udi_cdc_signal_framing_error>:
     718:	40 e1       	ldi	r20, 0x10	; 16
     71a:	50 e0       	ldi	r21, 0x00	; 0
     71c:	61 e0       	ldi	r22, 0x01	; 1
     71e:	80 e0       	ldi	r24, 0x00	; 0
     720:	0e 94 ed 02 	call	0x5da	; 0x5da <udi_cdc_ctrl_state_change>
     724:	08 95       	ret

00000726 <udi_cdc_signal_overrun>:
     726:	40 e4       	ldi	r20, 0x40	; 64
     728:	50 e0       	ldi	r21, 0x00	; 0
     72a:	61 e0       	ldi	r22, 0x01	; 1
     72c:	80 e0       	ldi	r24, 0x00	; 0
     72e:	0e 94 ed 02 	call	0x5da	; 0x5da <udi_cdc_ctrl_state_change>
     732:	08 95       	ret

00000734 <udi_cdc_multi_get_nb_received_data>:
     734:	cf 93       	push	r28
     736:	df 93       	push	r29
     738:	1f 92       	push	r1
     73a:	cd b7       	in	r28, 0x3d	; 61
     73c:	de b7       	in	r29, 0x3e	; 62
     73e:	8f b7       	in	r24, 0x3f	; 63
     740:	89 83       	std	Y+1, r24	; 0x01
     742:	f8 94       	cli
     744:	49 81       	ldd	r20, Y+1	; 0x01
     746:	20 91 43 21 	lds	r18, 0x2143	; 0x802143 <udi_cdc_rx_pos>
     74a:	30 91 44 21 	lds	r19, 0x2144	; 0x802144 <udi_cdc_rx_pos+0x1>
     74e:	e0 91 45 21 	lds	r30, 0x2145	; 0x802145 <udi_cdc_rx_buf_sel>
     752:	f0 e0       	ldi	r31, 0x00	; 0
     754:	ee 0f       	add	r30, r30
     756:	ff 1f       	adc	r31, r31
     758:	ea 5b       	subi	r30, 0xBA	; 186
     75a:	fe 4d       	sbci	r31, 0xDE	; 222
     75c:	80 81       	ld	r24, Z
     75e:	91 81       	ldd	r25, Z+1	; 0x01
     760:	4f bf       	out	0x3f, r20	; 63
     762:	82 1b       	sub	r24, r18
     764:	93 0b       	sbc	r25, r19
     766:	0f 90       	pop	r0
     768:	df 91       	pop	r29
     76a:	cf 91       	pop	r28
     76c:	08 95       	ret

0000076e <udi_cdc_multi_is_rx_ready>:
     76e:	0e 94 9a 03 	call	0x734	; 0x734 <udi_cdc_multi_get_nb_received_data>
     772:	21 e0       	ldi	r18, 0x01	; 1
     774:	89 2b       	or	r24, r25
     776:	09 f4       	brne	.+2      	; 0x77a <udi_cdc_multi_is_rx_ready+0xc>
     778:	20 e0       	ldi	r18, 0x00	; 0
     77a:	82 2f       	mov	r24, r18
     77c:	08 95       	ret

0000077e <udi_cdc_rx_start>:
     77e:	0f 93       	push	r16
     780:	1f 93       	push	r17
     782:	cf 93       	push	r28
     784:	df 93       	push	r29
     786:	1f 92       	push	r1
     788:	cd b7       	in	r28, 0x3d	; 61
     78a:	de b7       	in	r29, 0x3e	; 62
     78c:	8f b7       	in	r24, 0x3f	; 63
     78e:	89 83       	std	Y+1, r24	; 0x01
     790:	f8 94       	cli
     792:	99 81       	ldd	r25, Y+1	; 0x01
     794:	20 91 45 21 	lds	r18, 0x2145	; 0x802145 <udi_cdc_rx_buf_sel>
     798:	80 91 42 21 	lds	r24, 0x2142	; 0x802142 <udi_cdc_rx_trans_ongoing>
     79c:	81 11       	cpse	r24, r1
     79e:	10 c0       	rjmp	.+32     	; 0x7c0 <udi_cdc_rx_start+0x42>
     7a0:	60 91 43 21 	lds	r22, 0x2143	; 0x802143 <udi_cdc_rx_pos>
     7a4:	70 91 44 21 	lds	r23, 0x2144	; 0x802144 <udi_cdc_rx_pos+0x1>
     7a8:	02 2f       	mov	r16, r18
     7aa:	10 e0       	ldi	r17, 0x00	; 0
     7ac:	f8 01       	movw	r30, r16
     7ae:	ee 0f       	add	r30, r30
     7b0:	ff 1f       	adc	r31, r31
     7b2:	ea 5b       	subi	r30, 0xBA	; 186
     7b4:	fe 4d       	sbci	r31, 0xDE	; 222
     7b6:	40 81       	ld	r20, Z
     7b8:	51 81       	ldd	r21, Z+1	; 0x01
     7ba:	64 17       	cp	r22, r20
     7bc:	75 07       	cpc	r23, r21
     7be:	18 f4       	brcc	.+6      	; 0x7c6 <udi_cdc_rx_start+0x48>
     7c0:	9f bf       	out	0x3f, r25	; 63
     7c2:	80 e0       	ldi	r24, 0x00	; 0
     7c4:	29 c0       	rjmp	.+82     	; 0x818 <udi_cdc_rx_start+0x9a>
     7c6:	10 92 43 21 	sts	0x2143, r1	; 0x802143 <udi_cdc_rx_pos>
     7ca:	10 92 44 21 	sts	0x2144, r1	; 0x802144 <udi_cdc_rx_pos+0x1>
     7ce:	81 e0       	ldi	r24, 0x01	; 1
     7d0:	21 11       	cpse	r18, r1
     7d2:	80 e0       	ldi	r24, 0x00	; 0
     7d4:	80 93 45 21 	sts	0x2145, r24	; 0x802145 <udi_cdc_rx_buf_sel>
     7d8:	81 e0       	ldi	r24, 0x01	; 1
     7da:	80 93 42 21 	sts	0x2142, r24	; 0x802142 <udi_cdc_rx_trans_ongoing>
     7de:	9f bf       	out	0x3f, r25	; 63
     7e0:	80 e0       	ldi	r24, 0x00	; 0
     7e2:	0e 94 b7 03 	call	0x76e	; 0x76e <udi_cdc_multi_is_rx_ready>
     7e6:	88 23       	and	r24, r24
     7e8:	19 f0       	breq	.+6      	; 0x7f0 <udi_cdc_rx_start+0x72>
     7ea:	80 e0       	ldi	r24, 0x00	; 0
     7ec:	0e 94 2d 12 	call	0x245a	; 0x245a <uart_rx_notify>
     7f0:	a8 01       	movw	r20, r16
     7f2:	00 24       	eor	r0, r0
     7f4:	56 95       	lsr	r21
     7f6:	47 95       	ror	r20
     7f8:	07 94       	ror	r0
     7fa:	56 95       	lsr	r21
     7fc:	47 95       	ror	r20
     7fe:	07 94       	ror	r0
     800:	54 2f       	mov	r21, r20
     802:	40 2d       	mov	r20, r0
     804:	46 5b       	subi	r20, 0xB6	; 182
     806:	5e 4d       	sbci	r21, 0xDE	; 222
     808:	06 e4       	ldi	r16, 0x46	; 70
     80a:	14 e0       	ldi	r17, 0x04	; 4
     80c:	20 e4       	ldi	r18, 0x40	; 64
     80e:	30 e0       	ldi	r19, 0x00	; 0
     810:	61 e0       	ldi	r22, 0x01	; 1
     812:	82 e0       	ldi	r24, 0x02	; 2
     814:	0e 94 57 0e 	call	0x1cae	; 0x1cae <udd_ep_run>
     818:	0f 90       	pop	r0
     81a:	df 91       	pop	r29
     81c:	cf 91       	pop	r28
     81e:	1f 91       	pop	r17
     820:	0f 91       	pop	r16
     822:	08 95       	ret

00000824 <udi_cdc_data_enable>:
     824:	10 92 cb 21 	sts	0x21CB, r1	; 0x8021cb <udi_cdc_nb_data_enabled>
     828:	10 92 b9 20 	sts	0x20B9, r1	; 0x8020b9 <udi_cdc_tx_trans_ongoing>
     82c:	10 92 b8 20 	sts	0x20B8, r1	; 0x8020b8 <udi_cdc_tx_both_buf_to_send>
     830:	10 92 bc 20 	sts	0x20BC, r1	; 0x8020bc <udi_cdc_tx_buf_sel>
     834:	ed eb       	ldi	r30, 0xBD	; 189
     836:	f0 e2       	ldi	r31, 0x20	; 32
     838:	10 82       	st	Z, r1
     83a:	11 82       	std	Z+1, r1	; 0x01
     83c:	12 82       	std	Z+2, r1	; 0x02
     83e:	13 82       	std	Z+3, r1	; 0x03
     840:	10 92 ba 20 	sts	0x20BA, r1	; 0x8020ba <udi_cdc_tx_sof_num>
     844:	10 92 bb 20 	sts	0x20BB, r1	; 0x8020bb <udi_cdc_tx_sof_num+0x1>
     848:	80 e0       	ldi	r24, 0x00	; 0
     84a:	0e 94 f7 01 	call	0x3ee	; 0x3ee <udi_cdc_tx_send>
     84e:	10 92 42 21 	sts	0x2142, r1	; 0x802142 <udi_cdc_rx_trans_ongoing>
     852:	10 92 45 21 	sts	0x2145, r1	; 0x802145 <udi_cdc_rx_buf_sel>
     856:	e6 e4       	ldi	r30, 0x46	; 70
     858:	f1 e2       	ldi	r31, 0x21	; 33
     85a:	10 82       	st	Z, r1
     85c:	11 82       	std	Z+1, r1	; 0x01
     85e:	12 82       	std	Z+2, r1	; 0x02
     860:	13 82       	std	Z+3, r1	; 0x03
     862:	10 92 43 21 	sts	0x2143, r1	; 0x802143 <udi_cdc_rx_pos>
     866:	10 92 44 21 	sts	0x2144, r1	; 0x802144 <udi_cdc_rx_pos+0x1>
     86a:	80 e0       	ldi	r24, 0x00	; 0
     86c:	0e 94 bf 03 	call	0x77e	; 0x77e <udi_cdc_rx_start>
     870:	88 23       	and	r24, r24
     872:	59 f0       	breq	.+22     	; 0x88a <udi_cdc_data_enable+0x66>
     874:	90 91 cb 21 	lds	r25, 0x21CB	; 0x8021cb <udi_cdc_nb_data_enabled>
     878:	9f 5f       	subi	r25, 0xFF	; 255
     87a:	90 93 cb 21 	sts	0x21CB, r25	; 0x8021cb <udi_cdc_nb_data_enabled>
     87e:	90 91 cb 21 	lds	r25, 0x21CB	; 0x8021cb <udi_cdc_nb_data_enabled>
     882:	91 30       	cpi	r25, 0x01	; 1
     884:	11 f4       	brne	.+4      	; 0x88a <udi_cdc_data_enable+0x66>
     886:	90 93 ca 21 	sts	0x21CA, r25	; 0x8021ca <udi_cdc_data_running>
     88a:	08 95       	ret

0000088c <udi_cdc_data_received>:
     88c:	0f 93       	push	r16
     88e:	1f 93       	push	r17
     890:	81 11       	cpse	r24, r1
     892:	2a c0       	rjmp	.+84     	; 0x8e8 <udi_cdc_data_received+0x5c>
     894:	80 91 45 21 	lds	r24, 0x2145	; 0x802145 <udi_cdc_rx_buf_sel>
     898:	e1 e0       	ldi	r30, 0x01	; 1
     89a:	81 11       	cpse	r24, r1
     89c:	e0 e0       	ldi	r30, 0x00	; 0
     89e:	84 2f       	mov	r24, r20
     8a0:	61 15       	cp	r22, r1
     8a2:	71 05       	cpc	r23, r1
     8a4:	a9 f4       	brne	.+42     	; 0x8d0 <udi_cdc_data_received+0x44>
     8a6:	f0 e0       	ldi	r31, 0x00	; 0
     8a8:	00 24       	eor	r0, r0
     8aa:	f6 95       	lsr	r31
     8ac:	e7 95       	ror	r30
     8ae:	07 94       	ror	r0
     8b0:	f6 95       	lsr	r31
     8b2:	e7 95       	ror	r30
     8b4:	07 94       	ror	r0
     8b6:	fe 2f       	mov	r31, r30
     8b8:	e0 2d       	mov	r30, r0
     8ba:	af 01       	movw	r20, r30
     8bc:	46 5b       	subi	r20, 0xB6	; 182
     8be:	5e 4d       	sbci	r21, 0xDE	; 222
     8c0:	06 e4       	ldi	r16, 0x46	; 70
     8c2:	14 e0       	ldi	r17, 0x04	; 4
     8c4:	20 e4       	ldi	r18, 0x40	; 64
     8c6:	30 e0       	ldi	r19, 0x00	; 0
     8c8:	61 e0       	ldi	r22, 0x01	; 1
     8ca:	0e 94 57 0e 	call	0x1cae	; 0x1cae <udd_ep_run>
     8ce:	0c c0       	rjmp	.+24     	; 0x8e8 <udi_cdc_data_received+0x5c>
     8d0:	f0 e0       	ldi	r31, 0x00	; 0
     8d2:	ee 0f       	add	r30, r30
     8d4:	ff 1f       	adc	r31, r31
     8d6:	ea 5b       	subi	r30, 0xBA	; 186
     8d8:	fe 4d       	sbci	r31, 0xDE	; 222
     8da:	60 83       	st	Z, r22
     8dc:	71 83       	std	Z+1, r23	; 0x01
     8de:	10 92 42 21 	sts	0x2142, r1	; 0x802142 <udi_cdc_rx_trans_ongoing>
     8e2:	80 e0       	ldi	r24, 0x00	; 0
     8e4:	0e 94 bf 03 	call	0x77e	; 0x77e <udi_cdc_rx_start>
     8e8:	1f 91       	pop	r17
     8ea:	0f 91       	pop	r16
     8ec:	08 95       	ret

000008ee <udi_cdc_is_rx_ready>:
     8ee:	80 e0       	ldi	r24, 0x00	; 0
     8f0:	0e 94 b7 03 	call	0x76e	; 0x76e <udi_cdc_multi_is_rx_ready>
     8f4:	08 95       	ret

000008f6 <udi_cdc_multi_getc>:
     8f6:	ef 92       	push	r14
     8f8:	ff 92       	push	r15
     8fa:	1f 93       	push	r17
     8fc:	cf 93       	push	r28
     8fe:	df 93       	push	r29
     900:	1f 92       	push	r1
     902:	cd b7       	in	r28, 0x3d	; 61
     904:	de b7       	in	r29, 0x3e	; 62
     906:	11 e0       	ldi	r17, 0x01	; 1
     908:	80 91 e2 21 	lds	r24, 0x21E2	; 0x8021e2 <udi_cdc_line_coding+0x6>
     90c:	89 30       	cpi	r24, 0x09	; 9
     90e:	09 f0       	breq	.+2      	; 0x912 <udi_cdc_multi_getc+0x1c>
     910:	10 e0       	ldi	r17, 0x00	; 0
     912:	40 e0       	ldi	r20, 0x00	; 0
     914:	50 e0       	ldi	r21, 0x00	; 0
     916:	8f b7       	in	r24, 0x3f	; 63
     918:	89 83       	std	Y+1, r24	; 0x01
     91a:	f8 94       	cli
     91c:	a9 81       	ldd	r26, Y+1	; 0x01
     91e:	20 91 43 21 	lds	r18, 0x2143	; 0x802143 <udi_cdc_rx_pos>
     922:	30 91 44 21 	lds	r19, 0x2144	; 0x802144 <udi_cdc_rx_pos+0x1>
     926:	80 91 45 21 	lds	r24, 0x2145	; 0x802145 <udi_cdc_rx_buf_sel>
     92a:	90 e0       	ldi	r25, 0x00	; 0
     92c:	fc 01       	movw	r30, r24
     92e:	ee 0f       	add	r30, r30
     930:	ff 1f       	adc	r31, r31
     932:	ea 5b       	subi	r30, 0xBA	; 186
     934:	fe 4d       	sbci	r31, 0xDE	; 222
     936:	60 81       	ld	r22, Z
     938:	71 81       	ldd	r23, Z+1	; 0x01
     93a:	af bf       	out	0x3f, r26	; 63
     93c:	26 17       	cp	r18, r22
     93e:	37 07       	cpc	r19, r23
     940:	30 f0       	brcs	.+12     	; 0x94e <udi_cdc_multi_getc+0x58>
     942:	80 91 ca 21 	lds	r24, 0x21CA	; 0x8021ca <udi_cdc_data_running>
     946:	81 11       	cpse	r24, r1
     948:	e6 cf       	rjmp	.-52     	; 0x916 <udi_cdc_multi_getc+0x20>
     94a:	90 e0       	ldi	r25, 0x00	; 0
     94c:	22 c0       	rjmp	.+68     	; 0x992 <udi_cdc_multi_getc+0x9c>
     94e:	fc 01       	movw	r30, r24
     950:	00 24       	eor	r0, r0
     952:	f6 95       	lsr	r31
     954:	e7 95       	ror	r30
     956:	07 94       	ror	r0
     958:	f6 95       	lsr	r31
     95a:	e7 95       	ror	r30
     95c:	07 94       	ror	r0
     95e:	fe 2f       	mov	r31, r30
     960:	e0 2d       	mov	r30, r0
     962:	e2 0f       	add	r30, r18
     964:	f3 1f       	adc	r31, r19
     966:	e6 5b       	subi	r30, 0xB6	; 182
     968:	fe 4d       	sbci	r31, 0xDE	; 222
     96a:	80 81       	ld	r24, Z
     96c:	7a 01       	movw	r14, r20
     96e:	e8 2a       	or	r14, r24
     970:	2f 5f       	subi	r18, 0xFF	; 255
     972:	3f 4f       	sbci	r19, 0xFF	; 255
     974:	20 93 43 21 	sts	0x2143, r18	; 0x802143 <udi_cdc_rx_pos>
     978:	30 93 44 21 	sts	0x2144, r19	; 0x802144 <udi_cdc_rx_pos+0x1>
     97c:	80 e0       	ldi	r24, 0x00	; 0
     97e:	0e 94 bf 03 	call	0x77e	; 0x77e <udi_cdc_rx_start>
     982:	11 23       	and	r17, r17
     984:	21 f0       	breq	.+8      	; 0x98e <udi_cdc_multi_getc+0x98>
     986:	5e 2d       	mov	r21, r14
     988:	44 27       	eor	r20, r20
     98a:	10 e0       	ldi	r17, 0x00	; 0
     98c:	c4 cf       	rjmp	.-120    	; 0x916 <udi_cdc_multi_getc+0x20>
     98e:	8e 2d       	mov	r24, r14
     990:	9f 2d       	mov	r25, r15
     992:	0f 90       	pop	r0
     994:	df 91       	pop	r29
     996:	cf 91       	pop	r28
     998:	1f 91       	pop	r17
     99a:	ff 90       	pop	r15
     99c:	ef 90       	pop	r14
     99e:	08 95       	ret

000009a0 <udi_cdc_getc>:
     9a0:	80 e0       	ldi	r24, 0x00	; 0
     9a2:	0e 94 7b 04 	call	0x8f6	; 0x8f6 <udi_cdc_multi_getc>
     9a6:	08 95       	ret

000009a8 <udi_cdc_multi_get_free_tx_buffer>:
     9a8:	cf 93       	push	r28
     9aa:	df 93       	push	r29
     9ac:	1f 92       	push	r1
     9ae:	cd b7       	in	r28, 0x3d	; 61
     9b0:	de b7       	in	r29, 0x3e	; 62
     9b2:	8f b7       	in	r24, 0x3f	; 63
     9b4:	89 83       	std	Y+1, r24	; 0x01
     9b6:	f8 94       	cli
     9b8:	99 81       	ldd	r25, Y+1	; 0x01
     9ba:	80 91 bc 20 	lds	r24, 0x20BC	; 0x8020bc <udi_cdc_tx_buf_sel>
     9be:	e8 2f       	mov	r30, r24
     9c0:	f0 e0       	ldi	r31, 0x00	; 0
     9c2:	ee 0f       	add	r30, r30
     9c4:	ff 1f       	adc	r31, r31
     9c6:	e3 54       	subi	r30, 0x43	; 67
     9c8:	ff 4d       	sbci	r31, 0xDF	; 223
     9ca:	20 81       	ld	r18, Z
     9cc:	31 81       	ldd	r19, Z+1	; 0x01
     9ce:	20 34       	cpi	r18, 0x40	; 64
     9d0:	31 05       	cpc	r19, r1
     9d2:	89 f4       	brne	.+34     	; 0x9f6 <udi_cdc_multi_get_free_tx_buffer+0x4e>
     9d4:	40 91 b9 20 	lds	r20, 0x20B9	; 0x8020b9 <udi_cdc_tx_trans_ongoing>
     9d8:	41 11       	cpse	r20, r1
     9da:	0d c0       	rjmp	.+26     	; 0x9f6 <udi_cdc_multi_get_free_tx_buffer+0x4e>
     9dc:	40 91 b8 20 	lds	r20, 0x20B8	; 0x8020b8 <udi_cdc_tx_both_buf_to_send>
     9e0:	41 11       	cpse	r20, r1
     9e2:	09 c0       	rjmp	.+18     	; 0x9f6 <udi_cdc_multi_get_free_tx_buffer+0x4e>
     9e4:	21 e0       	ldi	r18, 0x01	; 1
     9e6:	20 93 b8 20 	sts	0x20B8, r18	; 0x8020b8 <udi_cdc_tx_both_buf_to_send>
     9ea:	81 11       	cpse	r24, r1
     9ec:	20 e0       	ldi	r18, 0x00	; 0
     9ee:	20 93 bc 20 	sts	0x20BC, r18	; 0x8020bc <udi_cdc_tx_buf_sel>
     9f2:	20 e0       	ldi	r18, 0x00	; 0
     9f4:	30 e0       	ldi	r19, 0x00	; 0
     9f6:	9f bf       	out	0x3f, r25	; 63
     9f8:	80 e4       	ldi	r24, 0x40	; 64
     9fa:	90 e0       	ldi	r25, 0x00	; 0
     9fc:	82 1b       	sub	r24, r18
     9fe:	93 0b       	sbc	r25, r19
     a00:	0f 90       	pop	r0
     a02:	df 91       	pop	r29
     a04:	cf 91       	pop	r28
     a06:	08 95       	ret

00000a08 <udi_cdc_multi_is_tx_ready>:

bool udi_cdc_multi_is_tx_ready(uint8_t port)
{
	return (udi_cdc_multi_get_free_tx_buffer(port) != 0);
     a08:	0e 94 d4 04 	call	0x9a8	; 0x9a8 <udi_cdc_multi_get_free_tx_buffer>
     a0c:	21 e0       	ldi	r18, 0x01	; 1
     a0e:	89 2b       	or	r24, r25
     a10:	09 f4       	brne	.+2      	; 0xa14 <udi_cdc_multi_is_tx_ready+0xc>
     a12:	20 e0       	ldi	r18, 0x00	; 0
}
     a14:	82 2f       	mov	r24, r18
     a16:	08 95       	ret

00000a18 <udi_cdc_is_tx_ready>:

bool udi_cdc_is_tx_ready(void)
{
	return udi_cdc_multi_is_tx_ready(0);
     a18:	80 e0       	ldi	r24, 0x00	; 0
     a1a:	0e 94 04 05 	call	0xa08	; 0xa08 <udi_cdc_multi_is_tx_ready>
}
     a1e:	08 95       	ret

00000a20 <udi_cdc_multi_putc>:

int udi_cdc_multi_putc(uint8_t port, int value)
{
     a20:	ff 92       	push	r15
     a22:	0f 93       	push	r16
     a24:	1f 93       	push	r17
     a26:	cf 93       	push	r28
     a28:	df 93       	push	r29
     a2a:	1f 92       	push	r1
     a2c:	cd b7       	in	r28, 0x3d	; 61
     a2e:	de b7       	in	r29, 0x3e	; 62
     a30:	f6 2e       	mov	r15, r22
     a32:	17 2f       	mov	r17, r23

#if UDI_CDC_PORT_NB == 1 // To optimize code
	port = 0;
#endif

	b_databit_9 = (9 == udi_cdc_line_coding[port].bDataBits);
     a34:	01 e0       	ldi	r16, 0x01	; 1
     a36:	80 91 e2 21 	lds	r24, 0x21E2	; 0x8021e2 <udi_cdc_line_coding+0x6>
     a3a:	89 30       	cpi	r24, 0x09	; 9
     a3c:	09 f0       	breq	.+2      	; 0xa40 <udi_cdc_multi_putc+0x20>
     a3e:	00 e0       	ldi	r16, 0x00	; 0

udi_cdc_putc_process_one_byte:
	// Check available space
	if (!udi_cdc_multi_is_tx_ready(port)) {
     a40:	80 e0       	ldi	r24, 0x00	; 0
     a42:	0e 94 04 05 	call	0xa08	; 0xa08 <udi_cdc_multi_is_tx_ready>
     a46:	81 11       	cpse	r24, r1
     a48:	07 c0       	rjmp	.+14     	; 0xa58 <udi_cdc_multi_putc+0x38>
		if (!udi_cdc_data_running) {
     a4a:	80 91 ca 21 	lds	r24, 0x21CA	; 0x8021ca <udi_cdc_data_running>
     a4e:	81 11       	cpse	r24, r1
     a50:	f7 cf       	rjmp	.-18     	; 0xa40 <udi_cdc_multi_putc+0x20>
			return false;
     a52:	80 e0       	ldi	r24, 0x00	; 0
     a54:	90 e0       	ldi	r25, 0x00	; 0
     a56:	2d c0       	rjmp	.+90     	; 0xab2 <udi_cdc_multi_putc+0x92>

typedef uint8_t irqflags_t;

static inline irqflags_t cpu_irq_save(void)
{
	volatile irqflags_t flags = SREG;
     a58:	8f b7       	in	r24, 0x3f	; 63
     a5a:	89 83       	std	Y+1, r24	; 0x01
	cpu_irq_disable();
     a5c:	f8 94       	cli
	return flags;
     a5e:	29 81       	ldd	r18, Y+1	; 0x01
		goto udi_cdc_putc_process_one_byte;
	}

	// Write value
	flags = cpu_irq_save();
	buf_sel = udi_cdc_tx_buf_sel[port];
     a60:	e0 91 bc 20 	lds	r30, 0x20BC	; 0x8020bc <udi_cdc_tx_buf_sel>
	udi_cdc_tx_buf[port][buf_sel][udi_cdc_tx_buf_nb[port][buf_sel]++] = value;
     a64:	f0 e0       	ldi	r31, 0x00	; 0
     a66:	df 01       	movw	r26, r30
     a68:	aa 0f       	add	r26, r26
     a6a:	bb 1f       	adc	r27, r27
     a6c:	a3 54       	subi	r26, 0x43	; 67
     a6e:	bf 4d       	sbci	r27, 0xDF	; 223
     a70:	8d 91       	ld	r24, X+
     a72:	9c 91       	ld	r25, X
     a74:	11 97       	sbiw	r26, 0x01	; 1
     a76:	ac 01       	movw	r20, r24
     a78:	4f 5f       	subi	r20, 0xFF	; 255
     a7a:	5f 4f       	sbci	r21, 0xFF	; 255
     a7c:	4d 93       	st	X+, r20
     a7e:	5c 93       	st	X, r21
     a80:	00 24       	eor	r0, r0
     a82:	f6 95       	lsr	r31
     a84:	e7 95       	ror	r30
     a86:	07 94       	ror	r0
     a88:	f6 95       	lsr	r31
     a8a:	e7 95       	ror	r30
     a8c:	07 94       	ror	r0
     a8e:	fe 2f       	mov	r31, r30
     a90:	e0 2d       	mov	r30, r0
     a92:	8e 0f       	add	r24, r30
     a94:	9f 1f       	adc	r25, r31
     a96:	fc 01       	movw	r30, r24
     a98:	ee 53       	subi	r30, 0x3E	; 62
     a9a:	ff 4d       	sbci	r31, 0xDF	; 223
     a9c:	f0 82       	st	Z, r15
}

static inline void cpu_irq_restore(irqflags_t flags)
{
	barrier();
	SREG = flags;
     a9e:	2f bf       	out	0x3f, r18	; 63
	cpu_irq_restore(flags);

	if (b_databit_9) {
     aa0:	00 23       	and	r16, r16
     aa2:	29 f0       	breq	.+10     	; 0xaae <udi_cdc_multi_putc+0x8e>
		// Send MSB
		b_databit_9 = false;
		value = value >> 8;
     aa4:	f1 2e       	mov	r15, r17
     aa6:	11 0f       	add	r17, r17
     aa8:	11 0b       	sbc	r17, r17
	udi_cdc_tx_buf[port][buf_sel][udi_cdc_tx_buf_nb[port][buf_sel]++] = value;
	cpu_irq_restore(flags);

	if (b_databit_9) {
		// Send MSB
		b_databit_9 = false;
     aaa:	00 e0       	ldi	r16, 0x00	; 0
		value = value >> 8;
		goto udi_cdc_putc_process_one_byte;
     aac:	c9 cf       	rjmp	.-110    	; 0xa40 <udi_cdc_multi_putc+0x20>
	}
	return true;
     aae:	81 e0       	ldi	r24, 0x01	; 1
     ab0:	90 e0       	ldi	r25, 0x00	; 0
}
     ab2:	0f 90       	pop	r0
     ab4:	df 91       	pop	r29
     ab6:	cf 91       	pop	r28
     ab8:	1f 91       	pop	r17
     aba:	0f 91       	pop	r16
     abc:	ff 90       	pop	r15
     abe:	08 95       	ret

00000ac0 <udi_cdc_putc>:

int udi_cdc_putc(int value)
{
	return udi_cdc_multi_putc(0, value);
     ac0:	bc 01       	movw	r22, r24
     ac2:	80 e0       	ldi	r24, 0x00	; 0
     ac4:	0e 94 10 05 	call	0xa20	; 0xa20 <udi_cdc_multi_putc>
}
     ac8:	08 95       	ret

00000aca <udc_next_desc_in_iface>:
/*! \brief Stop the USB Device stack
 */
void udc_stop(void)
{
	udd_disable();
	udc_reset();
     aca:	e0 91 e8 21 	lds	r30, 0x21E8	; 0x8021e8 <udc_ptr_conf>
     ace:	f0 91 e9 21 	lds	r31, 0x21E9	; 0x8021e9 <udc_ptr_conf+0x1>
     ad2:	01 90       	ld	r0, Z+
     ad4:	f0 81       	ld	r31, Z
     ad6:	e0 2d       	mov	r30, r0
     ad8:	22 81       	ldd	r18, Z+2	; 0x02
     ada:	33 81       	ldd	r19, Z+3	; 0x03
     adc:	2e 0f       	add	r18, r30
     ade:	3f 1f       	adc	r19, r31
     ae0:	fc 01       	movw	r30, r24
     ae2:	40 81       	ld	r20, Z
     ae4:	e4 0f       	add	r30, r20
     ae6:	f1 1d       	adc	r31, r1
     ae8:	e2 17       	cp	r30, r18
     aea:	f3 07       	cpc	r31, r19
     aec:	b8 f4       	brcc	.+46     	; 0xb1c <udc_next_desc_in_iface+0x52>
     aee:	81 81       	ldd	r24, Z+1	; 0x01
     af0:	84 30       	cpi	r24, 0x04	; 4
     af2:	b9 f0       	breq	.+46     	; 0xb22 <udc_next_desc_in_iface+0x58>
     af4:	86 13       	cpse	r24, r22
     af6:	09 c0       	rjmp	.+18     	; 0xb0a <udc_next_desc_in_iface+0x40>
     af8:	05 c0       	rjmp	.+10     	; 0xb04 <udc_next_desc_in_iface+0x3a>
     afa:	81 81       	ldd	r24, Z+1	; 0x01
     afc:	84 30       	cpi	r24, 0x04	; 4
     afe:	a1 f0       	breq	.+40     	; 0xb28 <udc_next_desc_in_iface+0x5e>
     b00:	86 13       	cpse	r24, r22
     b02:	03 c0       	rjmp	.+6      	; 0xb0a <udc_next_desc_in_iface+0x40>
     b04:	8e 2f       	mov	r24, r30
     b06:	9f 2f       	mov	r25, r31
     b08:	08 95       	ret
     b0a:	80 81       	ld	r24, Z
     b0c:	e8 0f       	add	r30, r24
     b0e:	f1 1d       	adc	r31, r1
     b10:	e2 17       	cp	r30, r18
     b12:	f3 07       	cpc	r31, r19
     b14:	90 f3       	brcs	.-28     	; 0xafa <udc_next_desc_in_iface+0x30>
     b16:	80 e0       	ldi	r24, 0x00	; 0
     b18:	90 e0       	ldi	r25, 0x00	; 0
     b1a:	08 95       	ret
     b1c:	80 e0       	ldi	r24, 0x00	; 0
     b1e:	90 e0       	ldi	r25, 0x00	; 0
     b20:	08 95       	ret
     b22:	80 e0       	ldi	r24, 0x00	; 0
     b24:	90 e0       	ldi	r25, 0x00	; 0
     b26:	08 95       	ret
     b28:	80 e0       	ldi	r24, 0x00	; 0
     b2a:	90 e0       	ldi	r25, 0x00	; 0
     b2c:	08 95       	ret

00000b2e <udc_valid_address>:
     b2e:	80 91 32 23 	lds	r24, 0x2332	; 0x802332 <udd_g_ctrlreq+0x2>
     b32:	8f 77       	andi	r24, 0x7F	; 127
     b34:	0e 94 67 0d 	call	0x1ace	; 0x1ace <udd_set_address>
     b38:	08 95       	ret

00000b3a <udc_update_iface_desc>:
     b3a:	90 91 ea 21 	lds	r25, 0x21EA	; 0x8021ea <udc_num_configuration>
     b3e:	99 23       	and	r25, r25
     b40:	81 f1       	breq	.+96     	; 0xba2 <udc_update_iface_desc+0x68>
     b42:	e0 91 e8 21 	lds	r30, 0x21E8	; 0x8021e8 <udc_ptr_conf>
     b46:	f0 91 e9 21 	lds	r31, 0x21E9	; 0x8021e9 <udc_ptr_conf+0x1>
     b4a:	01 90       	ld	r0, Z+
     b4c:	f0 81       	ld	r31, Z
     b4e:	e0 2d       	mov	r30, r0
     b50:	94 81       	ldd	r25, Z+4	; 0x04
     b52:	89 17       	cp	r24, r25
     b54:	40 f5       	brcc	.+80     	; 0xba6 <udc_update_iface_desc+0x6c>
     b56:	e0 93 e6 21 	sts	0x21E6, r30	; 0x8021e6 <udc_ptr_iface>
     b5a:	f0 93 e7 21 	sts	0x21E7, r31	; 0x8021e7 <udc_ptr_iface+0x1>
     b5e:	22 81       	ldd	r18, Z+2	; 0x02
     b60:	33 81       	ldd	r19, Z+3	; 0x03
     b62:	2e 0f       	add	r18, r30
     b64:	3f 1f       	adc	r19, r31
     b66:	e2 17       	cp	r30, r18
     b68:	f3 07       	cpc	r31, r19
     b6a:	f8 f4       	brcc	.+62     	; 0xbaa <udc_update_iface_desc+0x70>
     b6c:	91 81       	ldd	r25, Z+1	; 0x01
     b6e:	94 30       	cpi	r25, 0x04	; 4
     b70:	61 f4       	brne	.+24     	; 0xb8a <udc_update_iface_desc+0x50>
     b72:	92 81       	ldd	r25, Z+2	; 0x02
     b74:	98 13       	cpse	r25, r24
     b76:	09 c0       	rjmp	.+18     	; 0xb8a <udc_update_iface_desc+0x50>
     b78:	93 81       	ldd	r25, Z+3	; 0x03
     b7a:	96 13       	cpse	r25, r22
     b7c:	06 c0       	rjmp	.+12     	; 0xb8a <udc_update_iface_desc+0x50>
     b7e:	e0 93 e6 21 	sts	0x21E6, r30	; 0x8021e6 <udc_ptr_iface>
     b82:	f0 93 e7 21 	sts	0x21E7, r31	; 0x8021e7 <udc_ptr_iface+0x1>
     b86:	81 e0       	ldi	r24, 0x01	; 1
     b88:	08 95       	ret
     b8a:	90 81       	ld	r25, Z
     b8c:	e9 0f       	add	r30, r25
     b8e:	f1 1d       	adc	r31, r1
     b90:	e2 17       	cp	r30, r18
     b92:	f3 07       	cpc	r31, r19
     b94:	58 f3       	brcs	.-42     	; 0xb6c <udc_update_iface_desc+0x32>
     b96:	e0 93 e6 21 	sts	0x21E6, r30	; 0x8021e6 <udc_ptr_iface>
     b9a:	f0 93 e7 21 	sts	0x21E7, r31	; 0x8021e7 <udc_ptr_iface+0x1>
     b9e:	80 e0       	ldi	r24, 0x00	; 0
     ba0:	08 95       	ret
     ba2:	80 e0       	ldi	r24, 0x00	; 0
     ba4:	08 95       	ret
     ba6:	80 e0       	ldi	r24, 0x00	; 0
     ba8:	08 95       	ret
     baa:	80 e0       	ldi	r24, 0x00	; 0
     bac:	08 95       	ret

00000bae <udc_iface_disable>:
     bae:	ef 92       	push	r14
     bb0:	ff 92       	push	r15
     bb2:	1f 93       	push	r17
     bb4:	cf 93       	push	r28
     bb6:	df 93       	push	r29
     bb8:	c8 2f       	mov	r28, r24
     bba:	60 e0       	ldi	r22, 0x00	; 0
     bbc:	0e 94 9d 05 	call	0xb3a	; 0xb3a <udc_update_iface_desc>
     bc0:	18 2f       	mov	r17, r24
     bc2:	88 23       	and	r24, r24
     bc4:	91 f1       	breq	.+100    	; 0xc2a <udc_iface_disable+0x7c>
     bc6:	a0 91 e8 21 	lds	r26, 0x21E8	; 0x8021e8 <udc_ptr_conf>
     bca:	b0 91 e9 21 	lds	r27, 0x21E9	; 0x8021e9 <udc_ptr_conf+0x1>
     bce:	ec 2f       	mov	r30, r28
     bd0:	f0 e0       	ldi	r31, 0x00	; 0
     bd2:	ee 0f       	add	r30, r30
     bd4:	ff 1f       	adc	r31, r31
     bd6:	12 96       	adiw	r26, 0x02	; 2
     bd8:	8d 91       	ld	r24, X+
     bda:	9c 91       	ld	r25, X
     bdc:	13 97       	sbiw	r26, 0x03	; 3
     bde:	e8 0f       	add	r30, r24
     be0:	f9 1f       	adc	r31, r25
     be2:	e0 80       	ld	r14, Z
     be4:	f1 80       	ldd	r15, Z+1	; 0x01
     be6:	d7 01       	movw	r26, r14
     be8:	16 96       	adiw	r26, 0x06	; 6
     bea:	ed 91       	ld	r30, X+
     bec:	fc 91       	ld	r31, X
     bee:	17 97       	sbiw	r26, 0x07	; 7
     bf0:	19 95       	eicall
     bf2:	68 2f       	mov	r22, r24
     bf4:	8c 2f       	mov	r24, r28
     bf6:	0e 94 9d 05 	call	0xb3a	; 0xb3a <udc_update_iface_desc>
     bfa:	18 2f       	mov	r17, r24
     bfc:	88 23       	and	r24, r24
     bfe:	a9 f0       	breq	.+42     	; 0xc2a <udc_iface_disable+0x7c>
     c00:	c0 91 e6 21 	lds	r28, 0x21E6	; 0x8021e6 <udc_ptr_iface>
     c04:	d0 91 e7 21 	lds	r29, 0x21E7	; 0x8021e7 <udc_ptr_iface+0x1>
     c08:	65 e0       	ldi	r22, 0x05	; 5
     c0a:	ce 01       	movw	r24, r28
     c0c:	0e 94 65 05 	call	0xaca	; 0xaca <udc_next_desc_in_iface>
     c10:	ec 01       	movw	r28, r24
     c12:	89 2b       	or	r24, r25
     c14:	21 f0       	breq	.+8      	; 0xc1e <udc_iface_disable+0x70>
     c16:	8a 81       	ldd	r24, Y+2	; 0x02
     c18:	0e 94 6c 0f 	call	0x1ed8	; 0x1ed8 <udd_ep_free>
     c1c:	f5 cf       	rjmp	.-22     	; 0xc08 <udc_iface_disable+0x5a>
     c1e:	d7 01       	movw	r26, r14
     c20:	12 96       	adiw	r26, 0x02	; 2
     c22:	ed 91       	ld	r30, X+
     c24:	fc 91       	ld	r31, X
     c26:	13 97       	sbiw	r26, 0x03	; 3
     c28:	19 95       	eicall
     c2a:	81 2f       	mov	r24, r17
     c2c:	df 91       	pop	r29
     c2e:	cf 91       	pop	r28
     c30:	1f 91       	pop	r17
     c32:	ff 90       	pop	r15
     c34:	ef 90       	pop	r14
     c36:	08 95       	ret

00000c38 <udc_iface_enable>:
     c38:	1f 93       	push	r17
     c3a:	cf 93       	push	r28
     c3c:	df 93       	push	r29
     c3e:	18 2f       	mov	r17, r24
     c40:	0e 94 9d 05 	call	0xb3a	; 0xb3a <udc_update_iface_desc>
     c44:	88 23       	and	r24, r24
     c46:	49 f1       	breq	.+82     	; 0xc9a <udc_iface_enable+0x62>
     c48:	c0 91 e6 21 	lds	r28, 0x21E6	; 0x8021e6 <udc_ptr_iface>
     c4c:	d0 91 e7 21 	lds	r29, 0x21E7	; 0x8021e7 <udc_ptr_iface+0x1>
     c50:	65 e0       	ldi	r22, 0x05	; 5
     c52:	ce 01       	movw	r24, r28
     c54:	0e 94 65 05 	call	0xaca	; 0xaca <udc_next_desc_in_iface>
     c58:	ec 01       	movw	r28, r24
     c5a:	89 2b       	or	r24, r25
     c5c:	49 f0       	breq	.+18     	; 0xc70 <udc_iface_enable+0x38>
     c5e:	4c 81       	ldd	r20, Y+4	; 0x04
     c60:	5d 81       	ldd	r21, Y+5	; 0x05
     c62:	6b 81       	ldd	r22, Y+3	; 0x03
     c64:	8a 81       	ldd	r24, Y+2	; 0x02
     c66:	0e 94 7c 0d 	call	0x1af8	; 0x1af8 <udd_ep_alloc>
     c6a:	81 11       	cpse	r24, r1
     c6c:	f1 cf       	rjmp	.-30     	; 0xc50 <udc_iface_enable+0x18>
     c6e:	15 c0       	rjmp	.+42     	; 0xc9a <udc_iface_enable+0x62>
     c70:	a0 91 e8 21 	lds	r26, 0x21E8	; 0x8021e8 <udc_ptr_conf>
     c74:	b0 91 e9 21 	lds	r27, 0x21E9	; 0x8021e9 <udc_ptr_conf+0x1>
     c78:	e1 2f       	mov	r30, r17
     c7a:	f0 e0       	ldi	r31, 0x00	; 0
     c7c:	ee 0f       	add	r30, r30
     c7e:	ff 1f       	adc	r31, r31
     c80:	12 96       	adiw	r26, 0x02	; 2
     c82:	8d 91       	ld	r24, X+
     c84:	9c 91       	ld	r25, X
     c86:	13 97       	sbiw	r26, 0x03	; 3
     c88:	e8 0f       	add	r30, r24
     c8a:	f9 1f       	adc	r31, r25
     c8c:	01 90       	ld	r0, Z+
     c8e:	f0 81       	ld	r31, Z
     c90:	e0 2d       	mov	r30, r0
     c92:	01 90       	ld	r0, Z+
     c94:	f0 81       	ld	r31, Z
     c96:	e0 2d       	mov	r30, r0
     c98:	19 95       	eicall
     c9a:	df 91       	pop	r29
     c9c:	cf 91       	pop	r28
     c9e:	1f 91       	pop	r17
     ca0:	08 95       	ret

00000ca2 <udc_reset>:
     ca2:	cf 93       	push	r28
     ca4:	80 91 ea 21 	lds	r24, 0x21EA	; 0x8021ea <udc_num_configuration>
     ca8:	88 23       	and	r24, r24
     caa:	c9 f0       	breq	.+50     	; 0xcde <udc_reset+0x3c>
     cac:	e0 91 e8 21 	lds	r30, 0x21E8	; 0x8021e8 <udc_ptr_conf>
     cb0:	f0 91 e9 21 	lds	r31, 0x21E9	; 0x8021e9 <udc_ptr_conf+0x1>
     cb4:	01 90       	ld	r0, Z+
     cb6:	f0 81       	ld	r31, Z
     cb8:	e0 2d       	mov	r30, r0
     cba:	84 81       	ldd	r24, Z+4	; 0x04
     cbc:	88 23       	and	r24, r24
     cbe:	79 f0       	breq	.+30     	; 0xcde <udc_reset+0x3c>
     cc0:	c0 e0       	ldi	r28, 0x00	; 0
     cc2:	8c 2f       	mov	r24, r28
     cc4:	0e 94 d7 05 	call	0xbae	; 0xbae <udc_iface_disable>
     cc8:	cf 5f       	subi	r28, 0xFF	; 255
     cca:	e0 91 e8 21 	lds	r30, 0x21E8	; 0x8021e8 <udc_ptr_conf>
     cce:	f0 91 e9 21 	lds	r31, 0x21E9	; 0x8021e9 <udc_ptr_conf+0x1>
     cd2:	01 90       	ld	r0, Z+
     cd4:	f0 81       	ld	r31, Z
     cd6:	e0 2d       	mov	r30, r0
     cd8:	84 81       	ldd	r24, Z+4	; 0x04
     cda:	c8 17       	cp	r28, r24
     cdc:	90 f3       	brcs	.-28     	; 0xcc2 <udc_reset+0x20>
     cde:	10 92 ea 21 	sts	0x21EA, r1	; 0x8021ea <udc_num_configuration>
     ce2:	81 e0       	ldi	r24, 0x01	; 1
     ce4:	90 e0       	ldi	r25, 0x00	; 0
     ce6:	80 93 ee 21 	sts	0x21EE, r24	; 0x8021ee <udc_device_status>
     cea:	90 93 ef 21 	sts	0x21EF, r25	; 0x8021ef <udc_device_status+0x1>
     cee:	cf 91       	pop	r28
     cf0:	08 95       	ret

00000cf2 <udc_sof_notify>:
			CPU_TO_LE16(USB_DEV_STATUS_BUS_POWERED);
#endif
}

void udc_sof_notify(void)
{
     cf2:	cf 93       	push	r28
	uint8_t iface_num;

	if (udc_num_configuration) {
     cf4:	80 91 ea 21 	lds	r24, 0x21EA	; 0x8021ea <udc_num_configuration>
     cf8:	88 23       	and	r24, r24
     cfa:	49 f1       	breq	.+82     	; 0xd4e <udc_sof_notify+0x5c>
		for (iface_num = 0;
				iface_num < udc_ptr_conf->desc->bNumInterfaces;
     cfc:	a0 91 e8 21 	lds	r26, 0x21E8	; 0x8021e8 <udc_ptr_conf>
     d00:	b0 91 e9 21 	lds	r27, 0x21E9	; 0x8021e9 <udc_ptr_conf+0x1>
     d04:	ed 91       	ld	r30, X+
     d06:	fc 91       	ld	r31, X
     d08:	11 97       	sbiw	r26, 0x01	; 1
void udc_sof_notify(void)
{
	uint8_t iface_num;

	if (udc_num_configuration) {
		for (iface_num = 0;
     d0a:	84 81       	ldd	r24, Z+4	; 0x04
     d0c:	88 23       	and	r24, r24
     d0e:	f9 f0       	breq	.+62     	; 0xd4e <udc_sof_notify+0x5c>
     d10:	c0 e0       	ldi	r28, 0x00	; 0
				iface_num < udc_ptr_conf->desc->bNumInterfaces;
				iface_num++) {
			if (udc_ptr_conf->udi_apis[iface_num]->sof_notify != NULL) {
     d12:	ec 2f       	mov	r30, r28
     d14:	f0 e0       	ldi	r31, 0x00	; 0
     d16:	ee 0f       	add	r30, r30
     d18:	ff 1f       	adc	r31, r31
     d1a:	12 96       	adiw	r26, 0x02	; 2
     d1c:	8d 91       	ld	r24, X+
     d1e:	9c 91       	ld	r25, X
     d20:	13 97       	sbiw	r26, 0x03	; 3
     d22:	e8 0f       	add	r30, r24
     d24:	f9 1f       	adc	r31, r25
     d26:	01 90       	ld	r0, Z+
     d28:	f0 81       	ld	r31, Z
     d2a:	e0 2d       	mov	r30, r0
     d2c:	00 84       	ldd	r0, Z+8	; 0x08
     d2e:	f1 85       	ldd	r31, Z+9	; 0x09
     d30:	e0 2d       	mov	r30, r0
     d32:	30 97       	sbiw	r30, 0x00	; 0
     d34:	09 f0       	breq	.+2      	; 0xd38 <udc_sof_notify+0x46>
				udc_ptr_conf->udi_apis[iface_num]->sof_notify();
     d36:	19 95       	eicall
	uint8_t iface_num;

	if (udc_num_configuration) {
		for (iface_num = 0;
				iface_num < udc_ptr_conf->desc->bNumInterfaces;
				iface_num++) {
     d38:	cf 5f       	subi	r28, 0xFF	; 255
{
	uint8_t iface_num;

	if (udc_num_configuration) {
		for (iface_num = 0;
				iface_num < udc_ptr_conf->desc->bNumInterfaces;
     d3a:	a0 91 e8 21 	lds	r26, 0x21E8	; 0x8021e8 <udc_ptr_conf>
     d3e:	b0 91 e9 21 	lds	r27, 0x21E9	; 0x8021e9 <udc_ptr_conf+0x1>
     d42:	ed 91       	ld	r30, X+
     d44:	fc 91       	ld	r31, X
     d46:	11 97       	sbiw	r26, 0x01	; 1
void udc_sof_notify(void)
{
	uint8_t iface_num;

	if (udc_num_configuration) {
		for (iface_num = 0;
     d48:	84 81       	ldd	r24, Z+4	; 0x04
     d4a:	c8 17       	cp	r28, r24
     d4c:	10 f3       	brcs	.-60     	; 0xd12 <udc_sof_notify+0x20>
			if (udc_ptr_conf->udi_apis[iface_num]->sof_notify != NULL) {
				udc_ptr_conf->udi_apis[iface_num]->sof_notify();
			}
		}
	}
}
     d4e:	cf 91       	pop	r28
     d50:	08 95       	ret

00000d52 <udc_process_setup>:
 * sent to a specific application callback.
 *
 * \return true if the request is supported, else the request is stalled by UDD
 */
bool udc_process_setup(void)
{
     d52:	0f 93       	push	r16
     d54:	1f 93       	push	r17
     d56:	cf 93       	push	r28
     d58:	df 93       	push	r29
	// By default no data (receive/send) and no callbacks registered
	udd_g_ctrlreq.payload_size = 0;
     d5a:	e0 e3       	ldi	r30, 0x30	; 48
     d5c:	f3 e2       	ldi	r31, 0x23	; 35
     d5e:	12 86       	std	Z+10, r1	; 0x0a
     d60:	13 86       	std	Z+11, r1	; 0x0b
	udd_g_ctrlreq.callback = NULL;
     d62:	14 86       	std	Z+12, r1	; 0x0c
     d64:	15 86       	std	Z+13, r1	; 0x0d
	udd_g_ctrlreq.over_under_run = NULL;
     d66:	16 86       	std	Z+14, r1	; 0x0e
     d68:	17 86       	std	Z+15, r1	; 0x0f

	if (Udd_setup_is_in()) {
     d6a:	80 81       	ld	r24, Z
     d6c:	88 23       	and	r24, r24
     d6e:	0c f0       	brlt	.+2      	; 0xd72 <udc_process_setup+0x20>
     d70:	70 c2       	rjmp	.+1248   	; 0x1252 <udc_process_setup+0x500>
		if (udd_g_ctrlreq.req.wLength == 0) {
     d72:	20 91 36 23 	lds	r18, 0x2336	; 0x802336 <udd_g_ctrlreq+0x6>
     d76:	30 91 37 23 	lds	r19, 0x2337	; 0x802337 <udd_g_ctrlreq+0x7>
     d7a:	21 15       	cp	r18, r1
     d7c:	31 05       	cpc	r19, r1
     d7e:	09 f0       	breq	.+2      	; 0xd82 <udc_process_setup+0x30>
     d80:	6d c2       	rjmp	.+1242   	; 0x125c <udc_process_setup+0x50a>
     d82:	63 c2       	rjmp	.+1222   	; 0x124a <udc_process_setup+0x4f8>
		// GET Standard Requests
		if (udd_g_ctrlreq.req.wLength == 0) {
			return false; // Error for USB host
		}

		if (USB_REQ_RECIP_DEVICE == Udd_setup_recipient()) {
     d84:	8f 71       	andi	r24, 0x1F	; 31
     d86:	09 f0       	breq	.+2      	; 0xd8a <udc_process_setup+0x38>
     d88:	aa c0       	rjmp	.+340    	; 0xede <udc_process_setup+0x18c>
			// Standard Get Device request
			switch (udd_g_ctrlreq.req.bRequest) {
     d8a:	90 91 31 23 	lds	r25, 0x2331	; 0x802331 <udd_g_ctrlreq+0x1>
     d8e:	96 30       	cpi	r25, 0x06	; 6
     d90:	81 f0       	breq	.+32     	; 0xdb2 <udc_process_setup+0x60>
     d92:	98 30       	cpi	r25, 0x08	; 8
     d94:	09 f4       	brne	.+2      	; 0xd98 <udc_process_setup+0x46>
     d96:	98 c0       	rjmp	.+304    	; 0xec8 <udc_process_setup+0x176>
     d98:	91 11       	cpse	r25, r1
     d9a:	a1 c0       	rjmp	.+322    	; 0xede <udc_process_setup+0x18c>
 *
 * \return true if success
 */
static bool udc_req_std_dev_get_status(void)
{
	if (udd_g_ctrlreq.req.wLength != sizeof(udc_device_status)) {
     d9c:	22 30       	cpi	r18, 0x02	; 2
     d9e:	31 05       	cpc	r19, r1
     da0:	09 f0       	breq	.+2      	; 0xda4 <udc_process_setup+0x52>
     da2:	d9 c1       	rjmp	.+946    	; 0x1156 <udc_process_setup+0x404>
		return false;
	}

	udd_set_setup_payload( (uint8_t *) & udc_device_status,
     da4:	62 e0       	ldi	r22, 0x02	; 2
     da6:	70 e0       	ldi	r23, 0x00	; 0
     da8:	8e ee       	ldi	r24, 0xEE	; 238
     daa:	91 e2       	ldi	r25, 0x21	; 33
     dac:	0e 94 75 0d 	call	0x1aea	; 0x1aea <udd_set_setup_payload>
     db0:	5a c2       	rjmp	.+1204   	; 0x1266 <udc_process_setup+0x514>
 */
static bool udc_req_std_dev_get_descriptor(void)
{
	uint8_t conf_num;

	conf_num = udd_g_ctrlreq.req.wValue & 0xff;
     db2:	80 91 32 23 	lds	r24, 0x2332	; 0x802332 <udd_g_ctrlreq+0x2>
     db6:	90 91 33 23 	lds	r25, 0x2333	; 0x802333 <udd_g_ctrlreq+0x3>

	// Check descriptor ID
	switch ((uint8_t) (udd_g_ctrlreq.req.wValue >> 8)) {
     dba:	29 2f       	mov	r18, r25
     dbc:	33 27       	eor	r19, r19
     dbe:	22 30       	cpi	r18, 0x02	; 2
     dc0:	31 05       	cpc	r19, r1
     dc2:	b1 f0       	breq	.+44     	; 0xdf0 <udc_process_setup+0x9e>
     dc4:	24 f4       	brge	.+8      	; 0xdce <udc_process_setup+0x7c>
     dc6:	21 30       	cpi	r18, 0x01	; 1
     dc8:	31 05       	cpc	r19, r1
     dca:	41 f0       	breq	.+16     	; 0xddc <udc_process_setup+0x8a>
     dcc:	bb c1       	rjmp	.+886    	; 0x1144 <udc_process_setup+0x3f2>
     dce:	23 30       	cpi	r18, 0x03	; 3
     dd0:	31 05       	cpc	r19, r1
     dd2:	f1 f1       	breq	.+124    	; 0xe50 <udc_process_setup+0xfe>
     dd4:	2f 30       	cpi	r18, 0x0F	; 15
     dd6:	31 05       	cpc	r19, r1
     dd8:	61 f1       	breq	.+88     	; 0xe32 <udc_process_setup+0xe0>
     dda:	b4 c1       	rjmp	.+872    	; 0x1144 <udc_process_setup+0x3f2>
		} else
#endif
		{
			udd_set_setup_payload(
				(uint8_t *) udc_config.confdev_lsfs,
				udc_config.confdev_lsfs->bLength);
     ddc:	80 91 14 20 	lds	r24, 0x2014	; 0x802014 <udc_config>
     de0:	90 91 15 20 	lds	r25, 0x2015	; 0x802015 <udc_config+0x1>
				(uint8_t *) udc_config.confdev_hs,
				udc_config.confdev_hs->bLength);
		} else
#endif
		{
			udd_set_setup_payload(
     de4:	dc 01       	movw	r26, r24
     de6:	6c 91       	ld	r22, X
     de8:	70 e0       	ldi	r23, 0x00	; 0
     dea:	0e 94 75 0d 	call	0x1aea	; 0x1aea <udd_set_setup_payload>
     dee:	5d c0       	rjmp	.+186    	; 0xeaa <udc_process_setup+0x158>
				le16_to_cpu(udc_config.conf_hs[conf_num].desc->wTotalLength));
		} else
#endif
		{
			// FS descriptor
			if (conf_num >= udc_config.confdev_lsfs->
     df0:	e0 91 14 20 	lds	r30, 0x2014	; 0x802014 <udc_config>
     df4:	f0 91 15 20 	lds	r31, 0x2015	; 0x802015 <udc_config+0x1>
     df8:	21 89       	ldd	r18, Z+17	; 0x11
     dfa:	82 17       	cp	r24, r18
     dfc:	08 f0       	brcs	.+2      	; 0xe00 <udc_process_setup+0xae>
     dfe:	ab c1       	rjmp	.+854    	; 0x1156 <udc_process_setup+0x404>
					bNumConfigurations) {
				return false;
			}
			udd_set_setup_payload(
				(uint8_t *)udc_config.conf_lsfs[conf_num].desc,
				le16_to_cpu(udc_config.conf_lsfs[conf_num].desc->wTotalLength));
     e00:	99 27       	eor	r25, r25
     e02:	88 0f       	add	r24, r24
     e04:	99 1f       	adc	r25, r25
     e06:	88 0f       	add	r24, r24
     e08:	99 1f       	adc	r25, r25
     e0a:	e0 91 16 20 	lds	r30, 0x2016	; 0x802016 <udc_config+0x2>
     e0e:	f0 91 17 20 	lds	r31, 0x2017	; 0x802017 <udc_config+0x3>
     e12:	e8 0f       	add	r30, r24
     e14:	f9 1f       	adc	r31, r25
     e16:	80 81       	ld	r24, Z
     e18:	91 81       	ldd	r25, Z+1	; 0x01
			// FS descriptor
			if (conf_num >= udc_config.confdev_lsfs->
					bNumConfigurations) {
				return false;
			}
			udd_set_setup_payload(
     e1a:	fc 01       	movw	r30, r24
     e1c:	62 81       	ldd	r22, Z+2	; 0x02
     e1e:	73 81       	ldd	r23, Z+3	; 0x03
     e20:	0e 94 75 0d 	call	0x1aea	; 0x1aea <udd_set_setup_payload>
				(uint8_t *)udc_config.conf_lsfs[conf_num].desc,
				le16_to_cpu(udc_config.conf_lsfs[conf_num].desc->wTotalLength));
		}
		((usb_conf_desc_t *) udd_g_ctrlreq.payload)->bDescriptorType =
     e24:	e0 91 38 23 	lds	r30, 0x2338	; 0x802338 <udd_g_ctrlreq+0x8>
     e28:	f0 91 39 23 	lds	r31, 0x2339	; 0x802339 <udd_g_ctrlreq+0x9>
     e2c:	82 e0       	ldi	r24, 0x02	; 2
     e2e:	81 83       	std	Z+1, r24	; 0x01
     e30:	3c c0       	rjmp	.+120    	; 0xeaa <udc_process_setup+0x158>
		break;
#endif

	case USB_DT_BOS:
		// Device BOS descriptor requested
		if (udc_config.conf_bos == NULL) {
     e32:	80 91 18 20 	lds	r24, 0x2018	; 0x802018 <udc_config+0x4>
     e36:	90 91 19 20 	lds	r25, 0x2019	; 0x802019 <udc_config+0x5>
     e3a:	00 97       	sbiw	r24, 0x00	; 0
     e3c:	09 f4       	brne	.+2      	; 0xe40 <udc_process_setup+0xee>
     e3e:	8b c1       	rjmp	.+790    	; 0x1156 <udc_process_setup+0x404>
			return false;
		}
		udd_set_setup_payload( (uint8_t *) udc_config.conf_bos,
     e40:	dc 01       	movw	r26, r24
     e42:	12 96       	adiw	r26, 0x02	; 2
     e44:	6d 91       	ld	r22, X+
     e46:	7c 91       	ld	r23, X
     e48:	13 97       	sbiw	r26, 0x03	; 3
     e4a:	0e 94 75 0d 	call	0x1aea	; 0x1aea <udd_set_setup_payload>
     e4e:	2d c0       	rjmp	.+90     	; 0xeaa <udc_process_setup+0x158>
	uint8_t i;
	const uint8_t *str;
	uint8_t str_length = 0;

	// Link payload pointer to the string corresponding at request
	switch (udd_g_ctrlreq.req.wValue & 0xff) {
     e50:	99 27       	eor	r25, r25
     e52:	81 30       	cpi	r24, 0x01	; 1
     e54:	91 05       	cpc	r25, r1
     e56:	79 f0       	breq	.+30     	; 0xe76 <udc_process_setup+0x124>
     e58:	38 f0       	brcs	.+14     	; 0xe68 <udc_process_setup+0x116>
     e5a:	02 97       	sbiw	r24, 0x02	; 2
     e5c:	09 f0       	breq	.+2      	; 0xe60 <udc_process_setup+0x10e>
     e5e:	7b c1       	rjmp	.+758    	; 0x1156 <udc_process_setup+0x404>
		break;
#endif
#ifdef USB_DEVICE_PRODUCT_NAME
	case 2:
		str_length = USB_DEVICE_PRODUCT_NAME_SIZE;
		str = udc_string_product_name;
     e60:	88 e9       	ldi	r24, 0x98	; 152
     e62:	90 e2       	ldi	r25, 0x20	; 32
		str = udc_string_manufacturer_name;
		break;
#endif
#ifdef USB_DEVICE_PRODUCT_NAME
	case 2:
		str_length = USB_DEVICE_PRODUCT_NAME_SIZE;
     e64:	2f e0       	ldi	r18, 0x0F	; 15
     e66:	0a c0       	rjmp	.+20     	; 0xe7c <udc_process_setup+0x12a>
	uint8_t str_length = 0;

	// Link payload pointer to the string corresponding at request
	switch (udd_g_ctrlreq.req.wValue & 0xff) {
	case 0:
		udd_set_setup_payload((uint8_t *) &udc_string_desc_languageid,
     e68:	64 e0       	ldi	r22, 0x04	; 4
     e6a:	70 e0       	ldi	r23, 0x00	; 0
     e6c:	82 eb       	ldi	r24, 0xB2	; 178
     e6e:	90 e2       	ldi	r25, 0x20	; 32
     e70:	0e 94 75 0d 	call	0x1aea	; 0x1aea <udd_set_setup_payload>
     e74:	1a c0       	rjmp	.+52     	; 0xeaa <udc_process_setup+0x158>
		break;

#ifdef USB_DEVICE_MANUFACTURE_NAME
	case 1:
		str_length = USB_DEVICE_MANUFACTURE_NAME_SIZE;
		str = udc_string_manufacturer_name;
     e76:	88 ea       	ldi	r24, 0xA8	; 168
     e78:	90 e2       	ldi	r25, 0x20	; 32
				sizeof(udc_string_desc_languageid));
		break;

#ifdef USB_DEVICE_MANUFACTURE_NAME
	case 1:
		str_length = USB_DEVICE_MANUFACTURE_NAME_SIZE;
     e7a:	29 e0       	ldi	r18, 0x09	; 9
     e7c:	38 2f       	mov	r19, r24
     e7e:	aa e7       	ldi	r26, 0x7A	; 122
     e80:	b0 e2       	ldi	r27, 0x20	; 32
		str = udc_string_manufacturer_name;
		break;
#endif
#ifdef USB_DEVICE_PRODUCT_NAME
	case 2:
		str_length = USB_DEVICE_PRODUCT_NAME_SIZE;
     e82:	e8 2f       	mov	r30, r24
     e84:	f9 2f       	mov	r31, r25
		return false;
	}

	if (str_length) {
		for(i = 0; i < str_length; i++) {
			udc_string_desc.string[i] = cpu_to_le16((le16_t)str[i]);
     e86:	81 91       	ld	r24, Z+
     e88:	90 e0       	ldi	r25, 0x00	; 0
     e8a:	8d 93       	st	X+, r24
     e8c:	9d 93       	st	X+, r25
     e8e:	8e 2f       	mov	r24, r30
     e90:	83 1b       	sub	r24, r19
#endif
		return false;
	}

	if (str_length) {
		for(i = 0; i < str_length; i++) {
     e92:	82 17       	cp	r24, r18
     e94:	c0 f3       	brcs	.-16     	; 0xe86 <udc_process_setup+0x134>
			udc_string_desc.string[i] = cpu_to_le16((le16_t)str[i]);
		}

		udc_string_desc.header.bLength = 2 + (str_length) * 2;
     e96:	62 2f       	mov	r22, r18
     e98:	66 0f       	add	r22, r22
     e9a:	6e 5f       	subi	r22, 0xFE	; 254
     e9c:	60 93 78 20 	sts	0x2078, r22	; 0x802078 <udc_string_desc>
		udd_set_setup_payload(
     ea0:	70 e0       	ldi	r23, 0x00	; 0
     ea2:	88 e7       	ldi	r24, 0x78	; 120
     ea4:	90 e2       	ldi	r25, 0x20	; 32
     ea6:	0e 94 75 0d 	call	0x1aea	; 0x1aea <udd_set_setup_payload>
	default:
		// Unknown descriptor requested
		return false;
	}
	// if the descriptor is larger than length requested, then reduce it
	if (udd_g_ctrlreq.req.wLength < udd_g_ctrlreq.payload_size) {
     eaa:	e0 e3       	ldi	r30, 0x30	; 48
     eac:	f3 e2       	ldi	r31, 0x23	; 35
     eae:	86 81       	ldd	r24, Z+6	; 0x06
     eb0:	97 81       	ldd	r25, Z+7	; 0x07
     eb2:	22 85       	ldd	r18, Z+10	; 0x0a
     eb4:	33 85       	ldd	r19, Z+11	; 0x0b
     eb6:	82 17       	cp	r24, r18
     eb8:	93 07       	cpc	r25, r19
     eba:	08 f0       	brcs	.+2      	; 0xebe <udc_process_setup+0x16c>
     ebc:	d4 c1       	rjmp	.+936    	; 0x1266 <udc_process_setup+0x514>
		udd_g_ctrlreq.payload_size = udd_g_ctrlreq.req.wLength;
     ebe:	80 93 3a 23 	sts	0x233A, r24	; 0x80233a <udd_g_ctrlreq+0xa>
     ec2:	90 93 3b 23 	sts	0x233B, r25	; 0x80233b <udd_g_ctrlreq+0xb>
     ec6:	cf c1       	rjmp	.+926    	; 0x1266 <udc_process_setup+0x514>
 *
 * \return true if success
 */
static bool udc_req_std_dev_get_configuration(void)
{
	if (udd_g_ctrlreq.req.wLength != 1) {
     ec8:	21 30       	cpi	r18, 0x01	; 1
     eca:	31 05       	cpc	r19, r1
     ecc:	09 f0       	breq	.+2      	; 0xed0 <udc_process_setup+0x17e>
     ece:	43 c1       	rjmp	.+646    	; 0x1156 <udc_process_setup+0x404>
		return false;
	}

	udd_set_setup_payload(&udc_num_configuration,1);
     ed0:	61 e0       	ldi	r22, 0x01	; 1
     ed2:	70 e0       	ldi	r23, 0x00	; 0
     ed4:	8a ee       	ldi	r24, 0xEA	; 234
     ed6:	91 e2       	ldi	r25, 0x21	; 33
     ed8:	0e 94 75 0d 	call	0x1aea	; 0x1aea <udd_set_setup_payload>
     edc:	c4 c1       	rjmp	.+904    	; 0x1266 <udc_process_setup+0x514>
			default:
				break;
			}
		}

		if (USB_REQ_RECIP_INTERFACE == Udd_setup_recipient()) {
     ede:	81 30       	cpi	r24, 0x01	; 1
     ee0:	f1 f5       	brne	.+124    	; 0xf5e <udc_process_setup+0x20c>
			// Standard Get Interface request
			switch (udd_g_ctrlreq.req.bRequest) {
     ee2:	90 91 31 23 	lds	r25, 0x2331	; 0x802331 <udd_g_ctrlreq+0x1>
     ee6:	9a 30       	cpi	r25, 0x0A	; 10
     ee8:	d1 f5       	brne	.+116    	; 0xf5e <udc_process_setup+0x20c>
static bool udc_req_std_iface_get_setting(void)
{
	uint8_t iface_num;
	udi_api_t UDC_DESC_STORAGE *udi_api;

	if (udd_g_ctrlreq.req.wLength != 1) {
     eea:	21 30       	cpi	r18, 0x01	; 1
     eec:	31 05       	cpc	r19, r1
     eee:	09 f0       	breq	.+2      	; 0xef2 <udc_process_setup+0x1a0>
     ef0:	32 c1       	rjmp	.+612    	; 0x1156 <udc_process_setup+0x404>
		return false; // Error in request
	}
	if (!udc_num_configuration) {
     ef2:	80 91 ea 21 	lds	r24, 0x21EA	; 0x8021ea <udc_num_configuration>
     ef6:	88 23       	and	r24, r24
     ef8:	09 f4       	brne	.+2      	; 0xefc <udc_process_setup+0x1aa>
     efa:	2d c1       	rjmp	.+602    	; 0x1156 <udc_process_setup+0x404>
		return false; // The device is not is configured state yet
	}

	// Check the interface number included in the request
	iface_num = udd_g_ctrlreq.req.wIndex & 0xFF;
     efc:	c0 91 34 23 	lds	r28, 0x2334	; 0x802334 <udd_g_ctrlreq+0x4>
     f00:	d0 91 35 23 	lds	r29, 0x2335	; 0x802335 <udd_g_ctrlreq+0x5>
	if (iface_num >= udc_ptr_conf->desc->bNumInterfaces) {
     f04:	00 91 e8 21 	lds	r16, 0x21E8	; 0x8021e8 <udc_ptr_conf>
     f08:	10 91 e9 21 	lds	r17, 0x21E9	; 0x8021e9 <udc_ptr_conf+0x1>
     f0c:	d8 01       	movw	r26, r16
     f0e:	ed 91       	ld	r30, X+
     f10:	fc 91       	ld	r31, X
     f12:	84 81       	ldd	r24, Z+4	; 0x04
     f14:	c8 17       	cp	r28, r24
     f16:	08 f0       	brcs	.+2      	; 0xf1a <udc_process_setup+0x1c8>
     f18:	1e c1       	rjmp	.+572    	; 0x1156 <udc_process_setup+0x404>
		return false;
	}

	// Select first alternate setting of the interface to update udc_ptr_iface
	// before call iface->getsetting()
	if (!udc_update_iface_desc(iface_num, 0)) {
     f1a:	60 e0       	ldi	r22, 0x00	; 0
     f1c:	8c 2f       	mov	r24, r28
     f1e:	0e 94 9d 05 	call	0xb3a	; 0xb3a <udc_update_iface_desc>
     f22:	88 23       	and	r24, r24
     f24:	09 f4       	brne	.+2      	; 0xf28 <udc_process_setup+0x1d6>
     f26:	17 c1       	rjmp	.+558    	; 0x1156 <udc_process_setup+0x404>
		return false;
	}
	// Get alternate setting from UDI
	udi_api = udc_ptr_conf->udi_apis[iface_num];
     f28:	ce 01       	movw	r24, r28
     f2a:	99 27       	eor	r25, r25
     f2c:	88 0f       	add	r24, r24
     f2e:	99 1f       	adc	r25, r25
     f30:	d8 01       	movw	r26, r16
     f32:	12 96       	adiw	r26, 0x02	; 2
     f34:	ed 91       	ld	r30, X+
     f36:	fc 91       	ld	r31, X
     f38:	13 97       	sbiw	r26, 0x03	; 3
     f3a:	e8 0f       	add	r30, r24
     f3c:	f9 1f       	adc	r31, r25
	udc_iface_setting = udi_api->getsetting();
     f3e:	01 90       	ld	r0, Z+
     f40:	f0 81       	ld	r31, Z
     f42:	e0 2d       	mov	r30, r0
     f44:	86 81       	ldd	r24, Z+6	; 0x06
     f46:	97 81       	ldd	r25, Z+7	; 0x07
     f48:	fc 01       	movw	r30, r24
     f4a:	19 95       	eicall
     f4c:	80 93 ec 21 	sts	0x21EC, r24	; 0x8021ec <udc_iface_setting>

	// Link value to payload pointer of request
	udd_set_setup_payload(&udc_iface_setting,1);
     f50:	61 e0       	ldi	r22, 0x01	; 1
     f52:	70 e0       	ldi	r23, 0x00	; 0
     f54:	8c ee       	ldi	r24, 0xEC	; 236
     f56:	91 e2       	ldi	r25, 0x21	; 33
     f58:	0e 94 75 0d 	call	0x1aea	; 0x1aea <udd_set_setup_payload>
     f5c:	84 c1       	rjmp	.+776    	; 0x1266 <udc_process_setup+0x514>
			default:
				break;
			}
		}
#if (0!=USB_DEVICE_MAX_EP)
		if (USB_REQ_RECIP_ENDPOINT == Udd_setup_recipient()) {
     f5e:	82 30       	cpi	r24, 0x02	; 2
     f60:	09 f0       	breq	.+2      	; 0xf64 <udc_process_setup+0x212>
     f62:	f9 c0       	rjmp	.+498    	; 0x1156 <udc_process_setup+0x404>
			// Standard Get Endpoint request
			switch (udd_g_ctrlreq.req.bRequest) {
     f64:	80 91 31 23 	lds	r24, 0x2331	; 0x802331 <udd_g_ctrlreq+0x1>
     f68:	81 11       	cpse	r24, r1
     f6a:	ee c0       	rjmp	.+476    	; 0x1148 <udc_process_setup+0x3f6>
 */
static bool udc_req_std_ep_get_status(void)
{
	static le16_t udc_ep_status;

	if (udd_g_ctrlreq.req.wLength != sizeof(udc_ep_status)) {
     f6c:	22 30       	cpi	r18, 0x02	; 2
     f6e:	31 05       	cpc	r19, r1
     f70:	09 f0       	breq	.+2      	; 0xf74 <udc_process_setup+0x222>
     f72:	f1 c0       	rjmp	.+482    	; 0x1156 <udc_process_setup+0x404>
		return false;
	}

	udc_ep_status = udd_ep_is_halted(udd_g_ctrlreq.req.
     f74:	80 91 34 23 	lds	r24, 0x2334	; 0x802334 <udd_g_ctrlreq+0x4>
     f78:	0e 94 04 0e 	call	0x1c08	; 0x1c08 <udd_ep_is_halted>
     f7c:	90 e0       	ldi	r25, 0x00	; 0
     f7e:	80 93 e4 21 	sts	0x21E4, r24	; 0x8021e4 <udc_ep_status.5706>
     f82:	90 93 e5 21 	sts	0x21E5, r25	; 0x8021e5 <udc_ep_status.5706+0x1>
			wIndex & 0xFF) ? CPU_TO_LE16(USB_EP_STATUS_HALTED) : 0;

	udd_set_setup_payload( (uint8_t *) & udc_ep_status,
     f86:	62 e0       	ldi	r22, 0x02	; 2
     f88:	70 e0       	ldi	r23, 0x00	; 0
     f8a:	84 ee       	ldi	r24, 0xE4	; 228
     f8c:	91 e2       	ldi	r25, 0x21	; 33
     f8e:	0e 94 75 0d 	call	0x1aea	; 0x1aea <udd_set_setup_payload>
     f92:	69 c1       	rjmp	.+722    	; 0x1266 <udc_process_setup+0x514>
			}
		}
#endif
	} else {
		// SET Standard Requests
		if (USB_REQ_RECIP_DEVICE == Udd_setup_recipient()) {
     f94:	8f 71       	andi	r24, 0x1F	; 31
     f96:	09 f0       	breq	.+2      	; 0xf9a <udc_process_setup+0x248>
     f98:	86 c0       	rjmp	.+268    	; 0x10a6 <udc_process_setup+0x354>
			// Standard Set Device request
			switch (udd_g_ctrlreq.req.bRequest) {
     f9a:	90 91 31 23 	lds	r25, 0x2331	; 0x802331 <udd_g_ctrlreq+0x1>
     f9e:	93 30       	cpi	r25, 0x03	; 3
     fa0:	09 f4       	brne	.+2      	; 0xfa4 <udc_process_setup+0x252>
     fa2:	d4 c0       	rjmp	.+424    	; 0x114c <udc_process_setup+0x3fa>
     fa4:	18 f4       	brcc	.+6      	; 0xfac <udc_process_setup+0x25a>
     fa6:	91 30       	cpi	r25, 0x01	; 1
     fa8:	a1 f0       	breq	.+40     	; 0xfd2 <udc_process_setup+0x280>
     faa:	7d c0       	rjmp	.+250    	; 0x10a6 <udc_process_setup+0x354>
     fac:	95 30       	cpi	r25, 0x05	; 5
     fae:	19 f0       	breq	.+6      	; 0xfb6 <udc_process_setup+0x264>
     fb0:	99 30       	cpi	r25, 0x09	; 9
     fb2:	39 f1       	breq	.+78     	; 0x1002 <udc_process_setup+0x2b0>
     fb4:	78 c0       	rjmp	.+240    	; 0x10a6 <udc_process_setup+0x354>
 *
 * \return true if success
 */
static bool udc_req_std_dev_set_address(void)
{
	if (udd_g_ctrlreq.req.wLength) {
     fb6:	80 91 36 23 	lds	r24, 0x2336	; 0x802336 <udd_g_ctrlreq+0x6>
     fba:	90 91 37 23 	lds	r25, 0x2337	; 0x802337 <udd_g_ctrlreq+0x7>
     fbe:	89 2b       	or	r24, r25
     fc0:	09 f0       	breq	.+2      	; 0xfc4 <udc_process_setup+0x272>
     fc2:	c9 c0       	rjmp	.+402    	; 0x1156 <udc_process_setup+0x404>
		return false;
	}

	// The address must be changed at the end of setup request after the handshake
	// then we use a callback to change address
	udd_g_ctrlreq.callback = udc_valid_address;
     fc4:	87 e9       	ldi	r24, 0x97	; 151
     fc6:	95 e0       	ldi	r25, 0x05	; 5
     fc8:	80 93 3c 23 	sts	0x233C, r24	; 0x80233c <udd_g_ctrlreq+0xc>
     fcc:	90 93 3d 23 	sts	0x233D, r25	; 0x80233d <udd_g_ctrlreq+0xd>
     fd0:	4a c1       	rjmp	.+660    	; 0x1266 <udc_process_setup+0x514>
 *
 * \return true if success
 */
static bool udc_req_std_dev_clear_feature(void)
{
	if (udd_g_ctrlreq.req.wLength) {
     fd2:	80 91 36 23 	lds	r24, 0x2336	; 0x802336 <udd_g_ctrlreq+0x6>
     fd6:	90 91 37 23 	lds	r25, 0x2337	; 0x802337 <udd_g_ctrlreq+0x7>
     fda:	89 2b       	or	r24, r25
     fdc:	09 f0       	breq	.+2      	; 0xfe0 <udc_process_setup+0x28e>
     fde:	bb c0       	rjmp	.+374    	; 0x1156 <udc_process_setup+0x404>
		return false;
	}

	if (udd_g_ctrlreq.req.wValue == USB_DEV_FEATURE_REMOTE_WAKEUP) {
     fe0:	80 91 32 23 	lds	r24, 0x2332	; 0x802332 <udd_g_ctrlreq+0x2>
     fe4:	90 91 33 23 	lds	r25, 0x2333	; 0x802333 <udd_g_ctrlreq+0x3>
     fe8:	01 97       	sbiw	r24, 0x01	; 1
     fea:	09 f0       	breq	.+2      	; 0xfee <udc_process_setup+0x29c>
     fec:	b4 c0       	rjmp	.+360    	; 0x1156 <udc_process_setup+0x404>
		udc_device_status &= CPU_TO_LE16(~(uint32_t)USB_DEV_STATUS_REMOTEWAKEUP);
     fee:	80 91 ee 21 	lds	r24, 0x21EE	; 0x8021ee <udc_device_status>
     ff2:	90 91 ef 21 	lds	r25, 0x21EF	; 0x8021ef <udc_device_status+0x1>
     ff6:	8d 7f       	andi	r24, 0xFD	; 253
     ff8:	80 93 ee 21 	sts	0x21EE, r24	; 0x8021ee <udc_device_status>
     ffc:	90 93 ef 21 	sts	0x21EF, r25	; 0x8021ef <udc_device_status+0x1>
    1000:	32 c1       	rjmp	.+612    	; 0x1266 <udc_process_setup+0x514>
static bool udc_req_std_dev_set_configuration(void)
{
	uint8_t iface_num;

	// Check request length
	if (udd_g_ctrlreq.req.wLength) {
    1002:	80 91 36 23 	lds	r24, 0x2336	; 0x802336 <udd_g_ctrlreq+0x6>
    1006:	90 91 37 23 	lds	r25, 0x2337	; 0x802337 <udd_g_ctrlreq+0x7>
    100a:	89 2b       	or	r24, r25
    100c:	09 f0       	breq	.+2      	; 0x1010 <udc_process_setup+0x2be>
    100e:	a3 c0       	rjmp	.+326    	; 0x1156 <udc_process_setup+0x404>
		return false;
	}
	// Authorize configuration only if the address is valid
	if (!udd_getaddress()) {
    1010:	0e 94 6a 0d 	call	0x1ad4	; 0x1ad4 <udd_getaddress>
    1014:	88 23       	and	r24, r24
    1016:	09 f4       	brne	.+2      	; 0x101a <udc_process_setup+0x2c8>
    1018:	9e c0       	rjmp	.+316    	; 0x1156 <udc_process_setup+0x404>
		}
	} else
#endif
	{
		// FS descriptor
		if ((udd_g_ctrlreq.req.wValue & 0xFF) >
    101a:	20 91 32 23 	lds	r18, 0x2332	; 0x802332 <udd_g_ctrlreq+0x2>
    101e:	30 91 33 23 	lds	r19, 0x2333	; 0x802333 <udd_g_ctrlreq+0x3>
    1022:	33 27       	eor	r19, r19
				udc_config.confdev_lsfs->bNumConfigurations) {
    1024:	e0 91 14 20 	lds	r30, 0x2014	; 0x802014 <udc_config>
    1028:	f0 91 15 20 	lds	r31, 0x2015	; 0x802015 <udc_config+0x1>
		}
	} else
#endif
	{
		// FS descriptor
		if ((udd_g_ctrlreq.req.wValue & 0xFF) >
    102c:	81 89       	ldd	r24, Z+17	; 0x11
    102e:	90 e0       	ldi	r25, 0x00	; 0
    1030:	82 17       	cp	r24, r18
    1032:	93 07       	cpc	r25, r19
    1034:	08 f4       	brcc	.+2      	; 0x1038 <udc_process_setup+0x2e6>
    1036:	8f c0       	rjmp	.+286    	; 0x1156 <udc_process_setup+0x404>
			return false;
		}
	}

	// Reset current configuration
	udc_reset();
    1038:	0e 94 51 06 	call	0xca2	; 0xca2 <udc_reset>

	// Enable new configuration
	udc_num_configuration = udd_g_ctrlreq.req.wValue & 0xFF;
    103c:	80 91 32 23 	lds	r24, 0x2332	; 0x802332 <udd_g_ctrlreq+0x2>
    1040:	90 91 33 23 	lds	r25, 0x2333	; 0x802333 <udd_g_ctrlreq+0x3>
    1044:	80 93 ea 21 	sts	0x21EA, r24	; 0x8021ea <udc_num_configuration>
	if (udc_num_configuration == 0) {
    1048:	88 23       	and	r24, r24
    104a:	09 f4       	brne	.+2      	; 0x104e <udc_process_setup+0x2fc>
    104c:	0c c1       	rjmp	.+536    	; 0x1266 <udc_process_setup+0x514>
		udc_ptr_conf = &udc_config.conf_hs[udc_num_configuration - 1];
	} else
#endif
	{
		// FS descriptor
		udc_ptr_conf = &udc_config.conf_lsfs[udc_num_configuration - 1];
    104e:	99 27       	eor	r25, r25
    1050:	81 50       	subi	r24, 0x01	; 1
    1052:	90 4c       	sbci	r25, 0xC0	; 192
    1054:	88 0f       	add	r24, r24
    1056:	99 1f       	adc	r25, r25
    1058:	88 0f       	add	r24, r24
    105a:	99 1f       	adc	r25, r25
    105c:	e0 91 16 20 	lds	r30, 0x2016	; 0x802016 <udc_config+0x2>
    1060:	f0 91 17 20 	lds	r31, 0x2017	; 0x802017 <udc_config+0x3>
    1064:	e8 0f       	add	r30, r24
    1066:	f9 1f       	adc	r31, r25
    1068:	e0 93 e8 21 	sts	0x21E8, r30	; 0x8021e8 <udc_ptr_conf>
    106c:	f0 93 e9 21 	sts	0x21E9, r31	; 0x8021e9 <udc_ptr_conf+0x1>
	}
	// Enable all interfaces of the selected configuration
	for (iface_num = 0; iface_num < udc_ptr_conf->desc->bNumInterfaces;
    1070:	01 90       	ld	r0, Z+
    1072:	f0 81       	ld	r31, Z
    1074:	e0 2d       	mov	r30, r0
    1076:	84 81       	ldd	r24, Z+4	; 0x04
    1078:	88 23       	and	r24, r24
    107a:	09 f4       	brne	.+2      	; 0x107e <udc_process_setup+0x32c>
    107c:	f4 c0       	rjmp	.+488    	; 0x1266 <udc_process_setup+0x514>
    107e:	c0 e0       	ldi	r28, 0x00	; 0
			iface_num++) {
		if (!udc_iface_enable(iface_num, 0)) {
    1080:	60 e0       	ldi	r22, 0x00	; 0
    1082:	8c 2f       	mov	r24, r28
    1084:	0e 94 1c 06 	call	0xc38	; 0xc38 <udc_iface_enable>
    1088:	88 23       	and	r24, r24
    108a:	09 f4       	brne	.+2      	; 0x108e <udc_process_setup+0x33c>
    108c:	64 c0       	rjmp	.+200    	; 0x1156 <udc_process_setup+0x404>
		// FS descriptor
		udc_ptr_conf = &udc_config.conf_lsfs[udc_num_configuration - 1];
	}
	// Enable all interfaces of the selected configuration
	for (iface_num = 0; iface_num < udc_ptr_conf->desc->bNumInterfaces;
			iface_num++) {
    108e:	cf 5f       	subi	r28, 0xFF	; 255
	{
		// FS descriptor
		udc_ptr_conf = &udc_config.conf_lsfs[udc_num_configuration - 1];
	}
	// Enable all interfaces of the selected configuration
	for (iface_num = 0; iface_num < udc_ptr_conf->desc->bNumInterfaces;
    1090:	e0 91 e8 21 	lds	r30, 0x21E8	; 0x8021e8 <udc_ptr_conf>
    1094:	f0 91 e9 21 	lds	r31, 0x21E9	; 0x8021e9 <udc_ptr_conf+0x1>
    1098:	01 90       	ld	r0, Z+
    109a:	f0 81       	ld	r31, Z
    109c:	e0 2d       	mov	r30, r0
    109e:	84 81       	ldd	r24, Z+4	; 0x04
    10a0:	c8 17       	cp	r28, r24
    10a2:	70 f3       	brcs	.-36     	; 0x1080 <udc_process_setup+0x32e>
    10a4:	e0 c0       	rjmp	.+448    	; 0x1266 <udc_process_setup+0x514>
			default:
				break;
			}
		}

		if (USB_REQ_RECIP_INTERFACE == Udd_setup_recipient()) {
    10a6:	81 30       	cpi	r24, 0x01	; 1
    10a8:	f1 f4       	brne	.+60     	; 0x10e6 <udc_process_setup+0x394>
			// Standard Set Interface request
			switch (udd_g_ctrlreq.req.bRequest) {
    10aa:	90 91 31 23 	lds	r25, 0x2331	; 0x802331 <udd_g_ctrlreq+0x1>
    10ae:	9b 30       	cpi	r25, 0x0B	; 11
    10b0:	d1 f4       	brne	.+52     	; 0x10e6 <udc_process_setup+0x394>
 */
static bool udc_req_std_iface_set_setting(void)
{
	uint8_t iface_num, setting_num;

	if (udd_g_ctrlreq.req.wLength) {
    10b2:	80 91 36 23 	lds	r24, 0x2336	; 0x802336 <udd_g_ctrlreq+0x6>
    10b6:	90 91 37 23 	lds	r25, 0x2337	; 0x802337 <udd_g_ctrlreq+0x7>
    10ba:	89 2b       	or	r24, r25
    10bc:	09 f0       	breq	.+2      	; 0x10c0 <udc_process_setup+0x36e>
    10be:	4b c0       	rjmp	.+150    	; 0x1156 <udc_process_setup+0x404>
		return false; // Error in request
	}
	if (!udc_num_configuration) {
    10c0:	80 91 ea 21 	lds	r24, 0x21EA	; 0x8021ea <udc_num_configuration>
    10c4:	88 23       	and	r24, r24
    10c6:	09 f4       	brne	.+2      	; 0x10ca <udc_process_setup+0x378>
    10c8:	46 c0       	rjmp	.+140    	; 0x1156 <udc_process_setup+0x404>
		return false; // The device is not is configured state yet
	}

	iface_num = udd_g_ctrlreq.req.wIndex & 0xFF;
    10ca:	e0 e3       	ldi	r30, 0x30	; 48
    10cc:	f3 e2       	ldi	r31, 0x23	; 35
    10ce:	c4 81       	ldd	r28, Z+4	; 0x04
	setting_num = udd_g_ctrlreq.req.wValue & 0xFF;
    10d0:	d2 81       	ldd	r29, Z+2	; 0x02

	// Disable current setting
	if (!udc_iface_disable(iface_num)) {
    10d2:	8c 2f       	mov	r24, r28
    10d4:	0e 94 d7 05 	call	0xbae	; 0xbae <udc_iface_disable>
    10d8:	88 23       	and	r24, r24
    10da:	e9 f1       	breq	.+122    	; 0x1156 <udc_process_setup+0x404>
		return false;
	}

	// Enable new setting
	return udc_iface_enable(iface_num, setting_num);
    10dc:	6d 2f       	mov	r22, r29
    10de:	8c 2f       	mov	r24, r28
    10e0:	0e 94 1c 06 	call	0xc38	; 0xc38 <udc_iface_enable>
    10e4:	36 c0       	rjmp	.+108    	; 0x1152 <udc_process_setup+0x400>
			default:
				break;
			}
		}
#if (0!=USB_DEVICE_MAX_EP)
		if (USB_REQ_RECIP_ENDPOINT == Udd_setup_recipient()) {
    10e6:	82 30       	cpi	r24, 0x02	; 2
    10e8:	b1 f5       	brne	.+108    	; 0x1156 <udc_process_setup+0x404>
			// Standard Set Endpoint request
			switch (udd_g_ctrlreq.req.bRequest) {
    10ea:	80 91 31 23 	lds	r24, 0x2331	; 0x802331 <udd_g_ctrlreq+0x1>
    10ee:	81 30       	cpi	r24, 0x01	; 1
    10f0:	19 f0       	breq	.+6      	; 0x10f8 <udc_process_setup+0x3a6>
    10f2:	83 30       	cpi	r24, 0x03	; 3
    10f4:	91 f0       	breq	.+36     	; 0x111a <udc_process_setup+0x3c8>
    10f6:	2c c0       	rjmp	.+88     	; 0x1150 <udc_process_setup+0x3fe>
 *
 * \return true if success
 */
static bool udc_req_std_ep_clear_feature(void)
{
	if (udd_g_ctrlreq.req.wLength) {
    10f8:	80 91 36 23 	lds	r24, 0x2336	; 0x802336 <udd_g_ctrlreq+0x6>
    10fc:	90 91 37 23 	lds	r25, 0x2337	; 0x802337 <udd_g_ctrlreq+0x7>
    1100:	89 2b       	or	r24, r25
    1102:	49 f5       	brne	.+82     	; 0x1156 <udc_process_setup+0x404>
		return false;
	}

	if (udd_g_ctrlreq.req.wValue == USB_EP_FEATURE_HALT) {
    1104:	80 91 32 23 	lds	r24, 0x2332	; 0x802332 <udd_g_ctrlreq+0x2>
    1108:	90 91 33 23 	lds	r25, 0x2333	; 0x802333 <udd_g_ctrlreq+0x3>
    110c:	89 2b       	or	r24, r25
    110e:	19 f5       	brne	.+70     	; 0x1156 <udc_process_setup+0x404>
		return udd_ep_clear_halt(udd_g_ctrlreq.req.wIndex & 0xFF);
    1110:	80 91 34 23 	lds	r24, 0x2334	; 0x802334 <udd_g_ctrlreq+0x4>
    1114:	0e 94 1f 0e 	call	0x1c3e	; 0x1c3e <udd_ep_clear_halt>
    1118:	1c c0       	rjmp	.+56     	; 0x1152 <udc_process_setup+0x400>
 * \return true if success
 */
#if (0!=USB_DEVICE_MAX_EP)
static bool udc_req_std_ep_set_feature(void)
{
	if (udd_g_ctrlreq.req.wLength) {
    111a:	80 91 36 23 	lds	r24, 0x2336	; 0x802336 <udd_g_ctrlreq+0x6>
    111e:	90 91 37 23 	lds	r25, 0x2337	; 0x802337 <udd_g_ctrlreq+0x7>
    1122:	89 2b       	or	r24, r25
    1124:	c1 f4       	brne	.+48     	; 0x1156 <udc_process_setup+0x404>
		return false;
	}
	if (udd_g_ctrlreq.req.wValue == USB_EP_FEATURE_HALT) {
    1126:	80 91 32 23 	lds	r24, 0x2332	; 0x802332 <udd_g_ctrlreq+0x2>
    112a:	90 91 33 23 	lds	r25, 0x2333	; 0x802333 <udd_g_ctrlreq+0x3>
    112e:	89 2b       	or	r24, r25
    1130:	91 f4       	brne	.+36     	; 0x1156 <udc_process_setup+0x404>
		udd_ep_abort(udd_g_ctrlreq.req.wIndex & 0xFF);
    1132:	c0 e3       	ldi	r28, 0x30	; 48
    1134:	d3 e2       	ldi	r29, 0x23	; 35
    1136:	8c 81       	ldd	r24, Y+4	; 0x04
    1138:	0e 94 22 0f 	call	0x1e44	; 0x1e44 <udd_ep_abort>
		return udd_ep_set_halt(udd_g_ctrlreq.req.wIndex & 0xFF);
    113c:	8c 81       	ldd	r24, Y+4	; 0x04
    113e:	0e 94 89 0f 	call	0x1f12	; 0x1f12 <udd_ep_set_halt>
    1142:	07 c0       	rjmp	.+14     	; 0x1152 <udc_process_setup+0x400>
		}
		break;

	default:
		// Unknown descriptor requested
		return false;
    1144:	80 e0       	ldi	r24, 0x00	; 0
    1146:	05 c0       	rjmp	.+10     	; 0x1152 <udc_process_setup+0x400>
				break;
			}
		}
#endif
	}
	return false;
    1148:	80 e0       	ldi	r24, 0x00	; 0
    114a:	03 c0       	rjmp	.+6      	; 0x1152 <udc_process_setup+0x400>
			case USB_REQ_SET_ADDRESS:
				return udc_req_std_dev_set_address();
			case USB_REQ_CLEAR_FEATURE:
				return udc_req_std_dev_clear_feature();
			case USB_REQ_SET_FEATURE:
				return udc_req_std_dev_set_feature();
    114c:	80 e0       	ldi	r24, 0x00	; 0
    114e:	01 c0       	rjmp	.+2      	; 0x1152 <udc_process_setup+0x400>
				break;
			}
		}
#endif
	}
	return false;
    1150:	80 e0       	ldi	r24, 0x00	; 0
		}
	}

	// If standard request then try to decode it in UDC
	if (Udd_setup_type() == USB_REQ_TYPE_STANDARD) {
		if (udc_reqstd()) {
    1152:	81 11       	cpse	r24, r1
    1154:	89 c0       	rjmp	.+274    	; 0x1268 <udc_process_setup+0x516>
			return true;
		}
	}

	// If interface request then try to decode it in UDI
	if (Udd_setup_recipient() == USB_REQ_RECIP_INTERFACE) {
    1156:	80 91 30 23 	lds	r24, 0x2330	; 0x802330 <udd_g_ctrlreq>
    115a:	8f 71       	andi	r24, 0x1F	; 31
    115c:	81 30       	cpi	r24, 0x01	; 1
    115e:	81 f5       	brne	.+96     	; 0x11c0 <udc_process_setup+0x46e>
static bool udc_req_iface(void)
{
	uint8_t iface_num;
	udi_api_t UDC_DESC_STORAGE *udi_api;

	if (0 == udc_num_configuration) {
    1160:	80 91 ea 21 	lds	r24, 0x21EA	; 0x8021ea <udc_num_configuration>
    1164:	88 23       	and	r24, r24
    1166:	61 f1       	breq	.+88     	; 0x11c0 <udc_process_setup+0x46e>
		return false; // The device is not is configured state yet
	}
	// Check interface number
	iface_num = udd_g_ctrlreq.req.wIndex & 0xFF;
    1168:	00 91 34 23 	lds	r16, 0x2334	; 0x802334 <udd_g_ctrlreq+0x4>
    116c:	10 91 35 23 	lds	r17, 0x2335	; 0x802335 <udd_g_ctrlreq+0x5>
	if (iface_num >= udc_ptr_conf->desc->bNumInterfaces) {
    1170:	c0 91 e8 21 	lds	r28, 0x21E8	; 0x8021e8 <udc_ptr_conf>
    1174:	d0 91 e9 21 	lds	r29, 0x21E9	; 0x8021e9 <udc_ptr_conf+0x1>
    1178:	e8 81       	ld	r30, Y
    117a:	f9 81       	ldd	r31, Y+1	; 0x01
    117c:	84 81       	ldd	r24, Z+4	; 0x04
    117e:	08 17       	cp	r16, r24
    1180:	f8 f4       	brcc	.+62     	; 0x11c0 <udc_process_setup+0x46e>
	}

	//* To update udc_ptr_iface with the selected interface in request
	// Select first alternate setting of interface to update udc_ptr_iface
	// before calling udi_api->getsetting()
	if (!udc_update_iface_desc(iface_num, 0)) {
    1182:	60 e0       	ldi	r22, 0x00	; 0
    1184:	80 2f       	mov	r24, r16
    1186:	0e 94 9d 05 	call	0xb3a	; 0xb3a <udc_update_iface_desc>
    118a:	88 23       	and	r24, r24
    118c:	c9 f0       	breq	.+50     	; 0x11c0 <udc_process_setup+0x46e>
		return false;
	}
	// Select the interface with the current alternate setting
	udi_api = udc_ptr_conf->udi_apis[iface_num];
    118e:	f8 01       	movw	r30, r16
    1190:	ff 27       	eor	r31, r31
    1192:	cf 01       	movw	r24, r30
    1194:	88 0f       	add	r24, r24
    1196:	99 1f       	adc	r25, r25
    1198:	ea 81       	ldd	r30, Y+2	; 0x02
    119a:	fb 81       	ldd	r31, Y+3	; 0x03
    119c:	e8 0f       	add	r30, r24
    119e:	f9 1f       	adc	r31, r25
    11a0:	c0 81       	ld	r28, Z
    11a2:	d1 81       	ldd	r29, Z+1	; 0x01
	if (!udc_update_iface_desc(iface_num, udi_api->getsetting())) {
    11a4:	ee 81       	ldd	r30, Y+6	; 0x06
    11a6:	ff 81       	ldd	r31, Y+7	; 0x07
    11a8:	19 95       	eicall
    11aa:	68 2f       	mov	r22, r24
    11ac:	80 2f       	mov	r24, r16
    11ae:	0e 94 9d 05 	call	0xb3a	; 0xb3a <udc_update_iface_desc>
    11b2:	88 23       	and	r24, r24
    11b4:	29 f0       	breq	.+10     	; 0x11c0 <udc_process_setup+0x46e>
		return false;
	}

	// Send the SETUP request to the UDI corresponding to the interface number
	return udi_api->setup();
    11b6:	ec 81       	ldd	r30, Y+4	; 0x04
    11b8:	fd 81       	ldd	r31, Y+5	; 0x05
    11ba:	19 95       	eicall
		}
	}

	// If interface request then try to decode it in UDI
	if (Udd_setup_recipient() == USB_REQ_RECIP_INTERFACE) {
		if (udc_req_iface()) {
    11bc:	81 11       	cpse	r24, r1
    11be:	54 c0       	rjmp	.+168    	; 0x1268 <udc_process_setup+0x516>
			return true;
		}
	}

	// If endpoint request then try to decode it in UDI
	if (Udd_setup_recipient() == USB_REQ_RECIP_ENDPOINT) {
    11c0:	80 91 30 23 	lds	r24, 0x2330	; 0x802330 <udd_g_ctrlreq>
    11c4:	8f 71       	andi	r24, 0x1F	; 31
    11c6:	82 30       	cpi	r24, 0x02	; 2
    11c8:	09 f0       	breq	.+2      	; 0x11cc <udc_process_setup+0x47a>
    11ca:	41 c0       	rjmp	.+130    	; 0x124e <udc_process_setup+0x4fc>
static bool udc_req_ep(void)
{
	uint8_t iface_num;
	udi_api_t UDC_DESC_STORAGE *udi_api;

	if (0 == udc_num_configuration) {
    11cc:	80 91 ea 21 	lds	r24, 0x21EA	; 0x8021ea <udc_num_configuration>
    11d0:	88 23       	and	r24, r24
    11d2:	b9 f1       	breq	.+110    	; 0x1242 <udc_process_setup+0x4f0>
		return false; // The device is not is configured state yet
	}
	// Send this request on all enabled interfaces
	iface_num = udd_g_ctrlreq.req.wIndex & 0xFF;
	for (iface_num = 0; iface_num < udc_ptr_conf->desc->bNumInterfaces;
    11d4:	a0 91 e8 21 	lds	r26, 0x21E8	; 0x8021e8 <udc_ptr_conf>
    11d8:	b0 91 e9 21 	lds	r27, 0x21E9	; 0x8021e9 <udc_ptr_conf+0x1>
    11dc:	ed 91       	ld	r30, X+
    11de:	fc 91       	ld	r31, X
    11e0:	11 97       	sbiw	r26, 0x01	; 1
    11e2:	84 81       	ldd	r24, Z+4	; 0x04
    11e4:	88 23       	and	r24, r24
    11e6:	79 f1       	breq	.+94     	; 0x1246 <udc_process_setup+0x4f4>
    11e8:	c0 e0       	ldi	r28, 0x00	; 0
			iface_num++) {
		// Select the interface with the current alternate setting
		udi_api = udc_ptr_conf->udi_apis[iface_num];
    11ea:	ec 2f       	mov	r30, r28
    11ec:	f0 e0       	ldi	r31, 0x00	; 0
    11ee:	ee 0f       	add	r30, r30
    11f0:	ff 1f       	adc	r31, r31
    11f2:	12 96       	adiw	r26, 0x02	; 2
    11f4:	8d 91       	ld	r24, X+
    11f6:	9c 91       	ld	r25, X
    11f8:	13 97       	sbiw	r26, 0x03	; 3
    11fa:	e8 0f       	add	r30, r24
    11fc:	f9 1f       	adc	r31, r25
    11fe:	00 81       	ld	r16, Z
    1200:	11 81       	ldd	r17, Z+1	; 0x01
		if (!udc_update_iface_desc(iface_num, udi_api->getsetting())) {
    1202:	d8 01       	movw	r26, r16
    1204:	16 96       	adiw	r26, 0x06	; 6
    1206:	ed 91       	ld	r30, X+
    1208:	fc 91       	ld	r31, X
    120a:	17 97       	sbiw	r26, 0x07	; 7
    120c:	19 95       	eicall
    120e:	68 2f       	mov	r22, r24
    1210:	8c 2f       	mov	r24, r28
    1212:	0e 94 9d 05 	call	0xb3a	; 0xb3a <udc_update_iface_desc>
    1216:	88 23       	and	r24, r24
    1218:	39 f1       	breq	.+78     	; 0x1268 <udc_process_setup+0x516>
			return false;
		}

		// Send the SETUP request to the UDI
		if (udi_api->setup()) {
    121a:	d8 01       	movw	r26, r16
    121c:	14 96       	adiw	r26, 0x04	; 4
    121e:	ed 91       	ld	r30, X+
    1220:	fc 91       	ld	r31, X
    1222:	15 97       	sbiw	r26, 0x05	; 5
    1224:	19 95       	eicall
    1226:	81 11       	cpse	r24, r1
    1228:	1f c0       	rjmp	.+62     	; 0x1268 <udc_process_setup+0x516>
		return false; // The device is not is configured state yet
	}
	// Send this request on all enabled interfaces
	iface_num = udd_g_ctrlreq.req.wIndex & 0xFF;
	for (iface_num = 0; iface_num < udc_ptr_conf->desc->bNumInterfaces;
			iface_num++) {
    122a:	cf 5f       	subi	r28, 0xFF	; 255
	if (0 == udc_num_configuration) {
		return false; // The device is not is configured state yet
	}
	// Send this request on all enabled interfaces
	iface_num = udd_g_ctrlreq.req.wIndex & 0xFF;
	for (iface_num = 0; iface_num < udc_ptr_conf->desc->bNumInterfaces;
    122c:	a0 91 e8 21 	lds	r26, 0x21E8	; 0x8021e8 <udc_ptr_conf>
    1230:	b0 91 e9 21 	lds	r27, 0x21E9	; 0x8021e9 <udc_ptr_conf+0x1>
    1234:	ed 91       	ld	r30, X+
    1236:	fc 91       	ld	r31, X
    1238:	11 97       	sbiw	r26, 0x01	; 1
    123a:	94 81       	ldd	r25, Z+4	; 0x04
    123c:	c9 17       	cp	r28, r25
    123e:	a8 f2       	brcs	.-86     	; 0x11ea <udc_process_setup+0x498>
    1240:	13 c0       	rjmp	.+38     	; 0x1268 <udc_process_setup+0x516>
{
	uint8_t iface_num;
	udi_api_t UDC_DESC_STORAGE *udi_api;

	if (0 == udc_num_configuration) {
		return false; // The device is not is configured state yet
    1242:	80 e0       	ldi	r24, 0x00	; 0
    1244:	11 c0       	rjmp	.+34     	; 0x1268 <udc_process_setup+0x516>
		// Send the SETUP request to the UDI
		if (udi_api->setup()) {
			return true;
		}
	}
	return false;
    1246:	80 e0       	ldi	r24, 0x00	; 0
    1248:	0f c0       	rjmp	.+30     	; 0x1268 <udc_process_setup+0x516>
	udd_g_ctrlreq.callback = NULL;
	udd_g_ctrlreq.over_under_run = NULL;

	if (Udd_setup_is_in()) {
		if (udd_g_ctrlreq.req.wLength == 0) {
			return false; // Error from USB host
    124a:	80 e0       	ldi	r24, 0x00	; 0
    124c:	0d c0       	rjmp	.+26     	; 0x1268 <udc_process_setup+0x516>
	// Here SETUP request unknown by UDC and UDIs
#ifdef USB_DEVICE_SPECIFIC_REQUEST
	// Try to decode it in specific callback
	return USB_DEVICE_SPECIFIC_REQUEST(); // Ex: Vendor request,...
#else
	return false;
    124e:	80 e0       	ldi	r24, 0x00	; 0
    1250:	0b c0       	rjmp	.+22     	; 0x1268 <udc_process_setup+0x516>
			return false; // Error from USB host
		}
	}

	// If standard request then try to decode it in UDC
	if (Udd_setup_type() == USB_REQ_TYPE_STANDARD) {
    1252:	98 2f       	mov	r25, r24
    1254:	90 76       	andi	r25, 0x60	; 96
    1256:	09 f0       	breq	.+2      	; 0x125a <udc_process_setup+0x508>
    1258:	7e cf       	rjmp	.-260    	; 0x1156 <udc_process_setup+0x404>
    125a:	9c ce       	rjmp	.-712    	; 0xf94 <udc_process_setup+0x242>
    125c:	98 2f       	mov	r25, r24
    125e:	90 76       	andi	r25, 0x60	; 96
    1260:	09 f0       	breq	.+2      	; 0x1264 <udc_process_setup+0x512>
    1262:	79 cf       	rjmp	.-270    	; 0x1156 <udc_process_setup+0x404>
    1264:	8f cd       	rjmp	.-1250   	; 0xd84 <udc_process_setup+0x32>
		if (udc_reqstd()) {
			return true;
    1266:	81 e0       	ldi	r24, 0x01	; 1
	// Try to decode it in specific callback
	return USB_DEVICE_SPECIFIC_REQUEST(); // Ex: Vendor request,...
#else
	return false;
#endif
}
    1268:	df 91       	pop	r29
    126a:	cf 91       	pop	r28
    126c:	1f 91       	pop	r17
    126e:	0f 91       	pop	r16
    1270:	08 95       	ret

00001272 <twim_interrupt_handler>:
 * \brief Common TWI master interrupt service routine.
 *
 *  Check current status and calls the appropriate handler.
 */
static void twim_interrupt_handler(void)
{
    1272:	cf 93       	push	r28
    1274:	df 93       	push	r29
	uint8_t const master_status = transfer.bus->MASTER.STATUS;
    1276:	e0 91 f0 21 	lds	r30, 0x21F0	; 0x8021f0 <transfer>
    127a:	f0 91 f1 21 	lds	r31, 0x21F1	; 0x8021f1 <transfer+0x1>
    127e:	84 81       	ldd	r24, Z+4	; 0x04

	if (master_status & TWI_MASTER_ARBLOST_bm) {
    1280:	83 ff       	sbrs	r24, 3
    1282:	08 c0       	rjmp	.+16     	; 0x1294 <twim_interrupt_handler+0x22>

		transfer.bus->MASTER.STATUS = master_status | TWI_MASTER_ARBLOST_bm;
    1284:	88 60       	ori	r24, 0x08	; 8
    1286:	84 83       	std	Z+4, r24	; 0x04
		transfer.bus->MASTER.CTRLC  = TWI_MASTER_CMD_STOP_gc;
    1288:	83 e0       	ldi	r24, 0x03	; 3
    128a:	83 83       	std	Z+3, r24	; 0x03
		transfer.status = ERR_BUSY;
    128c:	86 ef       	ldi	r24, 0xF6	; 246
    128e:	80 93 fa 21 	sts	0x21FA, r24	; 0x8021fa <transfer+0xa>
    1292:	83 c0       	rjmp	.+262    	; 0x139a <twim_interrupt_handler+0x128>
    1294:	98 2f       	mov	r25, r24
    1296:	94 71       	andi	r25, 0x14	; 20

	} else if ((master_status & TWI_MASTER_BUSERR_bm) ||
    1298:	31 f0       	breq	.+12     	; 0x12a6 <twim_interrupt_handler+0x34>
		(master_status & TWI_MASTER_RXACK_bm)) {

		transfer.bus->MASTER.CTRLC = TWI_MASTER_CMD_STOP_gc;
    129a:	83 e0       	ldi	r24, 0x03	; 3
    129c:	83 83       	std	Z+3, r24	; 0x03
		transfer.status = ERR_IO_ERROR;
    129e:	8f ef       	ldi	r24, 0xFF	; 255
    12a0:	80 93 fa 21 	sts	0x21FA, r24	; 0x8021fa <transfer+0xa>
    12a4:	7a c0       	rjmp	.+244    	; 0x139a <twim_interrupt_handler+0x128>

	} else if (master_status & TWI_MASTER_WIF_bm) {
    12a6:	86 ff       	sbrs	r24, 6
    12a8:	43 c0       	rjmp	.+134    	; 0x1330 <twim_interrupt_handler+0xbe>
 *  Handles TWI transactions (master write) and responses to (N)ACK.
 */
static inline void twim_write_handler(void)
{
	TWI_t * const         bus = transfer.bus;
	twi_package_t * const pkg = transfer.pkg;
    12aa:	c0 ef       	ldi	r28, 0xF0	; 240
    12ac:	d1 e2       	ldi	r29, 0x21	; 33
    12ae:	aa 81       	ldd	r26, Y+2	; 0x02
    12b0:	bb 81       	ldd	r27, Y+3	; 0x03

	if (transfer.addr_count < pkg->addr_length) {
    12b2:	8c 81       	ldd	r24, Y+4	; 0x04
    12b4:	9d 81       	ldd	r25, Y+5	; 0x05
    12b6:	14 96       	adiw	r26, 0x04	; 4
    12b8:	2d 91       	ld	r18, X+
    12ba:	3c 91       	ld	r19, X
    12bc:	15 97       	sbiw	r26, 0x05	; 5
    12be:	82 17       	cp	r24, r18
    12c0:	93 07       	cpc	r25, r19
    12c2:	6c f4       	brge	.+26     	; 0x12de <twim_interrupt_handler+0x6c>

		const uint8_t * const data = pkg->addr;
		bus->MASTER.DATA = data[transfer.addr_count++];
    12c4:	9c 01       	movw	r18, r24
    12c6:	2f 5f       	subi	r18, 0xFF	; 255
    12c8:	3f 4f       	sbci	r19, 0xFF	; 255
    12ca:	20 93 f4 21 	sts	0x21F4, r18	; 0x8021f4 <transfer+0x4>
    12ce:	30 93 f5 21 	sts	0x21F5, r19	; 0x8021f5 <transfer+0x5>
    12d2:	a8 0f       	add	r26, r24
    12d4:	b9 1f       	adc	r27, r25
    12d6:	11 96       	adiw	r26, 0x01	; 1
    12d8:	8c 91       	ld	r24, X
    12da:	87 83       	std	Z+7, r24	; 0x07
    12dc:	5e c0       	rjmp	.+188    	; 0x139a <twim_interrupt_handler+0x128>

	} else if (transfer.data_count < pkg->length) {
    12de:	80 91 f6 21 	lds	r24, 0x21F6	; 0x8021f6 <transfer+0x6>
    12e2:	90 91 f7 21 	lds	r25, 0x21F7	; 0x8021f7 <transfer+0x7>
    12e6:	18 96       	adiw	r26, 0x08	; 8
    12e8:	2d 91       	ld	r18, X+
    12ea:	3c 91       	ld	r19, X
    12ec:	19 97       	sbiw	r26, 0x09	; 9
    12ee:	82 17       	cp	r24, r18
    12f0:	93 07       	cpc	r25, r19
    12f2:	c8 f4       	brcc	.+50     	; 0x1326 <twim_interrupt_handler+0xb4>

		if (transfer.read) {
    12f4:	20 91 f8 21 	lds	r18, 0x21F8	; 0x8021f8 <transfer+0x8>
    12f8:	22 23       	and	r18, r18
    12fa:	21 f0       	breq	.+8      	; 0x1304 <twim_interrupt_handler+0x92>

			/* Send repeated START condition (Address|R/W=1). */

			bus->MASTER.ADDR |= 0x01;
    12fc:	86 81       	ldd	r24, Z+6	; 0x06
    12fe:	81 60       	ori	r24, 0x01	; 1
    1300:	86 83       	std	Z+6, r24	; 0x06
    1302:	4b c0       	rjmp	.+150    	; 0x139a <twim_interrupt_handler+0x128>

		} else {
			const uint8_t * const data = pkg->buffer;
    1304:	16 96       	adiw	r26, 0x06	; 6
    1306:	2d 91       	ld	r18, X+
    1308:	3c 91       	ld	r19, X
    130a:	17 97       	sbiw	r26, 0x07	; 7
			bus->MASTER.DATA = data[transfer.data_count++];
    130c:	ac 01       	movw	r20, r24
    130e:	4f 5f       	subi	r20, 0xFF	; 255
    1310:	5f 4f       	sbci	r21, 0xFF	; 255
    1312:	40 93 f6 21 	sts	0x21F6, r20	; 0x8021f6 <transfer+0x6>
    1316:	50 93 f7 21 	sts	0x21F7, r21	; 0x8021f7 <transfer+0x7>
    131a:	d9 01       	movw	r26, r18
    131c:	a8 0f       	add	r26, r24
    131e:	b9 1f       	adc	r27, r25
    1320:	8c 91       	ld	r24, X
    1322:	87 83       	std	Z+7, r24	; 0x07
    1324:	3a c0       	rjmp	.+116    	; 0x139a <twim_interrupt_handler+0x128>

	} else {

		/* Send STOP condition to complete the transaction. */

		bus->MASTER.CTRLC = TWI_MASTER_CMD_STOP_gc;
    1326:	83 e0       	ldi	r24, 0x03	; 3
    1328:	83 83       	std	Z+3, r24	; 0x03
		transfer.status = STATUS_OK;
    132a:	10 92 fa 21 	sts	0x21FA, r1	; 0x8021fa <transfer+0xa>
    132e:	35 c0       	rjmp	.+106    	; 0x139a <twim_interrupt_handler+0x128>

	} else if (master_status & TWI_MASTER_WIF_bm) {

		twim_write_handler();

	} else if (master_status & TWI_MASTER_RIF_bm) {
    1330:	88 23       	and	r24, r24
    1332:	84 f5       	brge	.+96     	; 0x1394 <twim_interrupt_handler+0x122>
 *  reading bytes from the TWI slave.
 */
static inline void twim_read_handler(void)
{
	TWI_t * const         bus = transfer.bus;
	twi_package_t * const pkg = transfer.pkg;
    1334:	a0 ef       	ldi	r26, 0xF0	; 240
    1336:	b1 e2       	ldi	r27, 0x21	; 33
    1338:	12 96       	adiw	r26, 0x02	; 2
    133a:	cd 91       	ld	r28, X+
    133c:	dc 91       	ld	r29, X
    133e:	13 97       	sbiw	r26, 0x03	; 3

	if (transfer.data_count < pkg->length) {
    1340:	16 96       	adiw	r26, 0x06	; 6
    1342:	8d 91       	ld	r24, X+
    1344:	9c 91       	ld	r25, X
    1346:	17 97       	sbiw	r26, 0x07	; 7
    1348:	28 85       	ldd	r18, Y+8	; 0x08
    134a:	39 85       	ldd	r19, Y+9	; 0x09
    134c:	82 17       	cp	r24, r18
    134e:	93 07       	cpc	r25, r19
    1350:	d8 f4       	brcc	.+54     	; 0x1388 <twim_interrupt_handler+0x116>

		uint8_t * const data = pkg->buffer;
    1352:	6e 81       	ldd	r22, Y+6	; 0x06
    1354:	7f 81       	ldd	r23, Y+7	; 0x07
		data[transfer.data_count++] = bus->MASTER.DATA;
    1356:	9c 01       	movw	r18, r24
    1358:	2f 5f       	subi	r18, 0xFF	; 255
    135a:	3f 4f       	sbci	r19, 0xFF	; 255
    135c:	20 93 f6 21 	sts	0x21F6, r18	; 0x8021f6 <transfer+0x6>
    1360:	30 93 f7 21 	sts	0x21F7, r19	; 0x8021f7 <transfer+0x7>
    1364:	47 81       	ldd	r20, Z+7	; 0x07
    1366:	db 01       	movw	r26, r22
    1368:	a8 0f       	add	r26, r24
    136a:	b9 1f       	adc	r27, r25
    136c:	4c 93       	st	X, r20

		/* If there is more to read, issue ACK and start a byte read.
		 * Otherwise, issue NACK and STOP to complete the transaction.
		 */
		if (transfer.data_count < pkg->length) {
    136e:	88 85       	ldd	r24, Y+8	; 0x08
    1370:	99 85       	ldd	r25, Y+9	; 0x09
    1372:	28 17       	cp	r18, r24
    1374:	39 07       	cpc	r19, r25
    1376:	18 f4       	brcc	.+6      	; 0x137e <twim_interrupt_handler+0x10c>

			bus->MASTER.CTRLC = TWI_MASTER_CMD_RECVTRANS_gc;
    1378:	82 e0       	ldi	r24, 0x02	; 2
    137a:	83 83       	std	Z+3, r24	; 0x03
    137c:	0e c0       	rjmp	.+28     	; 0x139a <twim_interrupt_handler+0x128>

		} else {

			bus->MASTER.CTRLC = TWI_MASTER_ACKACT_bm | TWI_MASTER_CMD_STOP_gc;
    137e:	87 e0       	ldi	r24, 0x07	; 7
    1380:	83 83       	std	Z+3, r24	; 0x03
			transfer.status = STATUS_OK;
    1382:	10 92 fa 21 	sts	0x21FA, r1	; 0x8021fa <transfer+0xa>
    1386:	09 c0       	rjmp	.+18     	; 0x139a <twim_interrupt_handler+0x128>

	} else {

		/* Issue STOP and buffer overflow condition. */

		bus->MASTER.CTRLC = TWI_MASTER_CMD_STOP_gc;
    1388:	83 e0       	ldi	r24, 0x03	; 3
    138a:	83 83       	std	Z+3, r24	; 0x03
		transfer.status = ERR_NO_MEMORY;
    138c:	89 ef       	ldi	r24, 0xF9	; 249
    138e:	80 93 fa 21 	sts	0x21FA, r24	; 0x8021fa <transfer+0xa>
    1392:	03 c0       	rjmp	.+6      	; 0x139a <twim_interrupt_handler+0x128>

		twim_read_handler();

	} else {

		transfer.status = ERR_PROTOCOL;
    1394:	8b ef       	ldi	r24, 0xFB	; 251
    1396:	80 93 fa 21 	sts	0x21FA, r24	; 0x8021fa <transfer+0xa>
	}
}
    139a:	df 91       	pop	r29
    139c:	cf 91       	pop	r28
    139e:	08 95       	ret

000013a0 <__vector_13>:
 * parameters specified in the global \c transfer structure.
 */
static void twim_interrupt_handler(void);

#ifdef TWIC
ISR(TWIC_TWIM_vect) { twim_interrupt_handler(); }
    13a0:	1f 92       	push	r1
    13a2:	0f 92       	push	r0
    13a4:	0f b6       	in	r0, 0x3f	; 63
    13a6:	0f 92       	push	r0
    13a8:	11 24       	eor	r1, r1
    13aa:	08 b6       	in	r0, 0x38	; 56
    13ac:	0f 92       	push	r0
    13ae:	18 be       	out	0x38, r1	; 56
    13b0:	09 b6       	in	r0, 0x39	; 57
    13b2:	0f 92       	push	r0
    13b4:	19 be       	out	0x39, r1	; 57
    13b6:	0b b6       	in	r0, 0x3b	; 59
    13b8:	0f 92       	push	r0
    13ba:	1b be       	out	0x3b, r1	; 59
    13bc:	2f 93       	push	r18
    13be:	3f 93       	push	r19
    13c0:	4f 93       	push	r20
    13c2:	5f 93       	push	r21
    13c4:	6f 93       	push	r22
    13c6:	7f 93       	push	r23
    13c8:	8f 93       	push	r24
    13ca:	9f 93       	push	r25
    13cc:	af 93       	push	r26
    13ce:	bf 93       	push	r27
    13d0:	ef 93       	push	r30
    13d2:	ff 93       	push	r31
    13d4:	0e 94 39 09 	call	0x1272	; 0x1272 <twim_interrupt_handler>
    13d8:	ff 91       	pop	r31
    13da:	ef 91       	pop	r30
    13dc:	bf 91       	pop	r27
    13de:	af 91       	pop	r26
    13e0:	9f 91       	pop	r25
    13e2:	8f 91       	pop	r24
    13e4:	7f 91       	pop	r23
    13e6:	6f 91       	pop	r22
    13e8:	5f 91       	pop	r21
    13ea:	4f 91       	pop	r20
    13ec:	3f 91       	pop	r19
    13ee:	2f 91       	pop	r18
    13f0:	0f 90       	pop	r0
    13f2:	0b be       	out	0x3b, r0	; 59
    13f4:	0f 90       	pop	r0
    13f6:	09 be       	out	0x39, r0	; 57
    13f8:	0f 90       	pop	r0
    13fa:	08 be       	out	0x38, r0	; 56
    13fc:	0f 90       	pop	r0
    13fe:	0f be       	out	0x3f, r0	; 63
    1400:	0f 90       	pop	r0
    1402:	1f 90       	pop	r1
    1404:	18 95       	reti

00001406 <__vector_46>:
#endif
#ifdef TWID
ISR(TWID_TWIM_vect) { twim_interrupt_handler(); }
#endif
#ifdef TWIE
ISR(TWIE_TWIM_vect) { twim_interrupt_handler(); }
    1406:	1f 92       	push	r1
    1408:	0f 92       	push	r0
    140a:	0f b6       	in	r0, 0x3f	; 63
    140c:	0f 92       	push	r0
    140e:	11 24       	eor	r1, r1
    1410:	08 b6       	in	r0, 0x38	; 56
    1412:	0f 92       	push	r0
    1414:	18 be       	out	0x38, r1	; 56
    1416:	09 b6       	in	r0, 0x39	; 57
    1418:	0f 92       	push	r0
    141a:	19 be       	out	0x39, r1	; 57
    141c:	0b b6       	in	r0, 0x3b	; 59
    141e:	0f 92       	push	r0
    1420:	1b be       	out	0x3b, r1	; 59
    1422:	2f 93       	push	r18
    1424:	3f 93       	push	r19
    1426:	4f 93       	push	r20
    1428:	5f 93       	push	r21
    142a:	6f 93       	push	r22
    142c:	7f 93       	push	r23
    142e:	8f 93       	push	r24
    1430:	9f 93       	push	r25
    1432:	af 93       	push	r26
    1434:	bf 93       	push	r27
    1436:	ef 93       	push	r30
    1438:	ff 93       	push	r31
    143a:	0e 94 39 09 	call	0x1272	; 0x1272 <twim_interrupt_handler>
    143e:	ff 91       	pop	r31
    1440:	ef 91       	pop	r30
    1442:	bf 91       	pop	r27
    1444:	af 91       	pop	r26
    1446:	9f 91       	pop	r25
    1448:	8f 91       	pop	r24
    144a:	7f 91       	pop	r23
    144c:	6f 91       	pop	r22
    144e:	5f 91       	pop	r21
    1450:	4f 91       	pop	r20
    1452:	3f 91       	pop	r19
    1454:	2f 91       	pop	r18
    1456:	0f 90       	pop	r0
    1458:	0b be       	out	0x3b, r0	; 59
    145a:	0f 90       	pop	r0
    145c:	09 be       	out	0x39, r0	; 57
    145e:	0f 90       	pop	r0
    1460:	08 be       	out	0x38, r0	; 56
    1462:	0f 90       	pop	r0
    1464:	0f be       	out	0x3f, r0	; 63
    1466:	0f 90       	pop	r0
    1468:	1f 90       	pop	r1
    146a:	18 95       	reti

0000146c <udd_sleep_mode>:
	} else {
		// endpoint not halted then call directly callback
		callback();
	}
	return true;
}
    146c:	cf 93       	push	r28
    146e:	df 93       	push	r29
    1470:	1f 92       	push	r1
    1472:	1f 92       	push	r1
    1474:	cd b7       	in	r28, 0x3d	; 61
    1476:	de b7       	in	r29, 0x3e	; 62
    1478:	81 11       	cpse	r24, r1
    147a:	26 c0       	rjmp	.+76     	; 0x14c8 <udd_sleep_mode+0x5c>
    147c:	90 91 28 23 	lds	r25, 0x2328	; 0x802328 <udd_b_idle>
    1480:	99 23       	and	r25, r25
    1482:	f9 f0       	breq	.+62     	; 0x14c2 <udd_sleep_mode+0x56>
    1484:	90 91 2b 23 	lds	r25, 0x232B	; 0x80232b <sleepmgr_locks+0x1>
    1488:	91 11       	cpse	r25, r1
    148a:	01 c0       	rjmp	.+2      	; 0x148e <udd_sleep_mode+0x22>
    148c:	ff cf       	rjmp	.-2      	; 0x148c <udd_sleep_mode+0x20>
    148e:	9f b7       	in	r25, 0x3f	; 63
    1490:	9a 83       	std	Y+2, r25	; 0x02
    1492:	f8 94       	cli
    1494:	2a 81       	ldd	r18, Y+2	; 0x02
    1496:	ea e2       	ldi	r30, 0x2A	; 42
    1498:	f3 e2       	ldi	r31, 0x23	; 35
    149a:	91 81       	ldd	r25, Z+1	; 0x01
    149c:	91 50       	subi	r25, 0x01	; 1
    149e:	91 83       	std	Z+1, r25	; 0x01
    14a0:	2f bf       	out	0x3f, r18	; 63
    14a2:	0f c0       	rjmp	.+30     	; 0x14c2 <udd_sleep_mode+0x56>
    14a4:	90 91 2b 23 	lds	r25, 0x232B	; 0x80232b <sleepmgr_locks+0x1>
    14a8:	9f 3f       	cpi	r25, 0xFF	; 255
    14aa:	09 f4       	brne	.+2      	; 0x14ae <udd_sleep_mode+0x42>
    14ac:	ff cf       	rjmp	.-2      	; 0x14ac <udd_sleep_mode+0x40>
    14ae:	9f b7       	in	r25, 0x3f	; 63
    14b0:	99 83       	std	Y+1, r25	; 0x01
    14b2:	f8 94       	cli
    14b4:	29 81       	ldd	r18, Y+1	; 0x01
    14b6:	ea e2       	ldi	r30, 0x2A	; 42
    14b8:	f3 e2       	ldi	r31, 0x23	; 35
    14ba:	91 81       	ldd	r25, Z+1	; 0x01
    14bc:	9f 5f       	subi	r25, 0xFF	; 255
    14be:	91 83       	std	Z+1, r25	; 0x01
    14c0:	2f bf       	out	0x3f, r18	; 63
    14c2:	80 93 28 23 	sts	0x2328, r24	; 0x802328 <udd_b_idle>
    14c6:	05 c0       	rjmp	.+10     	; 0x14d2 <udd_sleep_mode+0x66>
    14c8:	90 91 28 23 	lds	r25, 0x2328	; 0x802328 <udd_b_idle>
    14cc:	99 23       	and	r25, r25
    14ce:	51 f3       	breq	.-44     	; 0x14a4 <udd_sleep_mode+0x38>
    14d0:	f8 cf       	rjmp	.-16     	; 0x14c2 <udd_sleep_mode+0x56>
    14d2:	0f 90       	pop	r0
    14d4:	0f 90       	pop	r0
    14d6:	df 91       	pop	r29
    14d8:	cf 91       	pop	r28
    14da:	08 95       	ret

000014dc <udd_ctrl_init>:
    14dc:	0f 93       	push	r16
    14de:	e8 ec       	ldi	r30, 0xC8	; 200
    14e0:	f4 e0       	ldi	r31, 0x04	; 4
    14e2:	80 81       	ld	r24, Z
    14e4:	8f 7d       	andi	r24, 0xDF	; 223
    14e6:	80 83       	st	Z, r24
    14e8:	80 81       	ld	r24, Z
    14ea:	8f 7d       	andi	r24, 0xDF	; 223
    14ec:	80 83       	st	Z, r24
    14ee:	ec ef       	ldi	r30, 0xFC	; 252
    14f0:	f2 e2       	ldi	r31, 0x22	; 34
    14f2:	02 e0       	ldi	r16, 0x02	; 2
    14f4:	05 93       	las	Z, r16
    14f6:	10 92 fe 22 	sts	0x22FE, r1	; 0x8022fe <udd_sram+0x16>
    14fa:	10 92 ff 22 	sts	0x22FF, r1	; 0x8022ff <udd_sram+0x17>
    14fe:	00 e2       	ldi	r16, 0x20	; 32
    1500:	06 93       	lac	Z, r16
    1502:	00 e4       	ldi	r16, 0x40	; 64
    1504:	06 93       	lac	Z, r16
    1506:	e4 ef       	ldi	r30, 0xF4	; 244
    1508:	f2 e2       	ldi	r31, 0x22	; 34
    150a:	00 e2       	ldi	r16, 0x20	; 32
    150c:	06 93       	lac	Z, r16
    150e:	00 e4       	ldi	r16, 0x40	; 64
    1510:	06 93       	lac	Z, r16
    1512:	e0 e3       	ldi	r30, 0x30	; 48
    1514:	f3 e2       	ldi	r31, 0x23	; 35
    1516:	14 86       	std	Z+12, r1	; 0x0c
    1518:	15 86       	std	Z+13, r1	; 0x0d
    151a:	16 86       	std	Z+14, r1	; 0x0e
    151c:	17 86       	std	Z+15, r1	; 0x0f
    151e:	12 86       	std	Z+10, r1	; 0x0a
    1520:	13 86       	std	Z+11, r1	; 0x0b
    1522:	10 92 e4 22 	sts	0x22E4, r1	; 0x8022e4 <udd_ep_control_state>
    1526:	0f 91       	pop	r16
    1528:	08 95       	ret

0000152a <udd_ctrl_stall_data>:
    152a:	0f 93       	push	r16
    152c:	85 e0       	ldi	r24, 0x05	; 5
    152e:	80 93 e4 22 	sts	0x22E4, r24	; 0x8022e4 <udd_ep_control_state>
    1532:	ed ef       	ldi	r30, 0xFD	; 253
    1534:	f2 e2       	ldi	r31, 0x22	; 34
    1536:	04 e0       	ldi	r16, 0x04	; 4
    1538:	05 93       	las	Z, r16
    153a:	e5 ef       	ldi	r30, 0xF5	; 245
    153c:	f2 e2       	ldi	r31, 0x22	; 34
    153e:	04 e0       	ldi	r16, 0x04	; 4
    1540:	05 93       	las	Z, r16
    1542:	0f 91       	pop	r16
    1544:	08 95       	ret

00001546 <udd_ctrl_send_zlp_in>:
    1546:	0f 93       	push	r16
    1548:	83 e0       	ldi	r24, 0x03	; 3
    154a:	80 93 e4 22 	sts	0x22E4, r24	; 0x8022e4 <udd_ep_control_state>
    154e:	10 92 fe 22 	sts	0x22FE, r1	; 0x8022fe <udd_sram+0x16>
    1552:	10 92 ff 22 	sts	0x22FF, r1	; 0x8022ff <udd_sram+0x17>
    1556:	ec ef       	ldi	r30, 0xFC	; 252
    1558:	f2 e2       	ldi	r31, 0x22	; 34
    155a:	02 e0       	ldi	r16, 0x02	; 2
    155c:	06 93       	lac	Z, r16
    155e:	0f 91       	pop	r16
    1560:	08 95       	ret

00001562 <udd_ctrl_endofrequest>:
    1562:	e0 91 3c 23 	lds	r30, 0x233C	; 0x80233c <udd_g_ctrlreq+0xc>
    1566:	f0 91 3d 23 	lds	r31, 0x233D	; 0x80233d <udd_g_ctrlreq+0xd>
    156a:	30 97       	sbiw	r30, 0x00	; 0
    156c:	09 f0       	breq	.+2      	; 0x1570 <udd_ctrl_endofrequest+0xe>
    156e:	19 95       	eicall
    1570:	08 95       	ret

00001572 <udd_ctrl_in_sent>:
    1572:	0f 93       	push	r16
    1574:	cf 93       	push	r28
    1576:	df 93       	push	r29
    1578:	80 91 e4 22 	lds	r24, 0x22E4	; 0x8022e4 <udd_ep_control_state>
    157c:	83 30       	cpi	r24, 0x03	; 3
    157e:	29 f4       	brne	.+10     	; 0x158a <udd_ctrl_in_sent+0x18>
    1580:	0e 94 b1 0a 	call	0x1562	; 0x1562 <udd_ctrl_endofrequest>
    1584:	0e 94 6e 0a 	call	0x14dc	; 0x14dc <udd_ctrl_init>
    1588:	5e c0       	rjmp	.+188    	; 0x1646 <udd_ctrl_in_sent+0xd4>
    158a:	80 91 e0 22 	lds	r24, 0x22E0	; 0x8022e0 <udd_ctrl_payload_nb_trans>
    158e:	90 91 e1 22 	lds	r25, 0x22E1	; 0x8022e1 <udd_ctrl_payload_nb_trans+0x1>
    1592:	c0 91 3a 23 	lds	r28, 0x233A	; 0x80233a <udd_g_ctrlreq+0xa>
    1596:	d0 91 3b 23 	lds	r29, 0x233B	; 0x80233b <udd_g_ctrlreq+0xb>
    159a:	c8 1b       	sub	r28, r24
    159c:	d9 0b       	sbc	r29, r25
    159e:	71 f5       	brne	.+92     	; 0x15fc <udd_ctrl_in_sent+0x8a>
    15a0:	20 91 e2 22 	lds	r18, 0x22E2	; 0x8022e2 <udd_ctrl_prev_payload_nb_trans>
    15a4:	30 91 e3 22 	lds	r19, 0x22E3	; 0x8022e3 <udd_ctrl_prev_payload_nb_trans+0x1>
    15a8:	82 0f       	add	r24, r18
    15aa:	93 1f       	adc	r25, r19
    15ac:	80 93 e2 22 	sts	0x22E2, r24	; 0x8022e2 <udd_ctrl_prev_payload_nb_trans>
    15b0:	90 93 e3 22 	sts	0x22E3, r25	; 0x8022e3 <udd_ctrl_prev_payload_nb_trans+0x1>
    15b4:	20 91 36 23 	lds	r18, 0x2336	; 0x802336 <udd_g_ctrlreq+0x6>
    15b8:	30 91 37 23 	lds	r19, 0x2337	; 0x802337 <udd_g_ctrlreq+0x7>
    15bc:	82 17       	cp	r24, r18
    15be:	93 07       	cpc	r25, r19
    15c0:	21 f0       	breq	.+8      	; 0x15ca <udd_ctrl_in_sent+0x58>
    15c2:	80 91 fb 21 	lds	r24, 0x21FB	; 0x8021fb <b_shortpacket.5993>
    15c6:	88 23       	and	r24, r24
    15c8:	41 f0       	breq	.+16     	; 0x15da <udd_ctrl_in_sent+0x68>
    15ca:	84 e0       	ldi	r24, 0x04	; 4
    15cc:	80 93 e4 22 	sts	0x22E4, r24	; 0x8022e4 <udd_ep_control_state>
    15d0:	e4 ef       	ldi	r30, 0xF4	; 244
    15d2:	f2 e2       	ldi	r31, 0x22	; 34
    15d4:	02 e0       	ldi	r16, 0x02	; 2
    15d6:	06 93       	lac	Z, r16
    15d8:	36 c0       	rjmp	.+108    	; 0x1646 <udd_ctrl_in_sent+0xd4>
    15da:	e0 91 3e 23 	lds	r30, 0x233E	; 0x80233e <udd_g_ctrlreq+0xe>
    15de:	f0 91 3f 23 	lds	r31, 0x233F	; 0x80233f <udd_g_ctrlreq+0xf>
    15e2:	30 97       	sbiw	r30, 0x00	; 0
    15e4:	99 f0       	breq	.+38     	; 0x160c <udd_ctrl_in_sent+0x9a>
    15e6:	19 95       	eicall
    15e8:	88 23       	and	r24, r24
    15ea:	81 f0       	breq	.+32     	; 0x160c <udd_ctrl_in_sent+0x9a>
    15ec:	10 92 e0 22 	sts	0x22E0, r1	; 0x8022e0 <udd_ctrl_payload_nb_trans>
    15f0:	10 92 e1 22 	sts	0x22E1, r1	; 0x8022e1 <udd_ctrl_payload_nb_trans+0x1>
    15f4:	c0 91 3a 23 	lds	r28, 0x233A	; 0x80233a <udd_g_ctrlreq+0xa>
    15f8:	d0 91 3b 23 	lds	r29, 0x233B	; 0x80233b <udd_g_ctrlreq+0xb>
    15fc:	c0 34       	cpi	r28, 0x40	; 64
    15fe:	d1 05       	cpc	r29, r1
    1600:	28 f0       	brcs	.+10     	; 0x160c <udd_ctrl_in_sent+0x9a>
    1602:	10 92 fb 21 	sts	0x21FB, r1	; 0x8021fb <b_shortpacket.5993>
    1606:	c0 e4       	ldi	r28, 0x40	; 64
    1608:	d0 e0       	ldi	r29, 0x00	; 0
    160a:	03 c0       	rjmp	.+6      	; 0x1612 <udd_ctrl_in_sent+0xa0>
    160c:	81 e0       	ldi	r24, 0x01	; 1
    160e:	80 93 fb 21 	sts	0x21FB, r24	; 0x8021fb <b_shortpacket.5993>
    1612:	e8 ee       	ldi	r30, 0xE8	; 232
    1614:	f2 e2       	ldi	r31, 0x22	; 34
    1616:	c6 8b       	std	Z+22, r28	; 0x16
    1618:	d7 8b       	std	Z+23, r29	; 0x17
    161a:	80 91 e0 22 	lds	r24, 0x22E0	; 0x8022e0 <udd_ctrl_payload_nb_trans>
    161e:	90 91 e1 22 	lds	r25, 0x22E1	; 0x8022e1 <udd_ctrl_payload_nb_trans+0x1>
    1622:	20 91 38 23 	lds	r18, 0x2338	; 0x802338 <udd_g_ctrlreq+0x8>
    1626:	30 91 39 23 	lds	r19, 0x2339	; 0x802339 <udd_g_ctrlreq+0x9>
    162a:	28 0f       	add	r18, r24
    162c:	39 1f       	adc	r19, r25
    162e:	20 8f       	std	Z+24, r18	; 0x18
    1630:	31 8f       	std	Z+25, r19	; 0x19
    1632:	c8 0f       	add	r28, r24
    1634:	d9 1f       	adc	r29, r25
    1636:	c0 93 e0 22 	sts	0x22E0, r28	; 0x8022e0 <udd_ctrl_payload_nb_trans>
    163a:	d0 93 e1 22 	sts	0x22E1, r29	; 0x8022e1 <udd_ctrl_payload_nb_trans+0x1>
    163e:	ec ef       	ldi	r30, 0xFC	; 252
    1640:	f2 e2       	ldi	r31, 0x22	; 34
    1642:	02 e0       	ldi	r16, 0x02	; 2
    1644:	06 93       	lac	Z, r16
    1646:	df 91       	pop	r29
    1648:	cf 91       	pop	r28
    164a:	0f 91       	pop	r16
    164c:	08 95       	ret

0000164e <udd_ep_get_size>:
    164e:	fc 01       	movw	r30, r24
    1650:	81 81       	ldd	r24, Z+1	; 0x01
    1652:	e8 2f       	mov	r30, r24
    1654:	e7 70       	andi	r30, 0x07	; 7
    1656:	8e 2f       	mov	r24, r30
    1658:	90 e0       	ldi	r25, 0x00	; 0
    165a:	fc 01       	movw	r30, r24
    165c:	31 97       	sbiw	r30, 0x01	; 1
    165e:	e7 30       	cpi	r30, 0x07	; 7
    1660:	f1 05       	cpc	r31, r1
    1662:	d8 f4       	brcc	.+54     	; 0x169a <udd_ep_get_size+0x4c>
    1664:	88 27       	eor	r24, r24
    1666:	e2 50       	subi	r30, 0x02	; 2
    1668:	ff 4f       	sbci	r31, 0xFF	; 255
    166a:	8f 4f       	sbci	r24, 0xFF	; 255
    166c:	0c 94 b2 13 	jmp	0x2764	; 0x2764 <__tablejump2__>
    1670:	80 e1       	ldi	r24, 0x10	; 16
    1672:	90 e0       	ldi	r25, 0x00	; 0
    1674:	08 95       	ret
    1676:	80 e2       	ldi	r24, 0x20	; 32
    1678:	90 e0       	ldi	r25, 0x00	; 0
    167a:	08 95       	ret
    167c:	80 e4       	ldi	r24, 0x40	; 64
    167e:	90 e0       	ldi	r25, 0x00	; 0
    1680:	08 95       	ret
    1682:	80 e8       	ldi	r24, 0x80	; 128
    1684:	90 e0       	ldi	r25, 0x00	; 0
    1686:	08 95       	ret
    1688:	80 e0       	ldi	r24, 0x00	; 0
    168a:	91 e0       	ldi	r25, 0x01	; 1
    168c:	08 95       	ret
    168e:	80 e0       	ldi	r24, 0x00	; 0
    1690:	92 e0       	ldi	r25, 0x02	; 2
    1692:	08 95       	ret
    1694:	8f ef       	ldi	r24, 0xFF	; 255
    1696:	93 e0       	ldi	r25, 0x03	; 3
    1698:	08 95       	ret
    169a:	88 e0       	ldi	r24, 0x08	; 8
    169c:	90 e0       	ldi	r25, 0x00	; 0
    169e:	08 95       	ret

000016a0 <udd_ep_get_job>:
    16a0:	28 2f       	mov	r18, r24
    16a2:	2f 70       	andi	r18, 0x0F	; 15
    16a4:	30 e0       	ldi	r19, 0x00	; 0
    16a6:	22 0f       	add	r18, r18
    16a8:	33 1f       	adc	r19, r19
    16aa:	08 2e       	mov	r0, r24
    16ac:	00 0c       	add	r0, r0
    16ae:	99 0b       	sbc	r25, r25
    16b0:	88 27       	eor	r24, r24
    16b2:	99 0f       	add	r25, r25
    16b4:	88 1f       	adc	r24, r24
    16b6:	99 27       	eor	r25, r25
    16b8:	82 0f       	add	r24, r18
    16ba:	93 1f       	adc	r25, r19
    16bc:	02 97       	sbiw	r24, 0x02	; 2
    16be:	9c 01       	movw	r18, r24
    16c0:	22 0f       	add	r18, r18
    16c2:	33 1f       	adc	r19, r19
    16c4:	22 0f       	add	r18, r18
    16c6:	33 1f       	adc	r19, r19
    16c8:	22 0f       	add	r18, r18
    16ca:	33 1f       	adc	r19, r19
    16cc:	82 0f       	add	r24, r18
    16ce:	93 1f       	adc	r25, r19
    16d0:	84 58       	subi	r24, 0x84	; 132
    16d2:	9d 4d       	sbci	r25, 0xDD	; 221
    16d4:	08 95       	ret

000016d6 <udd_ctrl_interrupt_tc_setup>:
    16d6:	0f 93       	push	r16
    16d8:	cf 93       	push	r28
    16da:	80 91 cc 04 	lds	r24, 0x04CC	; 0x8004cc <__TEXT_REGION_LENGTH__+0x7004cc>
    16de:	80 ff       	sbrs	r24, 0
    16e0:	68 c0       	rjmp	.+208    	; 0x17b2 <udd_ctrl_interrupt_tc_setup+0xdc>
    16e2:	81 e0       	ldi	r24, 0x01	; 1
    16e4:	80 93 cc 04 	sts	0x04CC, r24	; 0x8004cc <__TEXT_REGION_LENGTH__+0x7004cc>
    16e8:	e4 ef       	ldi	r30, 0xF4	; 244
    16ea:	f2 e2       	ldi	r31, 0x22	; 34
    16ec:	00 e8       	ldi	r16, 0x80	; 128
    16ee:	06 93       	lac	Z, r16
    16f0:	ec ef       	ldi	r30, 0xFC	; 252
    16f2:	f2 e2       	ldi	r31, 0x22	; 34
    16f4:	00 e8       	ldi	r16, 0x80	; 128
    16f6:	06 93       	lac	Z, r16
    16f8:	80 93 ca 04 	sts	0x04CA, r24	; 0x8004ca <__TEXT_REGION_LENGTH__+0x7004ca>
    16fc:	e4 ef       	ldi	r30, 0xF4	; 244
    16fe:	f2 e2       	ldi	r31, 0x22	; 34
    1700:	00 e1       	ldi	r16, 0x10	; 16
    1702:	06 93       	lac	Z, r16
    1704:	80 91 e4 22 	lds	r24, 0x22E4	; 0x8022e4 <udd_ep_control_state>
    1708:	88 23       	and	r24, r24
    170a:	39 f0       	breq	.+14     	; 0x171a <udd_ctrl_interrupt_tc_setup+0x44>
    170c:	83 50       	subi	r24, 0x03	; 3
    170e:	82 30       	cpi	r24, 0x02	; 2
    1710:	10 f4       	brcc	.+4      	; 0x1716 <udd_ctrl_interrupt_tc_setup+0x40>
    1712:	0e 94 b1 0a 	call	0x1562	; 0x1562 <udd_ctrl_endofrequest>
    1716:	0e 94 6e 0a 	call	0x14dc	; 0x14dc <udd_ctrl_init>
    171a:	80 91 f6 22 	lds	r24, 0x22F6	; 0x8022f6 <udd_sram+0xe>
    171e:	90 91 f7 22 	lds	r25, 0x22F7	; 0x8022f7 <udd_sram+0xf>
    1722:	08 97       	sbiw	r24, 0x08	; 8
    1724:	09 f0       	breq	.+2      	; 0x1728 <udd_ctrl_interrupt_tc_setup+0x52>
    1726:	47 c0       	rjmp	.+142    	; 0x17b6 <udd_ctrl_interrupt_tc_setup+0xe0>
    1728:	88 e0       	ldi	r24, 0x08	; 8
    172a:	e0 ea       	ldi	r30, 0xA0	; 160
    172c:	f2 e2       	ldi	r31, 0x22	; 34
    172e:	a0 e3       	ldi	r26, 0x30	; 48
    1730:	b3 e2       	ldi	r27, 0x23	; 35
    1732:	01 90       	ld	r0, Z+
    1734:	0d 92       	st	X+, r0
    1736:	8a 95       	dec	r24
    1738:	e1 f7       	brne	.-8      	; 0x1732 <udd_ctrl_interrupt_tc_setup+0x5c>
    173a:	e8 ec       	ldi	r30, 0xC8	; 200
    173c:	f4 e0       	ldi	r31, 0x04	; 4
    173e:	80 81       	ld	r24, Z
    1740:	80 62       	ori	r24, 0x20	; 32
    1742:	80 83       	st	Z, r24
    1744:	80 81       	ld	r24, Z
    1746:	80 62       	ori	r24, 0x20	; 32
    1748:	80 83       	st	Z, r24
    174a:	0e 94 a9 06 	call	0xd52	; 0xd52 <udc_process_setup>
    174e:	c8 2f       	mov	r28, r24
    1750:	81 11       	cpse	r24, r1
    1752:	04 c0       	rjmp	.+8      	; 0x175c <udd_ctrl_interrupt_tc_setup+0x86>
    1754:	0e 94 95 0a 	call	0x152a	; 0x152a <udd_ctrl_stall_data>
    1758:	c1 e0       	ldi	r28, 0x01	; 1
    175a:	2e c0       	rjmp	.+92     	; 0x17b8 <udd_ctrl_interrupt_tc_setup+0xe2>
    175c:	80 91 30 23 	lds	r24, 0x2330	; 0x802330 <udd_g_ctrlreq>
    1760:	88 23       	and	r24, r24
    1762:	74 f4       	brge	.+28     	; 0x1780 <udd_ctrl_interrupt_tc_setup+0xaa>
    1764:	10 92 e2 22 	sts	0x22E2, r1	; 0x8022e2 <udd_ctrl_prev_payload_nb_trans>
    1768:	10 92 e3 22 	sts	0x22E3, r1	; 0x8022e3 <udd_ctrl_prev_payload_nb_trans+0x1>
    176c:	10 92 e0 22 	sts	0x22E0, r1	; 0x8022e0 <udd_ctrl_payload_nb_trans>
    1770:	10 92 e1 22 	sts	0x22E1, r1	; 0x8022e1 <udd_ctrl_payload_nb_trans+0x1>
    1774:	82 e0       	ldi	r24, 0x02	; 2
    1776:	80 93 e4 22 	sts	0x22E4, r24	; 0x8022e4 <udd_ep_control_state>
    177a:	0e 94 b9 0a 	call	0x1572	; 0x1572 <udd_ctrl_in_sent>
    177e:	1c c0       	rjmp	.+56     	; 0x17b8 <udd_ctrl_interrupt_tc_setup+0xe2>
    1780:	80 91 36 23 	lds	r24, 0x2336	; 0x802336 <udd_g_ctrlreq+0x6>
    1784:	90 91 37 23 	lds	r25, 0x2337	; 0x802337 <udd_g_ctrlreq+0x7>
    1788:	89 2b       	or	r24, r25
    178a:	19 f4       	brne	.+6      	; 0x1792 <udd_ctrl_interrupt_tc_setup+0xbc>
    178c:	0e 94 a3 0a 	call	0x1546	; 0x1546 <udd_ctrl_send_zlp_in>
    1790:	13 c0       	rjmp	.+38     	; 0x17b8 <udd_ctrl_interrupt_tc_setup+0xe2>
    1792:	10 92 e2 22 	sts	0x22E2, r1	; 0x8022e2 <udd_ctrl_prev_payload_nb_trans>
    1796:	10 92 e3 22 	sts	0x22E3, r1	; 0x8022e3 <udd_ctrl_prev_payload_nb_trans+0x1>
    179a:	10 92 e0 22 	sts	0x22E0, r1	; 0x8022e0 <udd_ctrl_payload_nb_trans>
    179e:	10 92 e1 22 	sts	0x22E1, r1	; 0x8022e1 <udd_ctrl_payload_nb_trans+0x1>
    17a2:	81 e0       	ldi	r24, 0x01	; 1
    17a4:	80 93 e4 22 	sts	0x22E4, r24	; 0x8022e4 <udd_ep_control_state>
    17a8:	e4 ef       	ldi	r30, 0xF4	; 244
    17aa:	f2 e2       	ldi	r31, 0x22	; 34
    17ac:	02 e0       	ldi	r16, 0x02	; 2
    17ae:	06 93       	lac	Z, r16
    17b0:	03 c0       	rjmp	.+6      	; 0x17b8 <udd_ctrl_interrupt_tc_setup+0xe2>
    17b2:	c0 e0       	ldi	r28, 0x00	; 0
    17b4:	01 c0       	rjmp	.+2      	; 0x17b8 <udd_ctrl_interrupt_tc_setup+0xe2>
    17b6:	c1 e0       	ldi	r28, 0x01	; 1
    17b8:	8c 2f       	mov	r24, r28
    17ba:	cf 91       	pop	r28
    17bc:	0f 91       	pop	r16
    17be:	08 95       	ret

000017c0 <udd_ep_trans_complet>:
    17c0:	8f 92       	push	r8
    17c2:	9f 92       	push	r9
    17c4:	af 92       	push	r10
    17c6:	bf 92       	push	r11
    17c8:	df 92       	push	r13
    17ca:	ef 92       	push	r14
    17cc:	ff 92       	push	r15
    17ce:	0f 93       	push	r16
    17d0:	1f 93       	push	r17
    17d2:	cf 93       	push	r28
    17d4:	df 93       	push	r29
    17d6:	d8 2e       	mov	r13, r24
    17d8:	0e 94 50 0b 	call	0x16a0	; 0x16a0 <udd_ep_get_job>
    17dc:	8c 01       	movw	r16, r24
    17de:	bd 2c       	mov	r11, r13
    17e0:	bb 1c       	adc	r11, r11
    17e2:	bb 24       	eor	r11, r11
    17e4:	bb 1c       	adc	r11, r11
    17e6:	cd 2d       	mov	r28, r13
    17e8:	cf 70       	andi	r28, 0x0F	; 15
    17ea:	d0 e0       	ldi	r29, 0x00	; 0
    17ec:	cc 0f       	add	r28, r28
    17ee:	dd 1f       	adc	r29, r29
    17f0:	cb 0d       	add	r28, r11
    17f2:	d1 1d       	adc	r29, r1
    17f4:	ce 01       	movw	r24, r28
    17f6:	88 0f       	add	r24, r24
    17f8:	99 1f       	adc	r25, r25
    17fa:	88 0f       	add	r24, r24
    17fc:	99 1f       	adc	r25, r25
    17fe:	88 0f       	add	r24, r24
    1800:	99 1f       	adc	r25, r25
    1802:	9c 01       	movw	r18, r24
    1804:	2c 50       	subi	r18, 0x0C	; 12
    1806:	3d 4d       	sbci	r19, 0xDD	; 221
    1808:	79 01       	movw	r14, r18
    180a:	c9 01       	movw	r24, r18
    180c:	0e 94 27 0b 	call	0x164e	; 0x164e <udd_ep_get_size>
    1810:	4c 01       	movw	r8, r24
    1812:	bb 20       	and	r11, r11
    1814:	09 f4       	brne	.+2      	; 0x1818 <udd_ep_trans_complet+0x58>
    1816:	7b c0       	rjmp	.+246    	; 0x190e <udd_ep_trans_complet+0x14e>
    1818:	fe 01       	movw	r30, r28
    181a:	ee 0f       	add	r30, r30
    181c:	ff 1f       	adc	r31, r31
    181e:	ee 0f       	add	r30, r30
    1820:	ff 1f       	adc	r31, r31
    1822:	ee 0f       	add	r30, r30
    1824:	ff 1f       	adc	r31, r31
    1826:	e8 51       	subi	r30, 0x18	; 24
    1828:	fd 4d       	sbci	r31, 0xDD	; 221
    182a:	22 89       	ldd	r18, Z+18	; 0x12
    182c:	33 89       	ldd	r19, Z+19	; 0x13
    182e:	d8 01       	movw	r26, r16
    1830:	15 96       	adiw	r26, 0x05	; 5
    1832:	8d 91       	ld	r24, X+
    1834:	9c 91       	ld	r25, X
    1836:	16 97       	sbiw	r26, 0x06	; 6
    1838:	82 0f       	add	r24, r18
    183a:	93 1f       	adc	r25, r19
    183c:	15 96       	adiw	r26, 0x05	; 5
    183e:	8d 93       	st	X+, r24
    1840:	9c 93       	st	X, r25
    1842:	16 97       	sbiw	r26, 0x06	; 6
    1844:	13 96       	adiw	r26, 0x03	; 3
    1846:	2d 91       	ld	r18, X+
    1848:	3c 91       	ld	r19, X
    184a:	14 97       	sbiw	r26, 0x04	; 4
    184c:	82 17       	cp	r24, r18
    184e:	93 07       	cpc	r25, r19
    1850:	09 f4       	brne	.+2      	; 0x1854 <udd_ep_trans_complet+0x94>
    1852:	47 c0       	rjmp	.+142    	; 0x18e2 <udd_ep_trans_complet+0x122>
    1854:	28 1b       	sub	r18, r24
    1856:	39 0b       	sbc	r19, r25
    1858:	21 15       	cp	r18, r1
    185a:	b4 e0       	ldi	r27, 0x04	; 4
    185c:	3b 07       	cpc	r19, r27
    185e:	40 f0       	brcs	.+16     	; 0x1870 <udd_ep_trans_complet+0xb0>
    1860:	2f ef       	ldi	r18, 0xFF	; 255
    1862:	33 e0       	ldi	r19, 0x03	; 3
    1864:	c9 01       	movw	r24, r18
    1866:	b4 01       	movw	r22, r8
    1868:	0e 94 7c 13 	call	0x26f8	; 0x26f8 <__udivmodhi4>
    186c:	28 1b       	sub	r18, r24
    186e:	39 0b       	sbc	r19, r25
    1870:	f8 01       	movw	r30, r16
    1872:	80 81       	ld	r24, Z
    1874:	81 ff       	sbrs	r24, 1
    1876:	0a c0       	rjmp	.+20     	; 0x188c <udd_ep_trans_complet+0xcc>
    1878:	c9 01       	movw	r24, r18
    187a:	b4 01       	movw	r22, r8
    187c:	0e 94 7c 13 	call	0x26f8	; 0x26f8 <__udivmodhi4>
    1880:	41 e0       	ldi	r20, 0x01	; 1
    1882:	89 2b       	or	r24, r25
    1884:	09 f0       	breq	.+2      	; 0x1888 <udd_ep_trans_complet+0xc8>
    1886:	40 e0       	ldi	r20, 0x00	; 0
    1888:	84 2f       	mov	r24, r20
    188a:	01 c0       	rjmp	.+2      	; 0x188e <udd_ep_trans_complet+0xce>
    188c:	80 e0       	ldi	r24, 0x00	; 0
    188e:	d8 01       	movw	r26, r16
    1890:	9c 91       	ld	r25, X
    1892:	80 fb       	bst	r24, 0
    1894:	91 f9       	bld	r25, 1
    1896:	9c 93       	st	X, r25
    1898:	fe 01       	movw	r30, r28
    189a:	ee 0f       	add	r30, r30
    189c:	ff 1f       	adc	r31, r31
    189e:	ee 0f       	add	r30, r30
    18a0:	ff 1f       	adc	r31, r31
    18a2:	ee 0f       	add	r30, r30
    18a4:	ff 1f       	adc	r31, r31
    18a6:	e8 51       	subi	r30, 0x18	; 24
    18a8:	fd 4d       	sbci	r31, 0xDD	; 221
    18aa:	12 8a       	std	Z+18, r1	; 0x12
    18ac:	13 8a       	std	Z+19, r1	; 0x13
    18ae:	26 87       	std	Z+14, r18	; 0x0e
    18b0:	37 87       	std	Z+15, r19	; 0x0f
    18b2:	11 96       	adiw	r26, 0x01	; 1
    18b4:	2d 91       	ld	r18, X+
    18b6:	3c 91       	ld	r19, X
    18b8:	12 97       	sbiw	r26, 0x02	; 2
    18ba:	15 96       	adiw	r26, 0x05	; 5
    18bc:	8d 91       	ld	r24, X+
    18be:	9c 91       	ld	r25, X
    18c0:	16 97       	sbiw	r26, 0x06	; 6
    18c2:	82 0f       	add	r24, r18
    18c4:	93 1f       	adc	r25, r19
    18c6:	cc 0f       	add	r28, r28
    18c8:	dd 1f       	adc	r29, r29
    18ca:	cc 0f       	add	r28, r28
    18cc:	dd 1f       	adc	r29, r29
    18ce:	cc 0f       	add	r28, r28
    18d0:	dd 1f       	adc	r29, r29
    18d2:	c8 50       	subi	r28, 0x08	; 8
    18d4:	dd 4d       	sbci	r29, 0xDD	; 221
    18d6:	88 83       	st	Y, r24
    18d8:	99 83       	std	Y+1, r25	; 0x01
    18da:	f7 01       	movw	r30, r14
    18dc:	02 e0       	ldi	r16, 0x02	; 2
    18de:	06 93       	lac	Z, r16
    18e0:	e8 c0       	rjmp	.+464    	; 0x1ab2 <udd_ep_trans_complet+0x2f2>
    18e2:	d8 01       	movw	r26, r16
    18e4:	8c 91       	ld	r24, X
    18e6:	81 ff       	sbrs	r24, 1
    18e8:	d1 c0       	rjmp	.+418    	; 0x1a8c <udd_ep_trans_complet+0x2cc>
    18ea:	8d 7f       	andi	r24, 0xFD	; 253
    18ec:	8c 93       	st	X, r24
    18ee:	cc 0f       	add	r28, r28
    18f0:	dd 1f       	adc	r29, r29
    18f2:	cc 0f       	add	r28, r28
    18f4:	dd 1f       	adc	r29, r29
    18f6:	cc 0f       	add	r28, r28
    18f8:	dd 1f       	adc	r29, r29
    18fa:	c8 51       	subi	r28, 0x18	; 24
    18fc:	dd 4d       	sbci	r29, 0xDD	; 221
    18fe:	1a 8a       	std	Y+18, r1	; 0x12
    1900:	1b 8a       	std	Y+19, r1	; 0x13
    1902:	1e 86       	std	Y+14, r1	; 0x0e
    1904:	1f 86       	std	Y+15, r1	; 0x0f
    1906:	f7 01       	movw	r30, r14
    1908:	02 e0       	ldi	r16, 0x02	; 2
    190a:	06 93       	lac	Z, r16
    190c:	d2 c0       	rjmp	.+420    	; 0x1ab2 <udd_ep_trans_complet+0x2f2>
    190e:	fe 01       	movw	r30, r28
    1910:	ee 0f       	add	r30, r30
    1912:	ff 1f       	adc	r31, r31
    1914:	ee 0f       	add	r30, r30
    1916:	ff 1f       	adc	r31, r31
    1918:	ee 0f       	add	r30, r30
    191a:	ff 1f       	adc	r31, r31
    191c:	e8 51       	subi	r30, 0x18	; 24
    191e:	fd 4d       	sbci	r31, 0xDD	; 221
    1920:	a6 84       	ldd	r10, Z+14	; 0x0e
    1922:	b7 84       	ldd	r11, Z+15	; 0x0f
    1924:	d8 01       	movw	r26, r16
    1926:	8c 91       	ld	r24, X
    1928:	82 ff       	sbrs	r24, 2
    192a:	1b c0       	rjmp	.+54     	; 0x1962 <udd_ep_trans_complet+0x1a2>
    192c:	11 96       	adiw	r26, 0x01	; 1
    192e:	ed 91       	ld	r30, X+
    1930:	fc 91       	ld	r31, X
    1932:	12 97       	sbiw	r26, 0x02	; 2
    1934:	15 96       	adiw	r26, 0x05	; 5
    1936:	2d 91       	ld	r18, X+
    1938:	3c 91       	ld	r19, X
    193a:	16 97       	sbiw	r26, 0x06	; 6
    193c:	13 96       	adiw	r26, 0x03	; 3
    193e:	8d 91       	ld	r24, X+
    1940:	9c 91       	ld	r25, X
    1942:	14 97       	sbiw	r26, 0x04	; 4
    1944:	b4 01       	movw	r22, r8
    1946:	0e 94 7c 13 	call	0x26f8	; 0x26f8 <__udivmodhi4>
    194a:	b0 e4       	ldi	r27, 0x40	; 64
    194c:	db 9e       	mul	r13, r27
    194e:	b0 01       	movw	r22, r0
    1950:	11 24       	eor	r1, r1
    1952:	64 54       	subi	r22, 0x44	; 68
    1954:	7e 4d       	sbci	r23, 0xDE	; 222
    1956:	ac 01       	movw	r20, r24
    1958:	cf 01       	movw	r24, r30
    195a:	82 0f       	add	r24, r18
    195c:	93 1f       	adc	r25, r19
    195e:	0e 94 bb 13 	call	0x2776	; 0x2776 <memcpy>
    1962:	f8 01       	movw	r30, r16
    1964:	25 81       	ldd	r18, Z+5	; 0x05
    1966:	36 81       	ldd	r19, Z+6	; 0x06
    1968:	2a 0d       	add	r18, r10
    196a:	3b 1d       	adc	r19, r11
    196c:	25 83       	std	Z+5, r18	; 0x05
    196e:	36 83       	std	Z+6, r19	; 0x06
    1970:	83 81       	ldd	r24, Z+3	; 0x03
    1972:	94 81       	ldd	r25, Z+4	; 0x04
    1974:	82 17       	cp	r24, r18
    1976:	93 07       	cpc	r25, r19
    1978:	68 f4       	brcc	.+26     	; 0x1994 <udd_ep_trans_complet+0x1d4>
    197a:	85 83       	std	Z+5, r24	; 0x05
    197c:	96 83       	std	Z+6, r25	; 0x06
    197e:	cc 0f       	add	r28, r28
    1980:	dd 1f       	adc	r29, r29
    1982:	cc 0f       	add	r28, r28
    1984:	dd 1f       	adc	r29, r29
    1986:	cc 0f       	add	r28, r28
    1988:	dd 1f       	adc	r29, r29
    198a:	c8 51       	subi	r28, 0x18	; 24
    198c:	dd 4d       	sbci	r29, 0xDD	; 221
    198e:	8a 89       	ldd	r24, Y+18	; 0x12
    1990:	9b 89       	ldd	r25, Y+19	; 0x13
    1992:	7c c0       	rjmp	.+248    	; 0x1a8c <udd_ep_trans_complet+0x2cc>
    1994:	fe 01       	movw	r30, r28
    1996:	ee 0f       	add	r30, r30
    1998:	ff 1f       	adc	r31, r31
    199a:	ee 0f       	add	r30, r30
    199c:	ff 1f       	adc	r31, r31
    199e:	ee 0f       	add	r30, r30
    19a0:	ff 1f       	adc	r31, r31
    19a2:	e8 51       	subi	r30, 0x18	; 24
    19a4:	fd 4d       	sbci	r31, 0xDD	; 221
    19a6:	42 89       	ldd	r20, Z+18	; 0x12
    19a8:	53 89       	ldd	r21, Z+19	; 0x13
    19aa:	4a 15       	cp	r20, r10
    19ac:	5b 05       	cpc	r21, r11
    19ae:	09 f0       	breq	.+2      	; 0x19b2 <udd_ep_trans_complet+0x1f2>
    19b0:	6d c0       	rjmp	.+218    	; 0x1a8c <udd_ep_trans_complet+0x2cc>
    19b2:	28 17       	cp	r18, r24
    19b4:	39 07       	cpc	r19, r25
    19b6:	09 f4       	brne	.+2      	; 0x19ba <udd_ep_trans_complet+0x1fa>
    19b8:	69 c0       	rjmp	.+210    	; 0x1a8c <udd_ep_trans_complet+0x2cc>
    19ba:	ac 01       	movw	r20, r24
    19bc:	42 1b       	sub	r20, r18
    19be:	53 0b       	sbc	r21, r19
    19c0:	9a 01       	movw	r18, r20
    19c2:	21 15       	cp	r18, r1
    19c4:	54 e0       	ldi	r21, 0x04	; 4
    19c6:	35 07       	cpc	r19, r21
    19c8:	58 f0       	brcs	.+22     	; 0x19e0 <udd_ep_trans_complet+0x220>
    19ca:	2f ef       	ldi	r18, 0xFF	; 255
    19cc:	33 e0       	ldi	r19, 0x03	; 3
    19ce:	c9 01       	movw	r24, r18
    19d0:	b4 01       	movw	r22, r8
    19d2:	0e 94 7c 13 	call	0x26f8	; 0x26f8 <__udivmodhi4>
    19d6:	d9 01       	movw	r26, r18
    19d8:	a8 1b       	sub	r26, r24
    19da:	b9 0b       	sbc	r27, r25
    19dc:	cd 01       	movw	r24, r26
    19de:	08 c0       	rjmp	.+16     	; 0x19f0 <udd_ep_trans_complet+0x230>
    19e0:	c9 01       	movw	r24, r18
    19e2:	b4 01       	movw	r22, r8
    19e4:	0e 94 7c 13 	call	0x26f8	; 0x26f8 <__udivmodhi4>
    19e8:	f9 01       	movw	r30, r18
    19ea:	e8 1b       	sub	r30, r24
    19ec:	f9 0b       	sbc	r31, r25
    19ee:	cf 01       	movw	r24, r30
    19f0:	fe 01       	movw	r30, r28
    19f2:	ee 0f       	add	r30, r30
    19f4:	ff 1f       	adc	r31, r31
    19f6:	ee 0f       	add	r30, r30
    19f8:	ff 1f       	adc	r31, r31
    19fa:	ee 0f       	add	r30, r30
    19fc:	ff 1f       	adc	r31, r31
    19fe:	e8 51       	subi	r30, 0x18	; 24
    1a00:	fd 4d       	sbci	r31, 0xDD	; 221
    1a02:	16 86       	std	Z+14, r1	; 0x0e
    1a04:	17 86       	std	Z+15, r1	; 0x0f
    1a06:	88 15       	cp	r24, r8
    1a08:	99 05       	cpc	r25, r9
    1a0a:	00 f5       	brcc	.+64     	; 0x1a4c <udd_ep_trans_complet+0x28c>
    1a0c:	d8 01       	movw	r26, r16
    1a0e:	8c 91       	ld	r24, X
    1a10:	84 60       	ori	r24, 0x04	; 4
    1a12:	8c 93       	st	X, r24
    1a14:	b0 e4       	ldi	r27, 0x40	; 64
    1a16:	db 9e       	mul	r13, r27
    1a18:	c0 01       	movw	r24, r0
    1a1a:	11 24       	eor	r1, r1
    1a1c:	84 54       	subi	r24, 0x44	; 68
    1a1e:	9e 4d       	sbci	r25, 0xDE	; 222
    1a20:	fe 01       	movw	r30, r28
    1a22:	ee 0f       	add	r30, r30
    1a24:	ff 1f       	adc	r31, r31
    1a26:	ee 0f       	add	r30, r30
    1a28:	ff 1f       	adc	r31, r31
    1a2a:	ee 0f       	add	r30, r30
    1a2c:	ff 1f       	adc	r31, r31
    1a2e:	e8 50       	subi	r30, 0x08	; 8
    1a30:	fd 4d       	sbci	r31, 0xDD	; 221
    1a32:	80 83       	st	Z, r24
    1a34:	91 83       	std	Z+1, r25	; 0x01
    1a36:	cc 0f       	add	r28, r28
    1a38:	dd 1f       	adc	r29, r29
    1a3a:	cc 0f       	add	r28, r28
    1a3c:	dd 1f       	adc	r29, r29
    1a3e:	cc 0f       	add	r28, r28
    1a40:	dd 1f       	adc	r29, r29
    1a42:	c8 51       	subi	r28, 0x18	; 24
    1a44:	dd 4d       	sbci	r29, 0xDD	; 221
    1a46:	8a 8a       	std	Y+18, r8	; 0x12
    1a48:	9b 8a       	std	Y+19, r9	; 0x13
    1a4a:	1c c0       	rjmp	.+56     	; 0x1a84 <udd_ep_trans_complet+0x2c4>
    1a4c:	f8 01       	movw	r30, r16
    1a4e:	41 81       	ldd	r20, Z+1	; 0x01
    1a50:	52 81       	ldd	r21, Z+2	; 0x02
    1a52:	25 81       	ldd	r18, Z+5	; 0x05
    1a54:	36 81       	ldd	r19, Z+6	; 0x06
    1a56:	24 0f       	add	r18, r20
    1a58:	35 1f       	adc	r19, r21
    1a5a:	fe 01       	movw	r30, r28
    1a5c:	ee 0f       	add	r30, r30
    1a5e:	ff 1f       	adc	r31, r31
    1a60:	ee 0f       	add	r30, r30
    1a62:	ff 1f       	adc	r31, r31
    1a64:	ee 0f       	add	r30, r30
    1a66:	ff 1f       	adc	r31, r31
    1a68:	e8 50       	subi	r30, 0x08	; 8
    1a6a:	fd 4d       	sbci	r31, 0xDD	; 221
    1a6c:	20 83       	st	Z, r18
    1a6e:	31 83       	std	Z+1, r19	; 0x01
    1a70:	cc 0f       	add	r28, r28
    1a72:	dd 1f       	adc	r29, r29
    1a74:	cc 0f       	add	r28, r28
    1a76:	dd 1f       	adc	r29, r29
    1a78:	cc 0f       	add	r28, r28
    1a7a:	dd 1f       	adc	r29, r29
    1a7c:	c8 51       	subi	r28, 0x18	; 24
    1a7e:	dd 4d       	sbci	r29, 0xDD	; 221
    1a80:	8a 8b       	std	Y+18, r24	; 0x12
    1a82:	9b 8b       	std	Y+19, r25	; 0x13
    1a84:	f7 01       	movw	r30, r14
    1a86:	02 e0       	ldi	r16, 0x02	; 2
    1a88:	06 93       	lac	Z, r16
    1a8a:	13 c0       	rjmp	.+38     	; 0x1ab2 <udd_ep_trans_complet+0x2f2>
    1a8c:	d8 01       	movw	r26, r16
    1a8e:	8c 91       	ld	r24, X
    1a90:	80 ff       	sbrs	r24, 0
    1a92:	0f c0       	rjmp	.+30     	; 0x1ab2 <udd_ep_trans_complet+0x2f2>
    1a94:	8e 7f       	andi	r24, 0xFE	; 254
    1a96:	8c 93       	st	X, r24
    1a98:	17 96       	adiw	r26, 0x07	; 7
    1a9a:	ed 91       	ld	r30, X+
    1a9c:	fc 91       	ld	r31, X
    1a9e:	18 97       	sbiw	r26, 0x08	; 8
    1aa0:	30 97       	sbiw	r30, 0x00	; 0
    1aa2:	39 f0       	breq	.+14     	; 0x1ab2 <udd_ep_trans_complet+0x2f2>
    1aa4:	15 96       	adiw	r26, 0x05	; 5
    1aa6:	6d 91       	ld	r22, X+
    1aa8:	7c 91       	ld	r23, X
    1aaa:	16 97       	sbiw	r26, 0x06	; 6
    1aac:	4d 2d       	mov	r20, r13
    1aae:	80 e0       	ldi	r24, 0x00	; 0
    1ab0:	19 95       	eicall
    1ab2:	df 91       	pop	r29
    1ab4:	cf 91       	pop	r28
    1ab6:	1f 91       	pop	r17
    1ab8:	0f 91       	pop	r16
    1aba:	ff 90       	pop	r15
    1abc:	ef 90       	pop	r14
    1abe:	df 90       	pop	r13
    1ac0:	bf 90       	pop	r11
    1ac2:	af 90       	pop	r10
    1ac4:	9f 90       	pop	r9
    1ac6:	8f 90       	pop	r8
    1ac8:	08 95       	ret

00001aca <udd_is_high_speed>:
    1aca:	80 e0       	ldi	r24, 0x00	; 0
    1acc:	08 95       	ret

00001ace <udd_set_address>:
    1ace:	80 93 c3 04 	sts	0x04C3, r24	; 0x8004c3 <__TEXT_REGION_LENGTH__+0x7004c3>
    1ad2:	08 95       	ret

00001ad4 <udd_getaddress>:
    1ad4:	80 91 c3 04 	lds	r24, 0x04C3	; 0x8004c3 <__TEXT_REGION_LENGTH__+0x7004c3>
    1ad8:	08 95       	ret

00001ada <udd_get_frame_number>:
    1ada:	80 91 24 23 	lds	r24, 0x2324	; 0x802324 <udd_sram+0x3c>
    1ade:	90 91 25 23 	lds	r25, 0x2325	; 0x802325 <udd_sram+0x3d>
    1ae2:	08 95       	ret

00001ae4 <udd_get_micro_frame_number>:
    1ae4:	80 e0       	ldi	r24, 0x00	; 0
    1ae6:	90 e0       	ldi	r25, 0x00	; 0
    1ae8:	08 95       	ret

00001aea <udd_set_setup_payload>:
    1aea:	e0 e3       	ldi	r30, 0x30	; 48
    1aec:	f3 e2       	ldi	r31, 0x23	; 35
    1aee:	80 87       	std	Z+8, r24	; 0x08
    1af0:	91 87       	std	Z+9, r25	; 0x09
    1af2:	62 87       	std	Z+10, r22	; 0x0a
    1af4:	73 87       	std	Z+11, r23	; 0x0b
    1af6:	08 95       	ret

00001af8 <udd_ep_alloc>:
    1af8:	28 2f       	mov	r18, r24
    1afa:	2f 70       	andi	r18, 0x0F	; 15
    1afc:	30 e0       	ldi	r19, 0x00	; 0
    1afe:	22 0f       	add	r18, r18
    1b00:	33 1f       	adc	r19, r19
    1b02:	08 2e       	mov	r0, r24
    1b04:	00 0c       	add	r0, r0
    1b06:	99 0b       	sbc	r25, r25
    1b08:	88 27       	eor	r24, r24
    1b0a:	99 0f       	add	r25, r25
    1b0c:	88 1f       	adc	r24, r24
    1b0e:	99 27       	eor	r25, r25
    1b10:	82 0f       	add	r24, r18
    1b12:	93 1f       	adc	r25, r19
    1b14:	fc 01       	movw	r30, r24
    1b16:	ee 0f       	add	r30, r30
    1b18:	ff 1f       	adc	r31, r31
    1b1a:	ee 0f       	add	r30, r30
    1b1c:	ff 1f       	adc	r31, r31
    1b1e:	ee 0f       	add	r30, r30
    1b20:	ff 1f       	adc	r31, r31
    1b22:	e8 51       	subi	r30, 0x18	; 24
    1b24:	fd 4d       	sbci	r31, 0xDD	; 221
    1b26:	25 85       	ldd	r18, Z+13	; 0x0d
    1b28:	20 7c       	andi	r18, 0xC0	; 192
    1b2a:	09 f0       	breq	.+2      	; 0x1b2e <udd_ep_alloc+0x36>
    1b2c:	69 c0       	rjmp	.+210    	; 0x1c00 <udd_ep_alloc+0x108>
    1b2e:	63 70       	andi	r22, 0x03	; 3
    1b30:	61 30       	cpi	r22, 0x01	; 1
    1b32:	11 f0       	breq	.+4      	; 0x1b38 <udd_ep_alloc+0x40>
    1b34:	18 f4       	brcc	.+6      	; 0x1b3c <udd_ep_alloc+0x44>
    1b36:	04 c0       	rjmp	.+8      	; 0x1b40 <udd_ep_alloc+0x48>
    1b38:	20 ec       	ldi	r18, 0xC0	; 192
    1b3a:	03 c0       	rjmp	.+6      	; 0x1b42 <udd_ep_alloc+0x4a>
    1b3c:	20 e8       	ldi	r18, 0x80	; 128
    1b3e:	01 c0       	rjmp	.+2      	; 0x1b42 <udd_ep_alloc+0x4a>
    1b40:	20 e4       	ldi	r18, 0x40	; 64
    1b42:	40 38       	cpi	r20, 0x80	; 128
    1b44:	51 05       	cpc	r21, r1
    1b46:	e9 f0       	breq	.+58     	; 0x1b82 <udd_ep_alloc+0x8a>
    1b48:	50 f4       	brcc	.+20     	; 0x1b5e <udd_ep_alloc+0x66>
    1b4a:	40 32       	cpi	r20, 0x20	; 32
    1b4c:	51 05       	cpc	r21, r1
    1b4e:	a9 f0       	breq	.+42     	; 0x1b7a <udd_ep_alloc+0x82>
    1b50:	40 34       	cpi	r20, 0x40	; 64
    1b52:	51 05       	cpc	r21, r1
    1b54:	a1 f0       	breq	.+40     	; 0x1b7e <udd_ep_alloc+0x86>
    1b56:	40 31       	cpi	r20, 0x10	; 16
    1b58:	51 05       	cpc	r21, r1
    1b5a:	d9 f4       	brne	.+54     	; 0x1b92 <udd_ep_alloc+0x9a>
    1b5c:	0c c0       	rjmp	.+24     	; 0x1b76 <udd_ep_alloc+0x7e>
    1b5e:	41 15       	cp	r20, r1
    1b60:	32 e0       	ldi	r19, 0x02	; 2
    1b62:	53 07       	cpc	r21, r19
    1b64:	91 f0       	breq	.+36     	; 0x1b8a <udd_ep_alloc+0x92>
    1b66:	4f 3f       	cpi	r20, 0xFF	; 255
    1b68:	33 e0       	ldi	r19, 0x03	; 3
    1b6a:	53 07       	cpc	r21, r19
    1b6c:	81 f0       	breq	.+32     	; 0x1b8e <udd_ep_alloc+0x96>
    1b6e:	41 15       	cp	r20, r1
    1b70:	51 40       	sbci	r21, 0x01	; 1
    1b72:	79 f4       	brne	.+30     	; 0x1b92 <udd_ep_alloc+0x9a>
    1b74:	08 c0       	rjmp	.+16     	; 0x1b86 <udd_ep_alloc+0x8e>
    1b76:	41 e0       	ldi	r20, 0x01	; 1
    1b78:	0d c0       	rjmp	.+26     	; 0x1b94 <udd_ep_alloc+0x9c>
    1b7a:	42 e0       	ldi	r20, 0x02	; 2
    1b7c:	0b c0       	rjmp	.+22     	; 0x1b94 <udd_ep_alloc+0x9c>
    1b7e:	43 e0       	ldi	r20, 0x03	; 3
    1b80:	09 c0       	rjmp	.+18     	; 0x1b94 <udd_ep_alloc+0x9c>
    1b82:	44 e0       	ldi	r20, 0x04	; 4
    1b84:	07 c0       	rjmp	.+14     	; 0x1b94 <udd_ep_alloc+0x9c>
    1b86:	45 e0       	ldi	r20, 0x05	; 5
    1b88:	05 c0       	rjmp	.+10     	; 0x1b94 <udd_ep_alloc+0x9c>
    1b8a:	46 e0       	ldi	r20, 0x06	; 6
    1b8c:	03 c0       	rjmp	.+6      	; 0x1b94 <udd_ep_alloc+0x9c>
    1b8e:	47 e0       	ldi	r20, 0x07	; 7
    1b90:	01 c0       	rjmp	.+2      	; 0x1b94 <udd_ep_alloc+0x9c>
    1b92:	40 e0       	ldi	r20, 0x00	; 0
    1b94:	fc 01       	movw	r30, r24
    1b96:	ee 0f       	add	r30, r30
    1b98:	ff 1f       	adc	r31, r31
    1b9a:	ee 0f       	add	r30, r30
    1b9c:	ff 1f       	adc	r31, r31
    1b9e:	ee 0f       	add	r30, r30
    1ba0:	ff 1f       	adc	r31, r31
    1ba2:	e8 51       	subi	r30, 0x18	; 24
    1ba4:	fd 4d       	sbci	r31, 0xDD	; 221
    1ba6:	15 86       	std	Z+13, r1	; 0x0d
    1ba8:	36 e0       	ldi	r19, 0x06	; 6
    1baa:	34 87       	std	Z+12, r19	; 0x0c
    1bac:	24 2b       	or	r18, r20
    1bae:	25 87       	std	Z+13, r18	; 0x0d
    1bb0:	fc 01       	movw	r30, r24
    1bb2:	ee 0f       	add	r30, r30
    1bb4:	ff 1f       	adc	r31, r31
    1bb6:	ee 0f       	add	r30, r30
    1bb8:	ff 1f       	adc	r31, r31
    1bba:	ee 0f       	add	r30, r30
    1bbc:	ff 1f       	adc	r31, r31
    1bbe:	e8 51       	subi	r30, 0x18	; 24
    1bc0:	fd 4d       	sbci	r31, 0xDD	; 221
    1bc2:	25 85       	ldd	r18, Z+13	; 0x0d
    1bc4:	20 7c       	andi	r18, 0xC0	; 192
    1bc6:	20 3c       	cpi	r18, 0xC0	; 192
    1bc8:	69 f4       	brne	.+26     	; 0x1be4 <udd_ep_alloc+0xec>
    1bca:	fc 01       	movw	r30, r24
    1bcc:	ee 0f       	add	r30, r30
    1bce:	ff 1f       	adc	r31, r31
    1bd0:	ee 0f       	add	r30, r30
    1bd2:	ff 1f       	adc	r31, r31
    1bd4:	ee 0f       	add	r30, r30
    1bd6:	ff 1f       	adc	r31, r31
    1bd8:	e8 51       	subi	r30, 0x18	; 24
    1bda:	fd 4d       	sbci	r31, 0xDD	; 221
    1bdc:	25 85       	ldd	r18, Z+13	; 0x0d
    1bde:	27 70       	andi	r18, 0x07	; 7
    1be0:	27 30       	cpi	r18, 0x07	; 7
    1be2:	81 f0       	breq	.+32     	; 0x1c04 <udd_ep_alloc+0x10c>
    1be4:	88 0f       	add	r24, r24
    1be6:	99 1f       	adc	r25, r25
    1be8:	88 0f       	add	r24, r24
    1bea:	99 1f       	adc	r25, r25
    1bec:	88 0f       	add	r24, r24
    1bee:	99 1f       	adc	r25, r25
    1bf0:	fc 01       	movw	r30, r24
    1bf2:	e8 51       	subi	r30, 0x18	; 24
    1bf4:	fd 4d       	sbci	r31, 0xDD	; 221
    1bf6:	85 85       	ldd	r24, Z+13	; 0x0d
    1bf8:	80 62       	ori	r24, 0x20	; 32
    1bfa:	85 87       	std	Z+13, r24	; 0x0d
    1bfc:	81 e0       	ldi	r24, 0x01	; 1
    1bfe:	08 95       	ret
    1c00:	80 e0       	ldi	r24, 0x00	; 0
    1c02:	08 95       	ret
    1c04:	81 e0       	ldi	r24, 0x01	; 1
    1c06:	08 95       	ret

00001c08 <udd_ep_is_halted>:
    1c08:	e8 2f       	mov	r30, r24
    1c0a:	ef 70       	andi	r30, 0x0F	; 15
    1c0c:	f0 e0       	ldi	r31, 0x00	; 0
    1c0e:	ee 0f       	add	r30, r30
    1c10:	ff 1f       	adc	r31, r31
    1c12:	08 2e       	mov	r0, r24
    1c14:	00 0c       	add	r0, r0
    1c16:	99 0b       	sbc	r25, r25
    1c18:	88 27       	eor	r24, r24
    1c1a:	99 0f       	add	r25, r25
    1c1c:	88 1f       	adc	r24, r24
    1c1e:	99 27       	eor	r25, r25
    1c20:	e8 0f       	add	r30, r24
    1c22:	f9 1f       	adc	r31, r25
    1c24:	ee 0f       	add	r30, r30
    1c26:	ff 1f       	adc	r31, r31
    1c28:	ee 0f       	add	r30, r30
    1c2a:	ff 1f       	adc	r31, r31
    1c2c:	ee 0f       	add	r30, r30
    1c2e:	ff 1f       	adc	r31, r31
    1c30:	e8 51       	subi	r30, 0x18	; 24
    1c32:	fd 4d       	sbci	r31, 0xDD	; 221
    1c34:	85 85       	ldd	r24, Z+13	; 0x0d
    1c36:	82 fb       	bst	r24, 2
    1c38:	88 27       	eor	r24, r24
    1c3a:	80 f9       	bld	r24, 0
    1c3c:	08 95       	ret

00001c3e <udd_ep_clear_halt>:
    1c3e:	0f 93       	push	r16
    1c40:	28 2f       	mov	r18, r24
    1c42:	2f 70       	andi	r18, 0x0F	; 15
    1c44:	30 e0       	ldi	r19, 0x00	; 0
    1c46:	a9 01       	movw	r20, r18
    1c48:	44 0f       	add	r20, r20
    1c4a:	55 1f       	adc	r21, r21
    1c4c:	28 2f       	mov	r18, r24
    1c4e:	08 2e       	mov	r0, r24
    1c50:	00 0c       	add	r0, r0
    1c52:	33 0b       	sbc	r19, r19
    1c54:	22 27       	eor	r18, r18
    1c56:	33 0f       	add	r19, r19
    1c58:	22 1f       	adc	r18, r18
    1c5a:	33 27       	eor	r19, r19
    1c5c:	24 0f       	add	r18, r20
    1c5e:	35 1f       	adc	r19, r21
    1c60:	a9 01       	movw	r20, r18
    1c62:	44 0f       	add	r20, r20
    1c64:	55 1f       	adc	r21, r21
    1c66:	44 0f       	add	r20, r20
    1c68:	55 1f       	adc	r21, r21
    1c6a:	44 0f       	add	r20, r20
    1c6c:	55 1f       	adc	r21, r21
    1c6e:	fa 01       	movw	r30, r20
    1c70:	ec 50       	subi	r30, 0x0C	; 12
    1c72:	fd 4d       	sbci	r31, 0xDD	; 221
    1c74:	01 e0       	ldi	r16, 0x01	; 1
    1c76:	06 93       	lac	Z, r16
    1c78:	fa 01       	movw	r30, r20
    1c7a:	e8 51       	subi	r30, 0x18	; 24
    1c7c:	fd 4d       	sbci	r31, 0xDD	; 221
    1c7e:	95 85       	ldd	r25, Z+13	; 0x0d
    1c80:	92 ff       	sbrs	r25, 2
    1c82:	12 c0       	rjmp	.+36     	; 0x1ca8 <udd_ep_clear_halt+0x6a>
    1c84:	fa 01       	movw	r30, r20
    1c86:	e8 51       	subi	r30, 0x18	; 24
    1c88:	fd 4d       	sbci	r31, 0xDD	; 221
    1c8a:	95 85       	ldd	r25, Z+13	; 0x0d
    1c8c:	9b 7f       	andi	r25, 0xFB	; 251
    1c8e:	95 87       	std	Z+13, r25	; 0x0d
    1c90:	0e 94 50 0b 	call	0x16a0	; 0x16a0 <udd_ep_get_job>
    1c94:	fc 01       	movw	r30, r24
    1c96:	80 81       	ld	r24, Z
    1c98:	80 ff       	sbrs	r24, 0
    1c9a:	06 c0       	rjmp	.+12     	; 0x1ca8 <udd_ep_clear_halt+0x6a>
    1c9c:	8e 7f       	andi	r24, 0xFE	; 254
    1c9e:	80 83       	st	Z, r24
    1ca0:	07 80       	ldd	r0, Z+7	; 0x07
    1ca2:	f0 85       	ldd	r31, Z+8	; 0x08
    1ca4:	e0 2d       	mov	r30, r0
    1ca6:	19 95       	eicall
    1ca8:	81 e0       	ldi	r24, 0x01	; 1
    1caa:	0f 91       	pop	r16
    1cac:	08 95       	ret

00001cae <udd_ep_run>:
    1cae:	5f 92       	push	r5
    1cb0:	6f 92       	push	r6
    1cb2:	7f 92       	push	r7
    1cb4:	8f 92       	push	r8
    1cb6:	9f 92       	push	r9
    1cb8:	af 92       	push	r10
    1cba:	bf 92       	push	r11
    1cbc:	cf 92       	push	r12
    1cbe:	df 92       	push	r13
    1cc0:	ef 92       	push	r14
    1cc2:	ff 92       	push	r15
    1cc4:	0f 93       	push	r16
    1cc6:	1f 93       	push	r17
    1cc8:	cf 93       	push	r28
    1cca:	df 93       	push	r29
    1ccc:	1f 92       	push	r1
    1cce:	cd b7       	in	r28, 0x3d	; 61
    1cd0:	de b7       	in	r29, 0x3e	; 62
    1cd2:	78 2e       	mov	r7, r24
    1cd4:	66 2e       	mov	r6, r22
    1cd6:	4a 01       	movw	r8, r20
    1cd8:	59 01       	movw	r10, r18
    1cda:	0e 94 50 0b 	call	0x16a0	; 0x16a0 <udd_ep_get_job>
    1cde:	6c 01       	movw	r12, r24
    1ce0:	57 2c       	mov	r5, r7
    1ce2:	55 1c       	adc	r5, r5
    1ce4:	55 24       	eor	r5, r5
    1ce6:	55 1c       	adc	r5, r5
    1ce8:	87 2d       	mov	r24, r7
    1cea:	8f 70       	andi	r24, 0x0F	; 15
    1cec:	e8 2e       	mov	r14, r24
    1cee:	f1 2c       	mov	r15, r1
    1cf0:	ee 0c       	add	r14, r14
    1cf2:	ff 1c       	adc	r15, r15
    1cf4:	e5 0c       	add	r14, r5
    1cf6:	f1 1c       	adc	r15, r1
    1cf8:	f7 01       	movw	r30, r14
    1cfa:	ee 0f       	add	r30, r30
    1cfc:	ff 1f       	adc	r31, r31
    1cfe:	ee 0f       	add	r30, r30
    1d00:	ff 1f       	adc	r31, r31
    1d02:	ee 0f       	add	r30, r30
    1d04:	ff 1f       	adc	r31, r31
    1d06:	e8 51       	subi	r30, 0x18	; 24
    1d08:	fd 4d       	sbci	r31, 0xDD	; 221
    1d0a:	85 85       	ldd	r24, Z+13	; 0x0d
    1d0c:	80 7c       	andi	r24, 0xC0	; 192
    1d0e:	09 f4       	brne	.+2      	; 0x1d12 <udd_ep_run+0x64>
    1d10:	84 c0       	rjmp	.+264    	; 0x1e1a <udd_ep_run+0x16c>
    1d12:	f7 01       	movw	r30, r14
    1d14:	ee 0f       	add	r30, r30
    1d16:	ff 1f       	adc	r31, r31
    1d18:	ee 0f       	add	r30, r30
    1d1a:	ff 1f       	adc	r31, r31
    1d1c:	ee 0f       	add	r30, r30
    1d1e:	ff 1f       	adc	r31, r31
    1d20:	e8 51       	subi	r30, 0x18	; 24
    1d22:	fd 4d       	sbci	r31, 0xDD	; 221
    1d24:	85 85       	ldd	r24, Z+13	; 0x0d
    1d26:	80 7c       	andi	r24, 0xC0	; 192
    1d28:	80 3c       	cpi	r24, 0xC0	; 192
    1d2a:	61 f0       	breq	.+24     	; 0x1d44 <udd_ep_run+0x96>
    1d2c:	f7 01       	movw	r30, r14
    1d2e:	ee 0f       	add	r30, r30
    1d30:	ff 1f       	adc	r31, r31
    1d32:	ee 0f       	add	r30, r30
    1d34:	ff 1f       	adc	r31, r31
    1d36:	ee 0f       	add	r30, r30
    1d38:	ff 1f       	adc	r31, r31
    1d3a:	e8 51       	subi	r30, 0x18	; 24
    1d3c:	fd 4d       	sbci	r31, 0xDD	; 221
    1d3e:	85 85       	ldd	r24, Z+13	; 0x0d
    1d40:	82 fd       	sbrc	r24, 2
    1d42:	6d c0       	rjmp	.+218    	; 0x1e1e <udd_ep_run+0x170>
    1d44:	8f b7       	in	r24, 0x3f	; 63
    1d46:	89 83       	std	Y+1, r24	; 0x01
    1d48:	f8 94       	cli
    1d4a:	89 81       	ldd	r24, Y+1	; 0x01
    1d4c:	f6 01       	movw	r30, r12
    1d4e:	90 81       	ld	r25, Z
    1d50:	90 ff       	sbrs	r25, 0
    1d52:	03 c0       	rjmp	.+6      	; 0x1d5a <udd_ep_run+0xac>
    1d54:	8f bf       	out	0x3f, r24	; 63
    1d56:	51 2c       	mov	r5, r1
    1d58:	63 c0       	rjmp	.+198    	; 0x1e20 <udd_ep_run+0x172>
    1d5a:	f6 01       	movw	r30, r12
    1d5c:	90 81       	ld	r25, Z
    1d5e:	91 60       	ori	r25, 0x01	; 1
    1d60:	90 83       	st	Z, r25
    1d62:	8f bf       	out	0x3f, r24	; 63
    1d64:	81 82       	std	Z+1, r8	; 0x01
    1d66:	92 82       	std	Z+2, r9	; 0x02
    1d68:	a3 82       	std	Z+3, r10	; 0x03
    1d6a:	b4 82       	std	Z+4, r11	; 0x04
    1d6c:	15 82       	std	Z+5, r1	; 0x05
    1d6e:	16 82       	std	Z+6, r1	; 0x06
    1d70:	07 83       	std	Z+7, r16	; 0x07
    1d72:	10 87       	std	Z+8, r17	; 0x08
    1d74:	61 10       	cpse	r6, r1
    1d76:	06 c0       	rjmp	.+12     	; 0x1d84 <udd_ep_run+0xd6>
    1d78:	91 e0       	ldi	r25, 0x01	; 1
    1d7a:	a1 14       	cp	r10, r1
    1d7c:	b1 04       	cpc	r11, r1
    1d7e:	19 f0       	breq	.+6      	; 0x1d86 <udd_ep_run+0xd8>
    1d80:	90 e0       	ldi	r25, 0x00	; 0
    1d82:	01 c0       	rjmp	.+2      	; 0x1d86 <udd_ep_run+0xd8>
    1d84:	91 e0       	ldi	r25, 0x01	; 1
    1d86:	f6 01       	movw	r30, r12
    1d88:	80 81       	ld	r24, Z
    1d8a:	90 fb       	bst	r25, 0
    1d8c:	81 f9       	bld	r24, 1
    1d8e:	8b 7f       	andi	r24, 0xFB	; 251
    1d90:	80 83       	st	Z, r24
    1d92:	55 20       	and	r5, r5
    1d94:	61 f0       	breq	.+24     	; 0x1dae <udd_ep_run+0x100>
    1d96:	f7 01       	movw	r30, r14
    1d98:	ee 0f       	add	r30, r30
    1d9a:	ff 1f       	adc	r31, r31
    1d9c:	ee 0f       	add	r30, r30
    1d9e:	ff 1f       	adc	r31, r31
    1da0:	ee 0f       	add	r30, r30
    1da2:	ff 1f       	adc	r31, r31
    1da4:	e8 51       	subi	r30, 0x18	; 24
    1da6:	fd 4d       	sbci	r31, 0xDD	; 221
    1da8:	12 8a       	std	Z+18, r1	; 0x12
    1daa:	13 8a       	std	Z+19, r1	; 0x13
    1dac:	30 c0       	rjmp	.+96     	; 0x1e0e <udd_ep_run+0x160>
    1dae:	f7 01       	movw	r30, r14
    1db0:	ee 0f       	add	r30, r30
    1db2:	ff 1f       	adc	r31, r31
    1db4:	ee 0f       	add	r30, r30
    1db6:	ff 1f       	adc	r31, r31
    1db8:	ee 0f       	add	r30, r30
    1dba:	ff 1f       	adc	r31, r31
    1dbc:	e8 51       	subi	r30, 0x18	; 24
    1dbe:	fd 4d       	sbci	r31, 0xDD	; 221
    1dc0:	85 85       	ldd	r24, Z+13	; 0x0d
    1dc2:	80 7c       	andi	r24, 0xC0	; 192
    1dc4:	80 3c       	cpi	r24, 0xC0	; 192
    1dc6:	b1 f4       	brne	.+44     	; 0x1df4 <udd_ep_run+0x146>
    1dc8:	c7 01       	movw	r24, r14
    1dca:	88 0f       	add	r24, r24
    1dcc:	99 1f       	adc	r25, r25
    1dce:	88 0f       	add	r24, r24
    1dd0:	99 1f       	adc	r25, r25
    1dd2:	88 0f       	add	r24, r24
    1dd4:	99 1f       	adc	r25, r25
    1dd6:	8c 50       	subi	r24, 0x0C	; 12
    1dd8:	9d 4d       	sbci	r25, 0xDD	; 221
    1dda:	0e 94 27 0b 	call	0x164e	; 0x164e <udd_ep_get_size>
    1dde:	bc 01       	movw	r22, r24
    1de0:	c5 01       	movw	r24, r10
    1de2:	0e 94 7c 13 	call	0x26f8	; 0x26f8 <__udivmodhi4>
    1de6:	89 2b       	or	r24, r25
    1de8:	29 f0       	breq	.+10     	; 0x1df4 <udd_ep_run+0x146>
    1dea:	f6 01       	movw	r30, r12
    1dec:	80 81       	ld	r24, Z
    1dee:	8e 7f       	andi	r24, 0xFE	; 254
    1df0:	80 83       	st	Z, r24
    1df2:	16 c0       	rjmp	.+44     	; 0x1e20 <udd_ep_run+0x172>
    1df4:	f7 01       	movw	r30, r14
    1df6:	ee 0f       	add	r30, r30
    1df8:	ff 1f       	adc	r31, r31
    1dfa:	ee 0f       	add	r30, r30
    1dfc:	ff 1f       	adc	r31, r31
    1dfe:	ee 0f       	add	r30, r30
    1e00:	ff 1f       	adc	r31, r31
    1e02:	e8 51       	subi	r30, 0x18	; 24
    1e04:	fd 4d       	sbci	r31, 0xDD	; 221
    1e06:	16 86       	std	Z+14, r1	; 0x0e
    1e08:	17 86       	std	Z+15, r1	; 0x0f
    1e0a:	12 8a       	std	Z+18, r1	; 0x12
    1e0c:	13 8a       	std	Z+19, r1	; 0x13
    1e0e:	87 2d       	mov	r24, r7
    1e10:	0e 94 e0 0b 	call	0x17c0	; 0x17c0 <udd_ep_trans_complet>
    1e14:	55 24       	eor	r5, r5
    1e16:	53 94       	inc	r5
    1e18:	03 c0       	rjmp	.+6      	; 0x1e20 <udd_ep_run+0x172>
    1e1a:	51 2c       	mov	r5, r1
    1e1c:	01 c0       	rjmp	.+2      	; 0x1e20 <udd_ep_run+0x172>
    1e1e:	51 2c       	mov	r5, r1
    1e20:	85 2d       	mov	r24, r5
    1e22:	0f 90       	pop	r0
    1e24:	df 91       	pop	r29
    1e26:	cf 91       	pop	r28
    1e28:	1f 91       	pop	r17
    1e2a:	0f 91       	pop	r16
    1e2c:	ff 90       	pop	r15
    1e2e:	ef 90       	pop	r14
    1e30:	df 90       	pop	r13
    1e32:	cf 90       	pop	r12
    1e34:	bf 90       	pop	r11
    1e36:	af 90       	pop	r10
    1e38:	9f 90       	pop	r9
    1e3a:	8f 90       	pop	r8
    1e3c:	7f 90       	pop	r7
    1e3e:	6f 90       	pop	r6
    1e40:	5f 90       	pop	r5
    1e42:	08 95       	ret

00001e44 <udd_ep_abort>:
    1e44:	ff 92       	push	r15
    1e46:	0f 93       	push	r16
    1e48:	1f 93       	push	r17
    1e4a:	cf 93       	push	r28
    1e4c:	df 93       	push	r29
    1e4e:	18 2f       	mov	r17, r24
    1e50:	f8 2e       	mov	r15, r24
    1e52:	ff 1c       	adc	r15, r15
    1e54:	ff 24       	eor	r15, r15
    1e56:	ff 1c       	adc	r15, r15
    1e58:	c8 2f       	mov	r28, r24
    1e5a:	cf 70       	andi	r28, 0x0F	; 15
    1e5c:	d0 e0       	ldi	r29, 0x00	; 0
    1e5e:	cc 0f       	add	r28, r28
    1e60:	dd 1f       	adc	r29, r29
    1e62:	cf 0d       	add	r28, r15
    1e64:	d1 1d       	adc	r29, r1
    1e66:	0e 94 50 0b 	call	0x16a0	; 0x16a0 <udd_ep_get_job>
    1e6a:	dc 01       	movw	r26, r24
    1e6c:	fe 01       	movw	r30, r28
    1e6e:	ee 0f       	add	r30, r30
    1e70:	ff 1f       	adc	r31, r31
    1e72:	ee 0f       	add	r30, r30
    1e74:	ff 1f       	adc	r31, r31
    1e76:	ee 0f       	add	r30, r30
    1e78:	ff 1f       	adc	r31, r31
    1e7a:	ec 50       	subi	r30, 0x0C	; 12
    1e7c:	fd 4d       	sbci	r31, 0xDD	; 221
    1e7e:	02 e0       	ldi	r16, 0x02	; 2
    1e80:	05 93       	las	Z, r16
    1e82:	8c 91       	ld	r24, X
    1e84:	80 ff       	sbrs	r24, 0
    1e86:	22 c0       	rjmp	.+68     	; 0x1ecc <udd_ep_abort+0x88>
    1e88:	8e 7f       	andi	r24, 0xFE	; 254
    1e8a:	8c 93       	st	X, r24
    1e8c:	17 96       	adiw	r26, 0x07	; 7
    1e8e:	ed 91       	ld	r30, X+
    1e90:	fc 91       	ld	r31, X
    1e92:	18 97       	sbiw	r26, 0x08	; 8
    1e94:	30 97       	sbiw	r30, 0x00	; 0
    1e96:	d1 f0       	breq	.+52     	; 0x1ecc <udd_ep_abort+0x88>
    1e98:	ff 20       	and	r15, r15
    1e9a:	59 f0       	breq	.+22     	; 0x1eb2 <udd_ep_abort+0x6e>
    1e9c:	cc 0f       	add	r28, r28
    1e9e:	dd 1f       	adc	r29, r29
    1ea0:	cc 0f       	add	r28, r28
    1ea2:	dd 1f       	adc	r29, r29
    1ea4:	cc 0f       	add	r28, r28
    1ea6:	dd 1f       	adc	r29, r29
    1ea8:	c8 51       	subi	r28, 0x18	; 24
    1eaa:	dd 4d       	sbci	r29, 0xDD	; 221
    1eac:	6a 89       	ldd	r22, Y+18	; 0x12
    1eae:	7b 89       	ldd	r23, Y+19	; 0x13
    1eb0:	0a c0       	rjmp	.+20     	; 0x1ec6 <udd_ep_abort+0x82>
    1eb2:	cc 0f       	add	r28, r28
    1eb4:	dd 1f       	adc	r29, r29
    1eb6:	cc 0f       	add	r28, r28
    1eb8:	dd 1f       	adc	r29, r29
    1eba:	cc 0f       	add	r28, r28
    1ebc:	dd 1f       	adc	r29, r29
    1ebe:	c8 51       	subi	r28, 0x18	; 24
    1ec0:	dd 4d       	sbci	r29, 0xDD	; 221
    1ec2:	6e 85       	ldd	r22, Y+14	; 0x0e
    1ec4:	7f 85       	ldd	r23, Y+15	; 0x0f
    1ec6:	41 2f       	mov	r20, r17
    1ec8:	81 e0       	ldi	r24, 0x01	; 1
    1eca:	19 95       	eicall
    1ecc:	df 91       	pop	r29
    1ece:	cf 91       	pop	r28
    1ed0:	1f 91       	pop	r17
    1ed2:	0f 91       	pop	r16
    1ed4:	ff 90       	pop	r15
    1ed6:	08 95       	ret

00001ed8 <udd_ep_free>:
    1ed8:	cf 93       	push	r28
    1eda:	c8 2f       	mov	r28, r24
    1edc:	0e 94 22 0f 	call	0x1e44	; 0x1e44 <udd_ep_abort>
    1ee0:	ec 2f       	mov	r30, r28
    1ee2:	ef 70       	andi	r30, 0x0F	; 15
    1ee4:	f0 e0       	ldi	r31, 0x00	; 0
    1ee6:	ee 0f       	add	r30, r30
    1ee8:	ff 1f       	adc	r31, r31
    1eea:	8c 2f       	mov	r24, r28
    1eec:	cc 0f       	add	r28, r28
    1eee:	99 0b       	sbc	r25, r25
    1ef0:	88 27       	eor	r24, r24
    1ef2:	99 0f       	add	r25, r25
    1ef4:	88 1f       	adc	r24, r24
    1ef6:	99 27       	eor	r25, r25
    1ef8:	e8 0f       	add	r30, r24
    1efa:	f9 1f       	adc	r31, r25
    1efc:	ee 0f       	add	r30, r30
    1efe:	ff 1f       	adc	r31, r31
    1f00:	ee 0f       	add	r30, r30
    1f02:	ff 1f       	adc	r31, r31
    1f04:	ee 0f       	add	r30, r30
    1f06:	ff 1f       	adc	r31, r31
    1f08:	e8 51       	subi	r30, 0x18	; 24
    1f0a:	fd 4d       	sbci	r31, 0xDD	; 221
    1f0c:	15 86       	std	Z+13, r1	; 0x0d
    1f0e:	cf 91       	pop	r28
    1f10:	08 95       	ret

00001f12 <udd_ep_set_halt>:
    1f12:	e8 2f       	mov	r30, r24
    1f14:	ef 70       	andi	r30, 0x0F	; 15
    1f16:	f0 e0       	ldi	r31, 0x00	; 0
    1f18:	ee 0f       	add	r30, r30
    1f1a:	ff 1f       	adc	r31, r31
    1f1c:	28 2f       	mov	r18, r24
    1f1e:	08 2e       	mov	r0, r24
    1f20:	00 0c       	add	r0, r0
    1f22:	33 0b       	sbc	r19, r19
    1f24:	22 27       	eor	r18, r18
    1f26:	33 0f       	add	r19, r19
    1f28:	22 1f       	adc	r18, r18
    1f2a:	33 27       	eor	r19, r19
    1f2c:	e2 0f       	add	r30, r18
    1f2e:	f3 1f       	adc	r31, r19
    1f30:	ee 0f       	add	r30, r30
    1f32:	ff 1f       	adc	r31, r31
    1f34:	ee 0f       	add	r30, r30
    1f36:	ff 1f       	adc	r31, r31
    1f38:	ee 0f       	add	r30, r30
    1f3a:	ff 1f       	adc	r31, r31
    1f3c:	e8 51       	subi	r30, 0x18	; 24
    1f3e:	fd 4d       	sbci	r31, 0xDD	; 221
    1f40:	95 85       	ldd	r25, Z+13	; 0x0d
    1f42:	94 60       	ori	r25, 0x04	; 4
    1f44:	95 87       	std	Z+13, r25	; 0x0d
    1f46:	0e 94 22 0f 	call	0x1e44	; 0x1e44 <udd_ep_abort>
    1f4a:	81 e0       	ldi	r24, 0x01	; 1
    1f4c:	08 95       	ret

00001f4e <__vector_125>:
 * USB bus event interrupt includes :
 * - USB line events SOF, reset, suspend, resume, wakeup
 * - endpoint control errors underflow, overflow, stall
 */
ISR(USB_BUSEVENT_vect)
{
    1f4e:	1f 92       	push	r1
    1f50:	0f 92       	push	r0
    1f52:	0f b6       	in	r0, 0x3f	; 63
    1f54:	0f 92       	push	r0
    1f56:	11 24       	eor	r1, r1
    1f58:	08 b6       	in	r0, 0x38	; 56
    1f5a:	0f 92       	push	r0
    1f5c:	18 be       	out	0x38, r1	; 56
    1f5e:	09 b6       	in	r0, 0x39	; 57
    1f60:	0f 92       	push	r0
    1f62:	19 be       	out	0x39, r1	; 57
    1f64:	0b b6       	in	r0, 0x3b	; 59
    1f66:	0f 92       	push	r0
    1f68:	1b be       	out	0x3b, r1	; 59
    1f6a:	0f 93       	push	r16
    1f6c:	2f 93       	push	r18
    1f6e:	3f 93       	push	r19
    1f70:	4f 93       	push	r20
    1f72:	5f 93       	push	r21
    1f74:	6f 93       	push	r22
    1f76:	7f 93       	push	r23
    1f78:	8f 93       	push	r24
    1f7a:	9f 93       	push	r25
    1f7c:	af 93       	push	r26
    1f7e:	bf 93       	push	r27
    1f80:	ef 93       	push	r30
    1f82:	ff 93       	push	r31
	if (udd_is_start_of_frame_event()) {
    1f84:	80 91 cb 04 	lds	r24, 0x04CB	; 0x8004cb <__TEXT_REGION_LENGTH__+0x7004cb>
    1f88:	88 23       	and	r24, r24
    1f8a:	44 f4       	brge	.+16     	; 0x1f9c <__vector_125+0x4e>
		udd_ack_start_of_frame_event();
    1f8c:	80 e8       	ldi	r24, 0x80	; 128
    1f8e:	80 93 ca 04 	sts	0x04CA, r24	; 0x8004ca <__TEXT_REGION_LENGTH__+0x7004ca>
		udc_sof_notify();
    1f92:	0e 94 79 06 	call	0xcf2	; 0xcf2 <udc_sof_notify>
#ifdef UDC_SOF_EVENT
		UDC_SOF_EVENT();
    1f96:	0e 94 8a 11 	call	0x2314	; 0x2314 <main_sof_action>
#endif
		goto udd_interrupt_bus_event_end;
    1f9a:	8e c0       	rjmp	.+284    	; 0x20b8 <__vector_125+0x16a>
}

static bool udd_ctrl_interrupt_error(void)
{
	// Underflow only managed for control endpoint
	if (udd_is_underflow_event()) {
    1f9c:	80 91 cb 04 	lds	r24, 0x04CB	; 0x8004cb <__TEXT_REGION_LENGTH__+0x7004cb>
    1fa0:	82 ff       	sbrs	r24, 2
    1fa2:	22 c0       	rjmp	.+68     	; 0x1fe8 <__vector_125+0x9a>
		udd_ack_underflow_event();
    1fa4:	84 e0       	ldi	r24, 0x04	; 4
    1fa6:	80 93 ca 04 	sts	0x04CA, r24	; 0x8004ca <__TEXT_REGION_LENGTH__+0x7004ca>
		if (udd_control_in_underflow()) {
    1faa:	80 91 fc 22 	lds	r24, 0x22FC	; 0x8022fc <udd_sram+0x14>
    1fae:	86 ff       	sbrs	r24, 6
    1fb0:	83 c0       	rjmp	.+262    	; 0x20b8 <__vector_125+0x16a>
	udd_control_out_clear_NACK0();
}

static void udd_ctrl_underflow(void)
{
	if (udd_is_tc_event() || udd_ctrl_interrupt_tc_setup()) {
    1fb2:	80 91 cc 04 	lds	r24, 0x04CC	; 0x8004cc <__TEXT_REGION_LENGTH__+0x7004cc>
    1fb6:	81 fd       	sbrc	r24, 1
    1fb8:	7f c0       	rjmp	.+254    	; 0x20b8 <__vector_125+0x16a>
    1fba:	0e 94 6b 0b 	call	0x16d6	; 0x16d6 <udd_ctrl_interrupt_tc_setup>
    1fbe:	81 11       	cpse	r24, r1
    1fc0:	7b c0       	rjmp	.+246    	; 0x20b8 <__vector_125+0x16a>
		return; // underflow ignored if a transfer complete has been no processed
	}
	if (UDD_EPCTRL_DATA_OUT == udd_ep_control_state) {
    1fc2:	80 91 e4 22 	lds	r24, 0x22E4	; 0x8022e4 <udd_ep_control_state>
    1fc6:	81 30       	cpi	r24, 0x01	; 1
    1fc8:	19 f4       	brne	.+6      	; 0x1fd0 <__vector_125+0x82>
		// Host want to stop OUT transaction
		// then stop to wait OUT data phase and wait IN ZLP handshake
		udd_ctrl_send_zlp_in();
    1fca:	0e 94 a3 0a 	call	0x1546	; 0x1546 <udd_ctrl_send_zlp_in>
    1fce:	74 c0       	rjmp	.+232    	; 0x20b8 <__vector_125+0x16a>
	} else if (UDD_EPCTRL_HANDSHAKE_WAIT_OUT_ZLP == udd_ep_control_state) {
    1fd0:	84 30       	cpi	r24, 0x04	; 4
    1fd2:	09 f0       	breq	.+2      	; 0x1fd6 <__vector_125+0x88>
    1fd4:	71 c0       	rjmp	.+226    	; 0x20b8 <__vector_125+0x16a>
		// A OUT handshake is waiting by device,
		// but host want extra IN data then stall extra IN data and following status stage
		udd_control_in_enable_stall();
    1fd6:	ed ef       	ldi	r30, 0xFD	; 253
    1fd8:	f2 e2       	ldi	r31, 0x22	; 34
    1fda:	04 e0       	ldi	r16, 0x04	; 4
    1fdc:	05 93       	las	Z, r16
		udd_control_out_enable_stall();
    1fde:	e5 ef       	ldi	r30, 0xF5	; 245
    1fe0:	f2 e2       	ldi	r31, 0x22	; 34
    1fe2:	04 e0       	ldi	r16, 0x04	; 4
    1fe4:	05 93       	las	Z, r16
    1fe6:	68 c0       	rjmp	.+208    	; 0x20b8 <__vector_125+0x16a>
			udd_ctrl_underflow();
		}
		return true;
	}
	// Overflow only managed for control endpoint
	if (udd_is_overflow_event()) {
    1fe8:	80 91 cb 04 	lds	r24, 0x04CB	; 0x8004cb <__TEXT_REGION_LENGTH__+0x7004cb>
    1fec:	81 ff       	sbrs	r24, 1
    1fee:	5f c0       	rjmp	.+190    	; 0x20ae <__vector_125+0x160>
		udd_ack_overflow_event();
    1ff0:	82 e0       	ldi	r24, 0x02	; 2
    1ff2:	80 93 ca 04 	sts	0x04CA, r24	; 0x8004ca <__TEXT_REGION_LENGTH__+0x7004ca>
		if (udd_control_out_overflow()) {
    1ff6:	80 91 f4 22 	lds	r24, 0x22F4	; 0x8022f4 <udd_sram+0xc>
    1ffa:	86 ff       	sbrs	r24, 6
    1ffc:	5d c0       	rjmp	.+186    	; 0x20b8 <__vector_125+0x16a>
	}
}

static void udd_ctrl_overflow(void)
{
	if (udd_is_tc_event() || udd_ctrl_interrupt_tc_setup()) {
    1ffe:	80 91 cc 04 	lds	r24, 0x04CC	; 0x8004cc <__TEXT_REGION_LENGTH__+0x7004cc>
    2002:	81 fd       	sbrc	r24, 1
    2004:	59 c0       	rjmp	.+178    	; 0x20b8 <__vector_125+0x16a>
    2006:	0e 94 6b 0b 	call	0x16d6	; 0x16d6 <udd_ctrl_interrupt_tc_setup>
    200a:	81 11       	cpse	r24, r1
    200c:	55 c0       	rjmp	.+170    	; 0x20b8 <__vector_125+0x16a>
		return; // overflow ignored if a transfer complete has been no processed
	}
	if (UDD_EPCTRL_DATA_IN == udd_ep_control_state) {
    200e:	80 91 e4 22 	lds	r24, 0x22E4	; 0x8022e4 <udd_ep_control_state>
    2012:	82 30       	cpi	r24, 0x02	; 2
    2014:	41 f4       	brne	.+16     	; 0x2026 <__vector_125+0xd8>
	udd_control_in_clear_NACK0();
}

static void udd_ctrl_send_zlp_out(void)
{
	udd_ep_control_state = UDD_EPCTRL_HANDSHAKE_WAIT_OUT_ZLP;
    2016:	84 e0       	ldi	r24, 0x04	; 4
    2018:	80 93 e4 22 	sts	0x22E4, r24	; 0x8022e4 <udd_ep_control_state>
	// Valid reception of OUT packet on control endpoint
	udd_control_out_clear_NACK0();
    201c:	e4 ef       	ldi	r30, 0xF4	; 244
    201e:	f2 e2       	ldi	r31, 0x22	; 34
    2020:	02 e0       	ldi	r16, 0x02	; 2
    2022:	06 93       	lac	Z, r16
    2024:	49 c0       	rjmp	.+146    	; 0x20b8 <__vector_125+0x16a>
	}
	if (UDD_EPCTRL_DATA_IN == udd_ep_control_state) {
		// Host want to stop IN transaction
		// then stop to wait IN data phase and wait OUT ZLP handshake
		udd_ctrl_send_zlp_out();
	} else if (UDD_EPCTRL_HANDSHAKE_WAIT_IN_ZLP == udd_ep_control_state) {
    2026:	83 30       	cpi	r24, 0x03	; 3
    2028:	09 f0       	breq	.+2      	; 0x202c <__vector_125+0xde>
    202a:	46 c0       	rjmp	.+140    	; 0x20b8 <__vector_125+0x16a>
		// A IN handshake is waiting by device,
		// but host want extra OUT data then stall extra OUT data and following status stage
		udd_control_in_enable_stall();
    202c:	ed ef       	ldi	r30, 0xFD	; 253
    202e:	f2 e2       	ldi	r31, 0x22	; 34
    2030:	04 e0       	ldi	r16, 0x04	; 4
    2032:	05 93       	las	Z, r16
		udd_control_out_enable_stall();
    2034:	e5 ef       	ldi	r30, 0xF5	; 245
    2036:	f2 e2       	ldi	r31, 0x22	; 34
    2038:	04 e0       	ldi	r16, 0x04	; 4
    203a:	05 93       	las	Z, r16
    203c:	3d c0       	rjmp	.+122    	; 0x20b8 <__vector_125+0x16a>

	if (udd_ctrl_interrupt_error()) {
		goto udd_interrupt_bus_event_end;
	}
	if (udd_is_reset_event()) {
		udd_ack_reset_event();
    203e:	80 e1       	ldi	r24, 0x10	; 16
    2040:	80 93 ca 04 	sts	0x04CA, r24	; 0x8004ca <__TEXT_REGION_LENGTH__+0x7004ca>
#if (0!=USB_DEVICE_MAX_EP)
		// Abort all endpoint jobs on going
		uint8_t i;
		for (i = 1; i < USB_DEVICE_MAX_EP; i++) {
			udd_ep_abort(i);
    2044:	81 e0       	ldi	r24, 0x01	; 1
    2046:	0e 94 22 0f 	call	0x1e44	; 0x1e44 <udd_ep_abort>
			udd_ep_abort(i | USB_EP_DIR_IN);
    204a:	81 e8       	ldi	r24, 0x81	; 129
    204c:	0e 94 22 0f 	call	0x1e44	; 0x1e44 <udd_ep_abort>
		}
#endif
		udc_reset();
    2050:	0e 94 51 06 	call	0xca2	; 0xca2 <udc_reset>

		// Reset USB address to 0
		udd_set_device_address(0);
    2054:	10 92 c3 04 	sts	0x04C3, r1	; 0x8004c3 <__TEXT_REGION_LENGTH__+0x7004c3>
#endif
	}

	// Enable endpoint
	ep_ctrl = udd_ep_get_ctrl(ep);
	udd_endpoint_disable(ep_ctrl);
    2058:	e8 ee       	ldi	r30, 0xE8	; 232
    205a:	f2 e2       	ldi	r31, 0x22	; 34
    205c:	15 86       	std	Z+13, r1	; 0x0d
	udd_endpoint_clear_status(ep_ctrl);
    205e:	96 e0       	ldi	r25, 0x06	; 6
    2060:	94 87       	std	Z+12, r25	; 0x0c
	udd_endpoint_set_control(ep_ctrl, (uint8_t) type | (uint8_t) size);
    2062:	83 e4       	ldi	r24, 0x43	; 67
    2064:	85 87       	std	Z+13, r24	; 0x0d
#endif
	}

	// Enable endpoint
	ep_ctrl = udd_ep_get_ctrl(ep);
	udd_endpoint_disable(ep_ctrl);
    2066:	15 8a       	std	Z+21, r1	; 0x15
	udd_endpoint_clear_status(ep_ctrl);
    2068:	94 8b       	std	Z+20, r25	; 0x14
	udd_endpoint_set_control(ep_ctrl, (uint8_t) type | (uint8_t) size);
    206a:	85 8b       	std	Z+21, r24	; 0x15
		udd_set_device_address(0);
		// Alloc and configure control endpoint
		udd_ep_init(0, USB_EP_TYPE_CONTROL, USB_DEVICE_EP_CTRL_SIZE);
		udd_ep_init(0 | USB_EP_DIR_IN, USB_EP_TYPE_CONTROL,
				USB_DEVICE_EP_CTRL_SIZE);
		udd_control_out_set_buf(&udd_ctrl_buffer);
    206c:	80 ea       	ldi	r24, 0xA0	; 160
    206e:	92 e2       	ldi	r25, 0x22	; 34
    2070:	80 8b       	std	Z+16, r24	; 0x10
    2072:	91 8b       	std	Z+17, r25	; 0x11
		// Reset endpoint control management
		udd_ctrl_init();
    2074:	0e 94 6e 0a 	call	0x14dc	; 0x14dc <udd_ctrl_init>
		goto udd_interrupt_bus_event_end;
    2078:	1f c0       	rjmp	.+62     	; 0x20b8 <__vector_125+0x16a>
	}

	if (udd_is_suspend_event()) {
    207a:	80 91 cb 04 	lds	r24, 0x04CB	; 0x8004cb <__TEXT_REGION_LENGTH__+0x7004cb>
    207e:	86 ff       	sbrs	r24, 6
    2080:	09 c0       	rjmp	.+18     	; 0x2094 <__vector_125+0x146>
		udd_ack_suspend_event();
    2082:	80 e4       	ldi	r24, 0x40	; 64
    2084:	80 93 ca 04 	sts	0x04CA, r24	; 0x8004ca <__TEXT_REGION_LENGTH__+0x7004ca>
		udd_sleep_mode(false); // Enter in SUSPEND mode
    2088:	80 e0       	ldi	r24, 0x00	; 0
    208a:	0e 94 36 0a 	call	0x146c	; 0x146c <udd_sleep_mode>
#ifdef UDC_SUSPEND_EVENT
		UDC_SUSPEND_EVENT();
    208e:	0e 94 84 11 	call	0x2308	; 0x2308 <main_suspend_action>
#endif
		goto udd_interrupt_bus_event_end;
    2092:	12 c0       	rjmp	.+36     	; 0x20b8 <__vector_125+0x16a>
	}

	if (udd_is_resume_event()) {
    2094:	80 91 cb 04 	lds	r24, 0x04CB	; 0x8004cb <__TEXT_REGION_LENGTH__+0x7004cb>
    2098:	85 ff       	sbrs	r24, 5
    209a:	0e c0       	rjmp	.+28     	; 0x20b8 <__vector_125+0x16a>
		udd_ack_resume_event();
    209c:	80 e2       	ldi	r24, 0x20	; 32
    209e:	80 93 ca 04 	sts	0x04CA, r24	; 0x8004ca <__TEXT_REGION_LENGTH__+0x7004ca>
		udd_sleep_mode(true); // Enter in power reduction mode
    20a2:	81 e0       	ldi	r24, 0x01	; 1
    20a4:	0e 94 36 0a 	call	0x146c	; 0x146c <udd_sleep_mode>
#ifdef UDC_RESUME_EVENT
		UDC_RESUME_EVENT();
    20a8:	0e 94 87 11 	call	0x230e	; 0x230e <main_resume_action>
#endif
		goto udd_interrupt_bus_event_end;
    20ac:	05 c0       	rjmp	.+10     	; 0x20b8 <__vector_125+0x16a>
	}

	if (udd_ctrl_interrupt_error()) {
		goto udd_interrupt_bus_event_end;
	}
	if (udd_is_reset_event()) {
    20ae:	80 91 cb 04 	lds	r24, 0x04CB	; 0x8004cb <__TEXT_REGION_LENGTH__+0x7004cb>
    20b2:	84 ff       	sbrs	r24, 4
    20b4:	e2 cf       	rjmp	.-60     	; 0x207a <__vector_125+0x12c>
    20b6:	c3 cf       	rjmp	.-122    	; 0x203e <__vector_125+0xf0>
		goto udd_interrupt_bus_event_end;
	}

udd_interrupt_bus_event_end:
	return;
}
    20b8:	ff 91       	pop	r31
    20ba:	ef 91       	pop	r30
    20bc:	bf 91       	pop	r27
    20be:	af 91       	pop	r26
    20c0:	9f 91       	pop	r25
    20c2:	8f 91       	pop	r24
    20c4:	7f 91       	pop	r23
    20c6:	6f 91       	pop	r22
    20c8:	5f 91       	pop	r21
    20ca:	4f 91       	pop	r20
    20cc:	3f 91       	pop	r19
    20ce:	2f 91       	pop	r18
    20d0:	0f 91       	pop	r16
    20d2:	0f 90       	pop	r0
    20d4:	0b be       	out	0x3b, r0	; 59
    20d6:	0f 90       	pop	r0
    20d8:	09 be       	out	0x39, r0	; 57
    20da:	0f 90       	pop	r0
    20dc:	08 be       	out	0x38, r0	; 56
    20de:	0f 90       	pop	r0
    20e0:	0f be       	out	0x3f, r0	; 63
    20e2:	0f 90       	pop	r0
    20e4:	1f 90       	pop	r1
    20e6:	18 95       	reti

000020e8 <__vector_126>:
 * \brief Function called by USB transfer complete interrupt
 *
 * USB transfer complete interrupt includes events about endpoint transfer on all endpoints.
 */
ISR(USB_TRNCOMPL_vect)
{
    20e8:	1f 92       	push	r1
    20ea:	0f 92       	push	r0
    20ec:	0f b6       	in	r0, 0x3f	; 63
    20ee:	0f 92       	push	r0
    20f0:	11 24       	eor	r1, r1
    20f2:	08 b6       	in	r0, 0x38	; 56
    20f4:	0f 92       	push	r0
    20f6:	18 be       	out	0x38, r1	; 56
    20f8:	09 b6       	in	r0, 0x39	; 57
    20fa:	0f 92       	push	r0
    20fc:	19 be       	out	0x39, r1	; 57
    20fe:	0a b6       	in	r0, 0x3a	; 58
    2100:	0f 92       	push	r0
    2102:	1a be       	out	0x3a, r1	; 58
    2104:	0b b6       	in	r0, 0x3b	; 59
    2106:	0f 92       	push	r0
    2108:	1b be       	out	0x3b, r1	; 59
    210a:	0f 93       	push	r16
    210c:	1f 93       	push	r17
    210e:	2f 93       	push	r18
    2110:	3f 93       	push	r19
    2112:	4f 93       	push	r20
    2114:	5f 93       	push	r21
    2116:	6f 93       	push	r22
    2118:	7f 93       	push	r23
    211a:	8f 93       	push	r24
    211c:	9f 93       	push	r25
    211e:	af 93       	push	r26
    2120:	bf 93       	push	r27
    2122:	cf 93       	push	r28
    2124:	df 93       	push	r29
    2126:	ef 93       	push	r30
    2128:	ff 93       	push	r31
	int8_t rp;
	UDD_EP_t *ep_ctrl;
	udd_ep_id_t ep;
#endif

	if (!udd_is_tc_event()) {
    212a:	80 91 cc 04 	lds	r24, 0x04CC	; 0x8004cc <__TEXT_REGION_LENGTH__+0x7004cc>
    212e:	81 fd       	sbrc	r24, 1
    2130:	04 c0       	rjmp	.+8      	; 0x213a <__vector_126+0x52>
		// If no other transfer complete
		// then check reception of SETUP packet on control endpoint
		if (udd_ctrl_interrupt_tc_setup()) {
    2132:	0e 94 6b 0b 	call	0x16d6	; 0x16d6 <udd_ctrl_interrupt_tc_setup>
    2136:	81 11       	cpse	r24, r1
    2138:	ca c0       	rjmp	.+404    	; 0x22ce <__vector_126+0x1e6>
			goto udd_interrupt_tc_end;
		}
		Assert(false);
	}
	// Check IN/OUT transfer complete on all endpoints
	udd_ack_tc_event();
    213a:	82 e0       	ldi	r24, 0x02	; 2
    213c:	80 93 cc 04 	sts	0x04CC, r24	; 0x8004cc <__TEXT_REGION_LENGTH__+0x7004cc>

#if (0!=USB_DEVICE_MAX_EP)
	//** Decode TC FIFO
	// Compute ep addr
	rp = udd_get_fifo_rp();
    2140:	80 91 c5 04 	lds	r24, 0x04C5	; 0x8004c5 <__TEXT_REGION_LENGTH__+0x7004c5>
	i_fifo = 2 * (1 + ~rp);
    2144:	81 95       	neg	r24
    2146:	88 0f       	add	r24, r24
	ad = ((uint16_t) udd_sram.ep_ctrl) - i_fifo;
    2148:	e4 ef       	ldi	r30, 0xF4	; 244
    214a:	f2 e2       	ldi	r31, 0x22	; 34
    214c:	e8 1b       	sub	r30, r24
    214e:	f1 09       	sbc	r31, r1
	p_ad = (uint16_t *) ad;
	// Compute ep
	ep_index = (((uint16_t) * p_ad - ((uint16_t) udd_sram.ep_ctrl)) >> 3);
    2150:	20 81       	ld	r18, Z
    2152:	31 81       	ldd	r19, Z+1	; 0x01
    2154:	24 5f       	subi	r18, 0xF4	; 244
    2156:	32 42       	sbci	r19, 0x22	; 34
    2158:	36 95       	lsr	r19
    215a:	27 95       	ror	r18
    215c:	36 95       	lsr	r19
    215e:	27 95       	ror	r18
    2160:	36 95       	lsr	r19
    2162:	27 95       	ror	r18
	ep = (ep_index / 2) + ((ep_index & 1) ? USB_EP_DIR_IN : 0);
    2164:	82 2f       	mov	r24, r18
    2166:	86 95       	lsr	r24
    2168:	20 fd       	sbrc	r18, 0
    216a:	02 c0       	rjmp	.+4      	; 0x2170 <__vector_126+0x88>
    216c:	90 e0       	ldi	r25, 0x00	; 0
    216e:	01 c0       	rjmp	.+2      	; 0x2172 <__vector_126+0x8a>
    2170:	90 e8       	ldi	r25, 0x80	; 128
    2172:	89 0f       	add	r24, r25
	udd_endpoint_set_control(ep_ctrl, (uint8_t) type | (uint8_t) size);
}

static UDD_EP_t *udd_ep_get_ctrl(udd_ep_id_t ep)
{
	return &udd_sram.ep_ctrl[(2 * (ep & USB_EP_ADDR_MASK) +
    2174:	e8 2f       	mov	r30, r24
    2176:	ef 70       	andi	r30, 0x0F	; 15
    2178:	f0 e0       	ldi	r31, 0x00	; 0
    217a:	ee 0f       	add	r30, r30
    217c:	ff 1f       	adc	r31, r31
			((ep & USB_EP_DIR_IN) ? 1 : 0))];
    217e:	28 2f       	mov	r18, r24
    2180:	08 2e       	mov	r0, r24
    2182:	00 0c       	add	r0, r0
    2184:	33 0b       	sbc	r19, r19
    2186:	22 27       	eor	r18, r18
    2188:	33 0f       	add	r19, r19
    218a:	22 1f       	adc	r18, r18
    218c:	33 27       	eor	r19, r19
	udd_endpoint_set_control(ep_ctrl, (uint8_t) type | (uint8_t) size);
}

static UDD_EP_t *udd_ep_get_ctrl(udd_ep_id_t ep)
{
	return &udd_sram.ep_ctrl[(2 * (ep & USB_EP_ADDR_MASK) +
    218e:	e2 0f       	add	r30, r18
    2190:	f3 1f       	adc	r31, r19
	ep = (ep_index / 2) + ((ep_index & 1) ? USB_EP_DIR_IN : 0);
	Assert(USB_DEVICE_MAX_EP >= (ep & USB_EP_ADDR_MASK));

	// Ack IT TC of endpoint
	ep_ctrl = udd_ep_get_ctrl(ep);
	if (!udd_endpoint_transfer_complete(ep_ctrl)) {
    2192:	df 01       	movw	r26, r30
    2194:	aa 0f       	add	r26, r26
    2196:	bb 1f       	adc	r27, r27
    2198:	aa 0f       	add	r26, r26
    219a:	bb 1f       	adc	r27, r27
    219c:	aa 0f       	add	r26, r26
    219e:	bb 1f       	adc	r27, r27
    21a0:	a8 51       	subi	r26, 0x18	; 24
    21a2:	bd 4d       	sbci	r27, 0xDD	; 221
    21a4:	1c 96       	adiw	r26, 0x0c	; 12
    21a6:	9c 91       	ld	r25, X
    21a8:	95 ff       	sbrs	r25, 5
    21aa:	91 c0       	rjmp	.+290    	; 0x22ce <__vector_126+0x1e6>
